:100000000C94C4080C94E3080C94E3080C94730952
:100010000C94A9090C94E3080C94E3080C94E308ED
:100020000C94E3080C94E3080C94E3080C94E308A4
:100030000C94E3080C94E3080C94E3080C94D30CA0
:100040000C94E3080C94E3080C94E3080C94E30884
:100050000C948E650C944E5D0C94E3080C94E308AC
:100060000C94E3080C94235E0C94E3080C94175E44
:100070000C94E3080C94E3080C94E3080C94E30854
:100080000C94C1700C94E3080C94E3080C94E308FE
:100090000C94615E0C94E3080C94555E0C94E30898
:1000A0000C94E3080C94E3080C94E3080C94E30824
:1000B0000C94E3080C94E3080C94E3080C94E30814
:1000C0000C94E3080C94E3080C94E3080C94E30804
:1000D0000C94E3080C94E3080C94E3080C94E308F4
:1000E0000C94E3080C9447650C9451650C943D65A1
:1000F0000C94FD640C9482650C9473650C94676594
:100100000C945B650C94E3080C94E3080C94E308EE
:100110000C94E3080C94E3080C94E3080C94E308B3
:10012000FA79197A987A877BA77BC77BCF7B7C7B10
:10013000084AD73B3BCE016E84BCBFFDC12F3D6C4E
:1001400074319ABD56833DDA3D00C77F11BED9E4B4
:10015000BB4C3E916BAAAABE000000803F076342E1
:1001600036B79BD8A71A39685618AEBAAB558C1D4E
:100170003CB7CC5763BD6DEDFD753EF6177231BFD0
:10018000000000803F08000000BE922449123EABF0
:10019000AAAA2ABECDCCCC4C3E00000080BEABAAA1
:1001A000AAAA3E00000000BF000000803F0000003F
:1001B0000000084178D3BB4387D1133D190E3CC3DF
:1001C000BD4282AD2B3E68EC8276BED98FE1A93E5E
:1001D0004C80EFFFBE01C4FF7F3F00000000002500
:1001E000730A005854414C5F5452494D3D256400F8
:1001F00025730A0025730A00546573742036202580
:10020000730A005465737420352025730A00546501
:10021000737420342025730A0054657374203320CE
:1002200025730A005465737420322025730A005424
:1002300065737420312025730A006368616E3D2563
:10024000640A0074787077723D25640A0035303096
:100250006B0A003235306B0A003131356B0A0035DC
:10026000366B0A0033386B0A0025730A0073656E1B
:10027000743D252D75206475703D252D75206967A9
:100280006E6F7265643D252D752074746C5F7A65A0
:10029000726F3D252D750A0025372E3366202537D0
:1002A0002E33660025352E326620004572726F723D
:1002B000203020566F6C74004E6F74207375707010
:1002C0006F727465640A004572726F722030205636
:1002D0006F6C74004572726F72203020566F6C74B0
:1002E0000025630074746C3D252D64200074746CCB
:1002F0003D252D6420004E65772074746C3D252DBE
:100300006420002563004D533536313120503D25A2
:100310002D372E326620252D372E32666D0A00428B
:100320004D5030383520256C642050612020252D1B
:10033000372E32666D00256300545F484541545F97
:100340004944583D252D352E32662000545F4445E2
:10035000573D252D352E3266200041483D252D354F
:100360002E32662000545F53485432583D252D35B7
:100370002E3266200052485F53485432583D252D96
:10038000352E32662000545F52483D252D342E31E3
:1003900066200052483D252D342E3166200025630D
:1003A0000025630025630025630043757272656E46
:1003B00074207265706F727420696E7465727661F4
:1003C0006C3D252D75207365630A004E657720729C
:1003D00065706F727420696E74657276616C3D250C
:1003E0002D75207365630A002563007265706F7256
:1003F000745F616C6C3D007265706F72743D0025B6
:100400006300256300256300256300204F534343A9
:10041000414C3D2564200020467573653A20656592
:100420003D253032782068663D25303278206C6674
:100430003D25303278206C623D25303278004D43C6
:10044000553D2530366C7800256300252D31306C04
:100450007520252D31306C7520252D31306C75209F
:10046000252D31306C75200A007478206C656E2063
:10047000202020207268206D697373202020207254
:1004800068207374616C652020207268206D697328
:10049000630A002563004F4B0A00256300256300B3
:1004A000256300256300256300256300646562758C
:1004B000675F616C6C3D0064656275673D006465F3
:1004C0006275673D0025730A00646565700A006EF9
:1004D0006F6E650A00707772733D00696E74725FAB
:1004E0007365635F70313D252D372E33660A0069D1
:1004F0006E74725F70313D252D6C640A00696E74F4
:10050000725F7365635F70303D252D372E33660A49
:1005100000696E74725F70303D252D6C640A007640
:100520005F6D63753D252D352E32660A007070773C
:10053000723D25730A0064656275673D0025730A84
:10054000006175746F0A006C6F675F6D6F64653D65
:10055000007573625F7077723D25730A0072657073
:100560006F72743D007265706F72745F696E74654E
:100570007276616C3D252D750A0072656C61793D5E
:1005800025730A0074746C3D252D640A0052494D90
:10059000455F616464723D252D642E252D640A003B
:1005A0006E65696768626F725F7461626C655F73C4
:1005B000697A653D25640A00747870773D25640A80
:1005C000006368616E3D25640A006932633D00691D
:1005D000643D007478743D25730A00537973746523
:1005E0006D2053756D6D6172790A00745F68656185
:1005F000745F69647800745F646577006168007097
:100600005F6D73353631310072685F7368743278AC
:1006100000745F7368743278007061007000616408
:10062000340061643300616432006164310061331D
:1006300000613200613100765F696E00726800759A
:100640007074696D650070315F6C73740070315F38
:10065000740070310070305F6C73740070305F74C0
:1006600000703000765F6D637500745F6D637500B8
:100670007431007400696400653634007478740065
:100680002D002B006175746F006E6F6E6500706FCA
:100690007765725F736176655F6C6564727900720D
:1006A000656C61795F6C65647900636F6D7061730F
:1006B0007300616363656C007072657300705F70D6
:1006C0007772006165730070315F6C6564790070EA
:1006D000305F6C656472006576656E74006C65648D
:1006E000006F7700706B740074785F6C65647900DC
:1006F00072785F6C656472006F706572006E6F6E09
:1007000065002530327800765F6164343D252D38F0
:100710002E3666002000765F6164333D252D382E2D
:100720003666002000765F6164323D252D382E3616
:1007300066002000765F6164313D252D382E3666D7
:10074000002000765F6C696768743D252D382E3671
:1007500066002000765F61323D252D372E3366001E
:100760002000765F61313D252D372E336600200055
:10077000765F696E3D252D352E326600204E6576FA
:1007800065722D7573656420737461636B203E2000
:1007900025642062797465730A00757074696D65EB
:1007A0003D252D642D646179732D253032643A2501
:1007B0003032643A253032642D686F7572730A00E6
:1007C00074657374205B6F66667C317C327C337C2D
:1007D000347C355D20202020202020202D207465B1
:1007E0007374206D6F6465730A0D00263A205B54A4
:1007F0005820504B5420434F4E54454E545D2020BA
:10080000202020202020202D2073656E6420706B16
:10081000742066726F6D20636D646C696E652F6302
:100820006861740A0D00776474205B6F6E7C6F667C
:10083000667C746573745D20202020202020202099
:1008400020202D207761746368646F670A0D00753E
:1008500070677220202020202020202020202020AF
:1008600020202020202020202020202D20726562A2
:100870006F6F742076696120626F6F746C6F616452
:1008800065720A0D0075617274205B33386B7C35BC
:10089000366B7C3131356B7C3235306B7C353030AA
:1008A0006B5D202D20736574207465726D2F7561EA
:1008B00072742073706565640A0D00626F6F742036
:1008C0002020202020202020202020202020202028
:1008D000202020202020202D207265626F6F740A56
:1008E0000D0070777273205B646565707C6E6F6E4F
:1008F000655D2020202020202020202020202D2069
:100900006D637520736C656570206D6F64650A0D8D
:10091000007265737420656570726F6D20202020F1
:10092000202020202020202020202020202D207268
:100930006573746F726520656570726F6D0A0D0066
:1009400070707772205B6F6E7C6F66665D20202012
:100950002020202020202020202020202D207072E8
:100960006F6772616D6D61626C65207077720A0DE0
:1009700000747874205B737472696E675D20202048
:10098000202020202020202020202020202D205327
:100990006574207265706F7274207465787420734A
:1009A0007472696E670A0D0074787077205B313558
:1009B0002D305D20202020202020202020202020DD
:1009C000202020202D205458205077722E20486956
:1009D0006768657374203020283364426D290A0DDE
:1009E0000074746C205B302D31355D202020202078
:1009F000202020202020202020202020202D207496
:100A0000696D652D746F2D6C69766520666F722037
:100A10007061636B6574730A0D007373202020206E
:100A200020202020202020202020202020202020C6
:100A30002020202020202D2073797374656D207371
:100A4000756D6D6172790A0D00727320202020206F
:100A50002020202020202020202020202020202096
:100A600020202020202D20726164696F2073746122
:100A700074730A0D007269205B696E745D2020201A
:100A80002020202020202020202020202020202066
:100A9000202D207265706F727420696E7465727695
:100AA000616C0A0D007265205B2B7C2D5D205B6DF7
:100AB00061736B7C6175746F2C6D61736B5D20204D
:100AC000202D206D6F7465207265706F72742073B5
:100AD00065742F6D6F646966790A0D006F77202049
:100AE0002020202020202020202020202020202006
:100AF00020202020202020202D206F6E652D77695A
:100B000072652073656E736F72730A0D006C6F6788
:100B1000205B6175746F7C6F6E7C6F66665D2020F4
:100B20002020202020202020202D206D6F74657330
:100B30002064617461206F6E205553420A0D006E6F
:100B400065205B666C7573685D2020202020202066
:100B500020202020202020202020202D206E6569AC
:100B60006768626F72207461626C650A0D0065725D
:100B70007220202020202020202020202020202023
:100B8000202020202020202020202D206572726F20
:100B90007220696E666F0A0D006D6375202020203B
:100BA0002020202020202020202020202020202045
:100BB00020202020202D206D637520696E666F0A2D
:100BC0000D006964205B72657365745D20202020D0
:100BD00020202020202020202020202020202D2008
:100BE00069642068616E646C696E670A0D006875DF
:100BF0006D202020202020202020202020202020A8
:100C0000202020202020202020202D2068756D69A4
:100C1000646974792073656E736F720A0D00726572
:100C20006C6179205B6F6E7C6F66667C7374617437
:100C3000735D20202020202020202D2072656C61F3
:100C400079206E6574776F726B207265706F727445
:100C5000730A0D006465205B6D61736B5D2020205D
:100C60002020202020202020202020202020202084
:100C70002D2064656275670A0D006368616E205BF4
:100C800031312D32365D20202020202020202020D0
:100C90002020202020202D206368616E2031312DFE
:100CA00032362028322E3430352D32343830204D33
:100CB000687A290A0D0063616C69205B5B765F6965
:100CC0006E7C61317C61325D20766F6C747C726504
:100CD0007365747C6E6F6E655D202D2063616C6939
:100CE00062726174650A0D00616463202020202017
:100CF00020202020202020202020202020202020F4
:100D0000202020202D2073686F7720765F696E2C5D
:100D10002061312C20613220766F6C7461676573BD
:100D20000A0D0075202020202020202020202020B7
:100D30002020202020202020202020202020202DA6
:100D400020757074696D650A0D00762020202020C2
:100D50002020202020202020202020202020202093
:100D60002020202020202D2076657273696F6E0A66
:100D70000D0068202020202020202020202020205E
:100D800020202020202020202020202020202D2056
:100D900068656C700A0D00256300756E6B6E6F7769
:100DA0006E20636D640A00484D43353838330025A2
:100DB0007300257300202573002025362E3266200F
:100DC00000253032780074656D705F6578746572E7
:100DD0006E3D252D362E32660020257300202536E7
:100DE0002E3266204F6E2D426F61726400253032C4
:100DF000780074656D705F626F6172643D252D3699
:100E00002E3266000A00503A20256C642050612082
:100E100020252D372E3266206D0A002563002563BC
:100E2000004932433A2000452025642E2564206382
:100E30006C6F636B20256C752063707520256C7555
:100E4000206C706D20256C752069727120256C7581
:100E500020676C656420256C7520796C656420259D
:100E60006C7520726C656420256C75207478202563
:100E70006C75206C697374656E20256C75207365C4
:100E80006E736F727320256C752073657269616C67
:100E900020256C750A00532025642E256420636C80
:100EA0006F636B20256C7520747820256C7520721B
:100EB0007820256C752072747820256C75207272EC
:100EC0007820256C75207265786D697420256C75A5
:100ED0002061636B747820256C75206E6F61636B85
:100EE000747820256C752061636B727820256C7591
:100EF0002074696D65646F757420256C752062615E
:100F00006461636B727820256C7520746F6F6C6FF1
:100F10006E6720256C7520746F6F73686F72742014
:100F2000256C752062616473796E636820256C7529
:100F30002062616463726320256C7520636F6E7438
:100F4000656E74696F6E64726F7020256C752073A6
:100F5000656E64696E6764726F7020256C75206CB5
:100F60006C747820256C75206C6C727820256C75FB
:100F70000A00257325730A004F6E6C696E650A00BE
:100F80000A002C20636865636B20726174652025FC
:100F90007520487A0025732025732C206368616EC4
:100FA0006E656C20257520706F7765722025750041
:100FB0000A0025783A004D414320616464726573EC
:100FC00073200052616E646F6D20455549363420A0
:100FD000616464726573732067656E6572617465C0
:100FE000640A000A2A2A2A2A2A2A2A426F6F746966
:100FF0006E672025732A2A2A2A2A2A2A0A004545AA
:1010000050524F4D20697320636F72727570742C4B
:1010100020726577726974696E67207769746820D9
:1010200064656661756C74732E0A006C6F63616C25
:10103000686F73740041544D4547413132387266D0
:10104000613100020000FFFE0000016E616E006968
:101050006E660000407A10F35A00A0724E18090024
:1010600010A5D4E80000E87648170000E40B54020D
:101070000000CA9A3B000000E1F505000080969848
:1010800000000040420F000000A086010000001098
:101090002700000000E803000000006400000000DA
:1010A000000A00000000000100000000002C76D8BB
:1010B00088DC674F0823DFC1DFAE59E1B1B796E5A1
:1010C000E3E453C63AE651997696E8E6C28426EB05
:1010D000898C9B62ED407C6FFCEFBC9C9F40F2BA18
:1010E000A56FA5F490055A2AF75C936B6CF9676DB0
:1010F000C11BFCE0E40D47FEF520E6B500D0ED9005
:101100002E0300943577050080841E080000204ED1
:101110000A000000C80C333333330F986E1283116A
:1011200041EF8D2114893BE65516CFFEE6DB18D141
:10113000844B381BF77C1D901DA4BBE42420328413
:10114000725E228100C9F124ECA1E53D274E414E9B
:10115000494E495459494E46CDCCCC3D0AD7233C43
:1011600017B7D13877CC2B329595E6241FB14F0AAB
:10117000000020410000C84200401C4620BCBE4C7C
:10118000CA1B0E5AAEC59D7411241FBECFEFD1E409
:10119000DEBFCDBF19E0A0E0B2E0EAEEFCE101E085
:1011A0000BBF02C007900D92A234B107D9F710E32C
:1011B000A2E4B9E001C01D92A93CB107E1F70E9489
:1011C0009E7C0C94738E0C94000085ED94E09F93AC
:1011D0008F930E947B8B80914A0290914B020F90DB
:1011E0000F9093FF03C08FEC94E002C089EC94E071
:1011F0009F938F930E947B8B0F900F900895E091A7
:10120000D71AEF71F0E0E45DF44E80838091D71A35
:101210008F5F8093D71A809103288860809303287A
:1012200044E352E061E1CA010E943D4D80E090E05C
:101230000895CF93DF93EC018091490990914A0979
:1012400086FF1DC08E811F928F938D811F928F9379
:101250008C811F928F938B811F928F938A811F9213
:101260008F9386E593E09F938F930E94698B8DB750
:101270009EB70C960FB6F8949EBF0FBE8DBFBE01F1
:1012800080E899E00E946F4EBE0184E092E0DF9119
:10129000CF910C94E44D87EE93E08115910511F008
:1012A0000197F1F708958823B9F052985A981DBA1A
:1012B00080916900806280936900EA9A53985B98F4
:1012C000EB9A809169008068809369008091680042
:1012D0008160809368000895109269005A9AEA9894
:1012E0005B9AEB9808951F920F920FB60F921124FC
:1012F0008F939F93AF93BF938091680080FF20C02E
:101300008091E3279091E427A091E527B091E6270B
:101310000196A11DB11D8093E3279093E427A0932C
:10132000E527B093E6278091490990914A0987FF04
:1013300007C0749882E090E090937A0280937902DB
:10134000BF91AF919F918F910F900FBE0F901F9003
:1013500018951F920F920FB60F9211248F939F939F
:10136000AF93BF938091680080FF20C08091E727F2
:101370009091E827A091E927B091EA270196A11D55
:10138000B11D8093E7279093E827A093E927B093B6
:10139000EA278091490990914A0990FF07C0739804
:1013A00082E090E090937A0280937902BF91AF91AE
:1013B0009F918F910F900FBE0F901F901895809363
:1013C0007C0080917B00877F80937B0080917C00F4
:1013D000806C80937C0085E080937A0080917A0015
:1013E000806880937A0080917B0087FFFCCF80919A
:1013F0007B0085FFFCCF80917A00806480937A0027
:1014000080917A0086FDFCCF1092790010927800CE
:1014100084E090E060E070E020917A002064209306
:101420007A0020917A0026FDFCCF2091780030913F
:101430007900620F731F0197009771F710927C007B
:1014400080917A008F7780937A007695679576956C
:10145000679580E090E00E94F481089580E00E940A
:10146000DF09209175023091760240917702509108
:1014700078020E94D48321EE3AE744E95EE30E94B9
:101480008D80089580E18093510160E16093510166
:101490008091510185FF03C06F5F6F31B9F78BE415
:1014A000689FB0011124882777FD8095982F0E94AE
:1014B000F68120E030E64FE954E40E948D8020E080
:1014C00030E04AE754E40E9457810895CF93DF93B8
:1014D000EC0188819981009799F081309F4021F03B
:1014E0001982188283E011C0623171F40E94420AAD
:1014F00060937F2370938023809381239093822332
:1015000081E09FE09983888381E0DF91CF91089506
:1015100065FF4BC080917B00886080937B0089ECE5
:1015200080937C0085E080937A0080917A008068C7
:1015300080937A0080917B0087FFFCCF80917B00B5
:1015400085FFFCCF80917A00806480937A0080913F
:101550007A0086FDFCCF80917A00806480937A00C7
:1015600080917A0086FDFCCF6091780070917900BF
:1015700080E090E00E94F48127ED33EA40E95FE3E8
:101580000E94D48326E636E648E853E40E948C8025
:1015900060939C1A70939D1A80939E1A90939F1A41
:1015A00080917A008F7780937A000895BF92CF92CE
:1015B000DF92EF92FF920F931F93CF93DF93CDB7FC
:1015C000DEB729970FB6F894DEBF0FBECDBF6C0112
:1015D000109242098FEF898708EE1AE1B12C7E0143
:1015E00089E0E80EF11C89858823E9F1E8E0BE1660
:1015F000E1F1BE016F5F7F4FC7010E94D856898518
:101600008F3F11F08E3F19F4809342092CC0CE0118
:101610000196C114D10471F40E94F1568093002800
:10162000FE013196A8EFB7E281918D93EE15FF058B
:10163000D9F71DC00E94F156F8018083FE01319652
:1016400020E030E0A801485051098191DA01A20F51
:10165000B31F8C932F5F3F4F28303105B1F7B39400
:10166000075F1F4FC0CF8B2D03C088E001C081E012
:1016700029960FB6F894DEBF0FBECDBFDF91CF9194
:101680001F910F91FF90EF90DF90CF90BF90089542
:1016900084E09EE09F938F930E947B8B0F900F902E
:1016A00008952F923F924F925F926F927F928F9206
:1016B0009F92AF92BF92CF92DF92EF92FF920F93E1
:1016C0001F93CF93DF93EC014B01009711F427E0B8
:1016D00004C08130910549F426E04AE250E06BE213
:1016E00070E089E290E00E94B855CE010E94D60ACF
:1016F0009E012D5B364F5901D9018C93CD2B69F09A
:1017000098EEC92E9AE1D92EC0EEDAE1E12CF12C47
:1017100025EB222E2DE0322EA6C088EF97E20E9404
:101720002658BC01882777FD8095982F0E94F68166
:101730006B017C01892869F020E030E048EC52E43C
:101740000E9457819F938F937F936F9382EF9DE0C9
:10175000ACC0C8EFD7E20DEE1DE089911F928F93C8
:101760001F930F930E947B8B0F900F900F900F9001
:10177000B8E2C030DB0789F720E030E048EC52E403
:10178000C701B6010E9457819F938F937F936F93F8
:101790008DED9DE09F938F930E947B8B0F900F9018
:1017A0000F900F900F900F9080910028882319F0D0
:1017B00085E893E002C089EF93E09F938F9389EDD2
:1017C0009DE09F938F930E947B8B0F900F900F90C3
:1017D0000F9075C000E010E0FE01E00FF11F808166
:1017E0001F928F93A1ECBDE0BF93AF930E947B8BC0
:1017F0000F5F1F4F0F900F900F900F900830110543
:1018000059F720E030E048EC52E4C301B2010E94F5
:1018100057819F938F937F936F93A9EBBDE0BF9305
:10182000AF930E947B8B0F900F900F900F900F90B3
:101830000F90D6018C91882309F455C085E893E078
:101840009F938F933F922F920E947B8B0E94480B15
:10185000BFEFEB1AFB0AE9E0CE0ED11C29960F90E0
:101860000F900F900F90D5018C9190E0E816F9063B
:10187000ECF5CE010E942658BC01882777FD8095A3
:10188000982F0E94F6812B013C018114910409F4E8
:10189000A1CF20E030E048EC52E40E9457819F93B2
:1018A0008F937F936F9386EC9DE09F938F930E941D
:1018B0007B8B0F900F900F900F900F900F90DF91F8
:1018C000CF911F910F91FF90EF90DF90CF90BF903D
:1018D000AF909F908F907F906F905F904F903F90D0
:1018E0002F900C94480B89EF93E0AACFDF91CF9112
:1018F0001F910F91FF90EF90DF90CF90BF90AF902E
:101900009F908F907F906F905F904F903F902F901F
:101910000895CF93DF9300D0CDB7DEB78091F9273C
:1019200089838091FF278A83CE0101960E94314BE3
:101930000F900F90DF91CF910895CF93DF93EC013B
:101940002091F8273091F9274091FA275091FB27F1
:101950006091FC277091FD278091FE279091FF27D1
:10196000AFEF0E940487E1F427E04AE250E06BE227
:1019700070E089E290E00E94B85580E090E00E941B
:10198000D60ACD5BD64F888349E050E06AE070E02C
:1019900088EF97E20E94BE8CDF91CF910C94890C66
:1019A000DF91CF9108951F920F920FB60F921124DD
:1019B0000BB60F922F933F934F935F936F937F9349
:1019C0008F939F93AF93BF93CF93EF93FF938091A8
:1019D000032882608093032880914A0286FD2B9A17
:1019E00080914A0287FD2B9A8091790290917A0228
:1019F0001816190614F4749A739A809149099091F3
:101A00004A0985FF02C074987398809102029091F0
:101A1000030201979093030280930202892B09F03D
:101A200050C1809157099091580901969093580997
:101A3000809357098091832390918423A0918523DB
:101A4000B09186230196A11DB11D809383239093AD
:101A50008423A0938523B093862380E190E0909324
:101A600003028093020280914A0280FD02C01D9B06
:101A700007C0109247091092460983B7817F09C0B9
:101A800081E090E0909347098093460983B7817F76
:101A9000866083BF8091490990914A0997FF0BC0E6
:101AA0008091460990914709892B19F0749A73988F
:101AB00002C0739A7498609150027091510261153E
:101AC0007105B9F0809157099091580901960E94CB
:101AD000D584892B71F477988091490990914A09AE
:101AE00092FF07C0749884E090E090937A0280930C
:101AF0007902609150027091510261157105A1F057
:101B0000809157099091580901960E94D584892B9C
:101B100059F41092A2231092A12348E953E262E102
:101B20008CE092E00E943D4D609150027091510214
:101B300061157105B1F180915709909158090E9482
:101B4000D584892B71F581E080939823809152028E
:101B5000809399238091530280939A238091540219
:101B600080939B238091550280939C238091560201
:101B700080939D238091570280939E2380915802E9
:101B800080939F23809159028093A0231092A223D7
:101B90001092A12348E953E262E18AE292E00E94B6
:101BA0003D4D60914E0270914F0261157105A1F19A
:101BB00080915709909158090E94D584892B61F52D
:101BC0008091E3279091E427A091E527B091E62743
:101BD0004091751B5091761B6091771B7091781B1B
:101BE000841B950BA60BB70B8093AF1A9093B01A7A
:101BF000A093B11AB093B21A8091E3279091E42791
:101C0000A091E527B091E6278093751B9093761BF2
:101C1000A093771BB093781B60914C0270914D029A
:101C200061157105A1F180915709909158090E94A1
:101C3000D584892B61F58091E7279091E827A091C1
:101C4000E927B091EA274091791B50917A1B609166
:101C50007B1B70917C1B841B950BA60BB70B809391
:101C6000B31A9093B41AA093B51AB093B61A809190
:101C7000E7279091E827A091E927B091EA27809380
:101C8000791B90937A1BA0937B1BB0937C1B809154
:101C90004A0286FD2B9880914A0290914B0291FF57
:101CA00010C00E94C8618A3119F0C1E0C80F01C09C
:101CB000CBE00E9482608C2F90E00E94E0610E9445
:101CC000CA6040E050E060E08BE792E00E943D4D4A
:101CD000FF91EF91CF91BF91AF919F918F917F91A4
:101CE0006F915F914F913F912F910F900BBE0F908D
:101CF0000FBE0F901F9018958091D71A909197233F
:101D0000891B08950E947C0E882371F0E09197232F
:101D1000EF71F0E0E45DF44E808190E02091972334
:101D20002F5F2093972308958FEF9FEF0895CF9310
:101D3000DF93EC01109274091092730988819981E4
:101D40000097C1F08F35934021F01982188283E00B
:101D5000B6C0613109F0B2C0F89478940E94820E46
:101D6000992790936F0980936E098D3009F441C0D3
:101D70008F3F49F40E947C0E8111EECF8FE593E0F6
:101D8000998388839BC08231910509F458C08F37AD
:101D9000910509F050C080916C0990916D09181659
:101DA00019060CF56091C3307091C43088E090E062
:101DB0000E94378B6091C3307091C43080E290E014
:101DC0000E94378B6091C3307091C43088E090E0FE
:101DD0000E94378B80916C0990916D0901979093C7
:101DE0006D0980936C0980916C0990916D09CF9772
:101DF00009F6109297231092D71A80916C0990914E
:101E00006D09FC01ED55FC4D10829093740980938F
:101E1000730910926D0910926C09809101289091BC
:101E20000228009709F4A6CF40E050E060918211AB
:101E30000E943D4D9FCF8830910571F5ACCF6091E8
:101E4000C3307091C4308DE090E00E94378B1092C7
:101E50006B0910926A0980916A0990916B0920912F
:101E60006C0930916D09821793070CF0BCCFFC010F
:101E7000ED55FC4D80816091C3307091C43090E08D
:101E80000E94378B80916A0990916B09019690931B
:101E90006B0980936A09DFCF6091C3307091C430C1
:101EA0000E94378B80916C0990916D0920916E0989
:101EB000FC01ED55FC4D2083019691CF81E0DF912F
:101EC000CF9108958091460990914709892BB1F0EF
:101ED00080914A0290914B0293FD10C00E94826053
:101EE00083B7817F866083BFF89483B7816083BFA7
:101EF0007894889583B78E7F83BF78940895CF9325
:101F0000DF93EC0188819981009719F086329F4018
:101F100099F40E943F5F0E94620F40E050E065E844
:101F200080918611909187110E943D4D86E29FE03D
:101F30009983888381E003C01982188283E0DF914E
:101F4000CF910895CF93DF9300D0CDB7DEB7892B23
:101F500081F05F934F9382EB9DE09F938F93698312
:101F60007A830E947B8B0F900F900F900F907A8155
:101F700069817F936F938FEA9DE09F938F930E9477
:101F80007B8B0F900F900F900F900F900F90DF9121
:101F9000CF910895FF920F931F93CF93DF930E94E9
:101FA0003F5F80EB0E94A45881111CC00E94085919
:101FB00080917D1F90917E1F816090937E1F809302
:101FC0007D1F8EE893E09F938F938FEA9DE09F9310
:101FD0008F930E947B8B0F900F900F900F90C1E01A
:101FE000D0E002C0C0E0D0E0FEB08F2D8470F82EAB
:101FF000729A0E943F5F8EE40E94A458811116C01D
:102000000E94085980917D1F90917E1F826090935D
:102010007E1F80937D1F8E010F5F1F4F47EA58E0A0
:1020200066E973E0CE010E94A20FE801F11001C041
:1020300072980E943F5F8EEE0E94A458811116C0D4
:102040000E94085980917D1F90917E1F846090931B
:102050007E1F80937D1F8E010F5F1F4F47EA58E060
:102060006EE973E0CE010E94A20FE8010E943F5F7B
:1020700086EA0E94A458811116C00E9408598091D6
:102080007D1F90917E1F886090937E1F80937D1F9F
:102090008E010F5F1F4F47EA58E065EA73E0CE01FB
:1020A0000E94A20FE8010E943F5F8CE30E94A458A7
:1020B00081111EC00E94085980917D1F90917E1F42
:1020C000806190937E1F80937D1F8E010F5F1F4F55
:1020D00047EA58E06DEA73E0CE010E94A20F87EA5A
:1020E0009DE09F938F930E947B8B0F900F90E80150
:1020F0000E943F5F82ED0E94A458811116C00E9489
:10210000085980917D1F90917E1F806290937E1F61
:1021100080937D1F8E010F5F1F4F47EA58E065EBEC
:1021200073E0CE010E94A20FE8010E943F5F80E8A9
:102130000E94A458811116C00E94085980917D1FE9
:1021400090917E1F916090937E1F80937D1F8E01E2
:102150000F5F1F4F47EA58E06EEB73E0CE010E941D
:10216000A20FE8010E943F5F80ED0E94A4588111F8
:1021700016C00E94085980917D1F90917E1F806833
:1021800090937E1F80937D1F8E010F5F1F4F47EA44
:1021900058E064EC73E0CE010E94A20FE8010E94B7
:1021A0003F5F8CEE0E94A458811116C00E9408590E
:1021B00080917D1F90917E1F926090937E1F8093EF
:1021C0007D1F8E010F5F1F4F47EA58E06CEC73E0F4
:1021D000CE010E94A20FE80107E010E00E943F5FDD
:1021E0008CE70E94A458811113C00E940859809165
:1021F0007D1F90917E1F806490937E1F80937D1F32
:1022000047EA58E063ED73E0CE010E94A20F05C0DB
:10221000015011090115110509F70E940859DF91B4
:10222000CF911F910F91FF900C94480BCF93DF93A8
:1022300000D0CDB7DEB74A8369830E94DF58698139
:10224000862F0E9410594A81842F0E9410590F90A6
:102250000F90DF91CF910C940859AF92BF92DF920B
:10226000EF92FF920F931F93CF93DF9300D01F92B3
:10227000CDB7DEB7182FD22E4A835B8369830E94C5
:10228000DF586981862F0E941059812F81600E943A
:1022900006594A81A42E5B81B52E00E010E0ED2C9A
:1022A000F12C81E0E81AF1080D1580F40E151F05D8
:1022B00019F40E942B5902C00E942159F501808314
:1022C0000F5F1F4FFFEFAF1ABF0AEECF0F900F90B7
:1022D0000F90DF91CF911F910F91FF90EF90DF90C2
:1022E000BF90AF900C940859AF92BF92CF92DF92FB
:1022F000EF92FF920F931F93CF93DF93CDB7DEB78B
:1023000060970FB6F894DEBF0FBECDBFB82EA42ED7
:102310006623E9F18E010F5F1F4F80E1F8011192F2
:102320008A95E9F728E0A80168E980EB0E942D1161
:10233000BB2041F02CED33E03F932F930E94698B3B
:102340000F900F906E01F8E0CF0ED11C43EEE42EFB
:1023500043E0F42EF80181918F011F928F93FF9239
:10236000EF920E94698B0F900F900F900F900C15B9
:102370001D0581F788851F928F9328E334E03F93F2
:102380002F930E94698B0F900F900F900F90AA20AF
:10239000E9F18E010F5F1F4F80E1F80111928A95DC
:1023A000E9F728E0A80160E880EB0E942D11BB202E
:1023B00041F088EE93E09F938F930E94698B0F907A
:1023C0000F906E01F0E1CF0ED11C33EEE32E33E01F
:1023D000F32EF80181918F011F928F93FF92EF925C
:1023E0000E94698B0F900F900F900F900C151D0598
:1023F00081F788851F928F9388E394E09F938F9352
:102400000E94698B0F900F900F900F9060960FB6FF
:10241000F894DEBF0FBECDBFDF91CF911F910F911A
:10242000FF90EF90DF90CF90BF90AF900895CF9343
:10243000DF9300D0CDB7DEB71A82198222E0AE0159
:102440004F5F5F4F6AEA8EEE0E942D11898190E006
:10245000982F88272A81822B90934D1B80934C1BA9
:1024600022E0AE014F5F5F4F6CEA8EEE0E942D11AD
:10247000898190E0982F88272A81822B90934F1B87
:1024800080934E1B22E0AE014F5F5F4F6EEA8EEEEF
:102490000E942D11898190E0982F88272A81822B14
:1024A0009093511B8093501B22E0AE014F5F5F4F12
:1024B00060EB8EEE0E942D11898190E0982F882785
:1024C0002A81822B90935F1B80935E1B22E0AE01DA
:1024D0004F5F5F4F62EB8EEE0E942D11898190E07D
:1024E000982F88272A81822B9093611B8093601BF1
:1024F00022E0AE014F5F5F4F64EB8EEE0E942D1124
:10250000898190E0982F88272A81822B9093631BE2
:102510008093621B22E0AE014F5F5F4F66EB8EEE51
:102520000E942D11898190E0982F88272A81822B83
:102530009093531B8093521B22E0AE014F5F5F4F7D
:1025400068EB8EEE0E942D11898190E0982F8827EC
:102550002A81822B9093551B8093541B22E0AE015D
:102560004F5F5F4F6AEB8EEE0E942D11898190E0E4
:10257000982F88272A81822B9093591B8093581B70
:1025800022E0AE014F5F5F4F6CEB8EEE0E942D118B
:10259000898190E0982F88272A81822B90935B1B5A
:1025A00080935A1B22E0AE014F5F5F4F6EEB8EEEC1
:1025B0000E942D11898190E0982F88272A81822BF3
:1025C00090935D1B80935C1B0F900F90DF91CF91D8
:1025D00008952F923F924F925F926F927F928F92C7
:1025E0009F92AF92BF92CF92DF92EF92FF920F93A2
:1025F0001F93CF93DF93CDB7DEB76A970FB6F894EA
:10260000DEBF0FBECDBF182F488F298F19821A82C7
:102610001B828091701B811107C06A8F0E94171264
:1026200081E08093701B6A8D662309F46CC04EE2D2
:1026300064EF8EEE0E94161169E07AE180E090E08E
:102640000E94915822E0AE014F5F5F4F66EF8EEE21
:102650000E942D112981822F90E0A0E0B0E0222776
:10266000382F492F5A2F8A81282B8091621B9091F5
:10267000631B281B390B41095109A091601BB091C4
:10268000611B0E94B2846B017C018FE0F594E7949A
:10269000D794C7948A95D1F760915A1B70915B1BB0
:1026A000882777FD8095982F2BE0660F771F881F6E
:1026B000991F2A95D1F720915C1B30915D1B44270F
:1026C00037FD4095542F2C0D3D1D4E1D5F1D0E9462
:1026D0001F85C20ED31ED092571BC092561B88E096
:1026E000C80ED11C34E0D594C7943A95E1F7EE2496
:1026F000D7FCE094FE2CC092641BD092651BE09244
:10270000661BF092671B012F0295000F000F007CE3
:102710000C5CA12FB0E0BD8BAC8BA3E0B0E0012E30
:1027200002C0AA0FBB1F0A94E2F725E335E00E941E
:10273000AB84DC01CB010296A11DB11D8C879D8766
:10274000AE87BF8780E593ECA0E0B0E004C0B5950C
:10275000A795979587951A95D2F7888B998BAA8B11
:10276000BB8B10E0188619861A861B86A8E02A2ED5
:10277000312CAC89BD892A1A3B0A988D191709F4A6
:1027800036C1402F64EF8EEE0E9416116C857D8558
:102790008E859F850E94915823E0AE014F5F5F4F69
:1027A00066EF8EEE0E942D11E091561BF091571BA3
:1027B000E05AFF409F01DF010E9494846B017C017D
:1027C00080914E1B90914F1B9F8B8E8BA0904C1B2A
:1027D000B0904D1B2091501B3091511B0E9494844E
:1027E0002B013C013DE075946794579447943A95CA
:1027F000D1F7A091521BB091531BA70196016CE039
:1028000055954795379527956A95D1F70E94BD84D0
:10281000BB2797FDB095AB2F480E591E6A1E7B1E35
:1028200092E0490E511C611C711CB2E075946794D2
:1028300057944794BA95D1F7A0E85A0E611C711CC1
:10284000A0915E1BB0915F1BA30192010E94B28414
:10285000DC01CB012FE0B695A795979587952A9532
:10286000D1F78C839D83AE83BF8329818A8190E0D9
:10287000A0E0B0E04424582E692E7A2E622A8B8183
:10288000482A022C04C075946794579447940A947C
:10289000D2F74501AA2497FCA094BA2C42E0880CF8
:1028A000991CAA1CBB1C4A95D1F7A091541BB0914E
:1028B000551BA70196010E94BD846B017C0157E165
:1028C000F594E794D794C7945A95D1F72E893F8908
:1028D000DF010E949484EBE0959587957795679545
:1028E000EA95D1F7C60ED71EE81EF91E8C0C9D1C6A
:1028F000AE1CBF1C0C8804C0880C991CAA1CBB1CF5
:102900000A94D2F792E0890E911CA11CB11CF2E04E
:10291000B594A79497948794FA95D1F748185908D5
:102920006A087B08A3019201688979898A899B8951
:102930000E94C58497FD0DC0660F771F881F991FE1
:102940002C813D814E815F810E94FD8449015A01A5
:102950000CC02C813D814E815F810E94FD84490124
:102960005A01880C991CAA1CBB1C9927B7FC9A9584
:102970008B2D7A2D692D9B01AC010E94C5849B0192
:10298000AC01AEEDBBE00E94B2846C01FF24D7FC29
:10299000F094EF2CA3E4B3EEA50194010E94C0844F
:1029A000BB2797FDB095AB2FC80ED91EEA1EFB1EA4
:1029B000AFECCA0EAEE0DA1EE11CF11CA4E0F59407
:1029C000E794D794C794AA95D1F7C80CD91CEA1CF0
:1029D000FB1C88859985AA85BB858C0D9D1DAE1D28
:1029E000BF1D88879987AA87BB871F5FC6CE112323
:1029F00091F0212F30E040E050E0688579858A85AC
:102A00009B850E94FD842093681B3093691B409333
:102A10006A1B50936B1BA98DAA2389F16091681BD7
:102A20007091691B80916A1B90916B1B61157105F8
:102A30008105910521F10E94F68120E836EE45ECF2
:102A400057E40E94578121E03EED42E45EE30E949C
:102A500037849B01AC0160E070E080E89FE30E9456
:102A60008C802BE43AE34DEB57E30E94578160934F
:102A70006C1B70936D1B80936E1B90936F1B6A96FB
:102A80000FB6F894DEBF0FBECDBFDF91CF911F917F
:102A90000F91FF90EF90DF90CF90BF90AF909F90FD
:102AA0008F907F906F905F904F903F902F90089500
:102AB0000F931F93CF93DF9300D000D000D0CDB7FA
:102AC000DEB78E010F5F1F4F86E0F80111928A95E5
:102AD000E9F78091A61A811113C040E061E386EA0C
:102AE0000E9416114AE06CE286EA0E94161181E00B
:102AF0008093A61A6CE77EE380E090E00E949158F4
:102B000048E06DE286EA0E9416116CE77EE380E001
:102B100090E00E94915826E0A80162E386EA0E94B4
:102B20002D1147E06DE286EA0E9416118A8190E03D
:102B3000982F88272981822B9093A11A8093A01A1D
:102B40002C8130E0322F22274B81242B3093A31A83
:102B50002093A21A4E8150E0542F44276D81462BBA
:102B60005093A51A4093A41A5F934F933F932F93CA
:102B70009F938F938CEE93E09F938F930E94698B2A
:102B80000FB6F894DEBF0FBECDBF26960FB6F894F1
:102B9000DEBF0FBECDBFDF91CF911F910F91089582
:102BA000CF92DF92EF92FF920F931F93CF93DF9319
:102BB000CDB7DEB72A970FB6F894DEBF0FBECDBFF4
:102BC0008E010F5F1F4F86E0F80111928A95E9F799
:102BD00041E062E08CE30E94161148E560E08CE37E
:102BE0000E94161162E174E380E090E00E94915827
:102BF00026E0A80163E08CE30E942D1143E062E02F
:102C00008CE30E941611098110E0102F00278A81A1
:102C1000082B10937D1A00937C1AEB80F12CFE2C6C
:102C2000EE248C81E82AF0927F1AE0927E1ACD8001
:102C3000D12CDC2CCC248E81C82AD092811AC0924F
:102C4000801AB801882777FD8095982F0E94F68119
:102C50009B01AC01B701882777FD8095982F2F83C2
:102C6000388749875A870E94F6812F8138854985A0
:102C70005A850E94008120EE3EE245E652E40E9421
:102C8000D48320E030E044E353E40E948D809F939E
:102C90008F937F936F93DF92CF92FF92EF921F9368
:102CA0000F938AEF93E09F938F930E94698B0FB6E7
:102CB000F894DEBF0FBECDBF2A960FB6F894DEBFE4
:102CC0000FBECDBFDF91CF911F910F91FF90EF907D
:102CD000DF90CF900895CF93DF93EC0188819981A5
:102CE0000097F9F08F309F4021F01982188283E01D
:102CF00063C089E599E00E94E34F892BE1F0809160
:102D0000490990914A0993FD18C080914909909111
:102D10004A0994FD43C08091490990914A0995FD63
:102D200044C060E870E089E599E00E94BC4F8FE004
:102D30009FE09983888381E03FC080917D1F82FF5F
:102D4000E4CF21E048E061E083E00E94E912809155
:102D50006F1B8F9380916E1B8F9380916D1B8F9350
:102D600080916C1B8F9380916B1B8F9380916A1B5A
:102D70008F938091691B8F938091681B8F9386E05E
:102D80009EE09F938F930E947B8B8DB79EB70A9690
:102D90000FB6F8949EBF0FBE8DBFB7CF80917D1F39
:102DA00083FFB9CF0E945815B6CF80917D1F84FF55
:102DB000B8CF0E94D015B5CFDF91CF910895CF93B2
:102DC000C82F8CEE0E9406598C2F0E94105965E383
:102DD00075E080E090E00E9491588DEE0E940659C7
:102DE0000E942159C82F0E942B592C2F30E0322FDE
:102DF0002227A901482BCA01CF910895CF93DF93D1
:102E0000C82F8CEE0E9406598C2F0E94105962E147
:102E100074E380E090E00E9491588CEE0E94065985
:102E200080E00E94105965E375E080E090E00E9428
:102E300091588DEE0E9406590E942159C82F0E9478
:102E40002159D82F0E942B594D2F50E060E070E09F
:102E5000762F652F542F44276C2B482BCB01BA01BA
:102E6000DF91CF9108952F923F924F925F926F9290
:102E70007F928F929F92AF92BF92CF92DF92EF920A
:102E8000FF920F931F93CF93DF93CDB7DEB7CD544F
:102E9000D1090FB6F894DEBF0FBECDBF80910002FE
:102EA00090910102892BD1F110920102109200023F
:102EB0008CEE0E9406598EE10E9410596BE17EE46F
:102EC00080E090E00E94915882EA0E94DF16909381
:102ED00056098093550984EA0E94DF16909354099D
:102EE0008093530986EA0E94DF16909352098093DB
:102EF000510988EA0E94DF169093500980934F0988
:102F00008AEA0E94DF1690934E0980934D098CEA5D
:102F10000E94DF1690934C0980934B0988E40E942D
:102F2000FE166FAB78AF89AF9AAF88E50E94FE16A8
:102F30004B015C0180914D0990914E0920E030E0F9
:102F400040E050E0BA0126962FAF269727963FAF74
:102F5000279728964FAF289729965FAF29972A96EB
:102F60006FAF2A972B967FAF2B979C0140E050E0E4
:102F700060E070E080E090E008E00E94A6860E9499
:102F800052863901B42FA52FF62FE72F8C0194011B
:102F9000A50160E070E080E090E05301CB2EDA2ED6
:102FA000EF2EFE2E0E94DD8629833A832A011B0123
:102FB0004C01B101C401315041095F4F6F4F7F4F48
:102FC0008F4F9F4FA1E0B0E02596BFAFAEAF2597E2
:102FD00021153F4F4F4F5140610571058105910506
:102FE00009F020F425961FAE1EAE259725966EACEF
:102FF0007FAC259780914B0990914C095C01C12CC5
:10300000D12CE12CF12C00E010E029813A81A201C1
:10301000B101C4010E947585D22EE32EF42E052F36
:10302000162FB72FF82FE92FA0E00E94048784F411
:103030002150310940485F4F6F4F7F4F8F4F9F4F57
:10304000D22EE32EF42E052F162FB72FF82FE92FAF
:103050002D2D3E2D4F2D502F612F7B2F8F2F9E2FEB
:1030600007E10E94BF862B8F3C8F4D8F5E8F6F8F45
:1030700078A389A39AA32053384F4F4F5F4F6F4FC8
:103080007F4F8F4F9F4F2B8B3C8B4D8B5E8B6F8B6E
:10309000788F898F9A8F2056304F4F4F5F4F6F4FE9
:1030A0007F4F8F4F9F4F243D3043410551056105B0
:1030B00071058105910541F038F025966EAC7FAC25
:1030C0002597FFEF6F1A7F0A809153099091540959
:1030D0009C0140E050E060E070E080E090E000E1C2
:1030E0000E94A6862B833C834D835E836A87798703
:1030F0008F83988740914F0950915009A980BA80D9
:103100006201710184019A0140E050E060E070E0EA
:1031100080E090E00E947585D22EE32EF42E052FDC
:10312000162FB72FF82FE92FA0E00E9404875CF438
:10313000AFE70E94E686D22EE32EF42E052F162F3F
:10314000B72FF82FE92F2D2D3E2D4F2D502F612F0A
:103150007B2F8F2F9E2F07E00E94BF8659016A01A7
:103160007B018C012B813C814D815E816A85798553
:103170008F8198850E94DD862B833C834D835E83FF
:103180006F8378878F87988B2E5F3F4F434051091D
:103190006E4F7F4F8F4F9F4F22303105494F5F4F0A
:1031A000644071058105910521F018F01FEF611A47
:1031B000710A8091550990915609BC0180E090E018
:1031C00020E030E840E050E00E94CE8529873A8731
:1031D0004B875C876A8B798B8D879E8740915109DD
:1031E00050915209A980BA806201710184019A014B
:1031F00040E050E060E070E080E090E00E94758583
:10320000D22EE32EF42E052F162FB72FF82FE92FED
:10321000A0E00E94048784F421503F4F4F4F5F4F3E
:103220006F4F7F4F8F4F9F4FD22EE32EF42E052FDF
:10323000162FB72FF82FE92F2D2D3E2D4F2D502F64
:10324000612F7B2F8F2F9E2F08E00E94BF86590190
:103250006A017B018C0129853A854B855C856A89E9
:1032600079898D859E850E94DD8629873A874B87DF
:103270005C876D877E87898B9A8B2F5F3F4F41409C
:1032800051096109710981099109213030484C4F78
:103290005F47614071058105910521F018F0BFEF8E
:1032A0006B1A7B0A2B893C894D895E896F89788DE1
:1032B000898D9A8D2F3C3740410551056105710577
:1032C0008105910511F00CF0A5C1A980BA806201B9
:1032D000710184019501A201B101C4010E947585AB
:1032E000A12CB12CC12C10E8D12EE12CF12C00E046
:1032F00010E00E9438852BAF3CAF4DAF5EAF6FAF93
:1033000021967FAF219722968FAF229723969FAF6A
:103310002397AB8CBC8CCD8CDE8CEF8CF8A009A1F4
:103320001AA19501A601B701C8010E94758559012E
:103330006A017B01E82F192F02E00E94A6860E2F5A
:103340000E94DD8669017A01162F272EF82FE92FBA
:10335000322E8D2C942EAF2CB62E072F582EB92F2F
:10336000A0E00E9404875CF4A1E00E94E686322E71
:10337000832E942EA52EB62E072F582EB92F232D2F
:10338000382D492D5A2D6B2D702F852D9B2F01E047
:103390000E94BF862E962FAF2E972D963FAF2D976A
:1033A00049A75AA76BA77CA78DA79EA7522E432E8D
:1033B0004BA35CA36DA37EA38FA398A7B22D960108
:1033C000A701612F722D8F2F9E2FA0E00E940487EE
:1033D0004CF4A3E00E94E68669017A01162FB72F0C
:1033E000F82FE92F9601A701612F7B2F8F2F9E2F9A
:1033F00002E00E94BF862FA738AB49AB5AAB6BAB3C
:103400007CAB8DAB9EAB19014A01B62FA72F24963A
:103410008FAF2497F92F2B893C894D895E896F895D
:10342000788D898D9A8D24323A4F4F4F5F4F6F4F71
:103430007F4F8F4F9F4F0CF08CC02B8D3C8D4D8D4F
:103440005E8D6F8D78A189A19AA12455324F4F4F7F
:103450005F4F6F4F7F4F8F4F9F4F59016A017B0125
:103460008C010E94758519014A01B62FA72FFC0116
:1034700003E00E94A68651016401EB2EFA2E8F0113
:103480000E94F28659016A017B018C012E962FADB4
:103490002E972D963FAD2D9749A55AA56BA57CA5D6
:1034A0008DA59EA50E94DD86522E432E4BA35CA3C4
:1034B0006DA37EA38FA398A79101A4016B2F7A2FF0
:1034C000CF0102E00E94A68651016401EB2EFA2E84
:1034D0008F010E94F28602E00E94A6860E2F0E94B3
:1034E000F286F22E032F142FD52EE62EB72FF82FAB
:1034F000E92FA0E00E9404875CF4A1E00E94E68628
:10350000F22E032F142FD52EE62EB72FF82FE92FEA
:103510002F2D302F412F5D2D6E2D7B2F8F2F9E2F26
:1035200001E00E94BF8659016A017B018C012FA531
:1035300038A949A95AA96BA97CA98DA99EA90E945D
:10354000DD8619014A01B62FA72F24968FAF249745
:10355000F92F2B813C814D815E816F8178858F852C
:103560009889A52CB42CCBA0DCA0EDA0FEA00FA1C7
:1035700018A50E94F2862B833C834D835E836F8364
:1035800078878F87988B29853A854B855C856D85F3
:103590007E8589899A8951016401EB2EFA2E249641
:1035A0000FAD24971F2F0E94F28629873A874B87F9
:1035B0005C876D877E87898B9A8B2B893C894D89A7
:1035C0005E896F89788D898D9A8DABACBCACCDACA2
:1035D000DEACEFAC2196FFAC219722960FAD22977F
:1035E00023961FAD23970E94F2862056304F4F4FEF
:1035F0005F4F6F4F7F4F8F4F9F4F243D30434105AB
:103600005105610571058105910521F018F02FEF35
:10361000621A720A6FA978AD89AD9AADAB01BC018F
:1036200080E090E0DC0124964FAF249725965FAFB1
:10363000259726966FAF269727967FAF27972896D0
:103640008FAF289729969FAF29972A96AFAF2A97D1
:103650002B96BFAF2B97A984BA84CB84DC84ED84EE
:10366000FE8409891A899A01AB0160E070E080E06C
:1036700090E00E947585F22E032F142FD52EE62E92
:10368000B72FF82FE92FA0E00E94048784F421507F
:103690003109404E5F4F6F4F7F4F8F4F9F4FF22E3C
:1036A000032F142FD52EE62EB72FF82FE92F2F2D0D
:1036B000302F412F5D2D6E2D7B2F8F2F9E2F05E1FB
:1036C0000E94BF86AB80BC80CD80DE80EF80F88416
:1036D0000F8518890E94F286F22E032F142FD52E03
:1036E000E62EB72FF82FE92FA0E00E94048784F47C
:1036F000215030484F4F5F4F6F4F7F4F8F4F9F4F3D
:10370000F22E032F142FD52EE62EB72FF82FE92FE8
:103710002F2D302F412F5D2D6E2D7B2F8F2F9E2F24
:103720000FE00E94BF8669017A018B018A83998329
:1037300029011A014B015C01285E334041095109FE
:103740006109710981099109283D304D41405105B8
:10375000610571058105910521F018F0BFEF6B1A25
:103760007B0A0E940859672859F09601A701B80101
:103770008A8199810E94528629011A014B015C01BC
:103780009201A101B401C5010E94F08120E030E066
:1037900048EC52E40E945781C35BDF4F0FB6F894A8
:1037A000DEBF0FBECDBFDF91CF911F910F91FF9074
:1037B000EF90DF90CF90BF90AF909F908F907F90D1
:1037C0006F905F904F903F902F9008954F925F922F
:1037D0006F927F928F929F92AF92BF92CF92DF9221
:1037E000EF92FF922B013C0169017A0123EC35EF46
:1037F0004CE851E4C701B6010E94D4834B015C013F
:1038000028EB3EE143E753E4C701B6010E948D80F7
:103810009B01AC01C501B4010E9457810E94C48183
:103820004B015C0120E030E048EC52E4C301B201FE
:103830000E94578121E835E943EC50E40E94D4838B
:10384000A50194010E94D4834B015C0123E333E979
:1038500048E853E4C701B6010E948D809B01AC018A
:10386000C501B4010E94578123E333EB48E553E4DB
:103870000E94D483FF90EF90DF90CF90BF90AF90E5
:103880009F908F907F906F905F904F9008954F9290
:103890005F926F927F928F929F92AF92BF92CF92E0
:1038A000DF92EF92FF9269017A010E94568320E035
:1038B00030E040E050E40E948C8022E93CE54EED8F
:1038C0005EE30E9457814B015C0123EC35EF4CE82D
:1038D00051E4C701B6010E94D4832B013C0128EBBF
:1038E0003EE143E753E4C701B6010E948D809B018E
:1038F000AC01C301B2010E9457819B01AC01C5011B
:10390000B4010E948D806B017C0128EB3EE143E70E
:1039100053E40E94D4834B015C01A701960163EC40
:1039200075EF8CE891E40E948C809B01AC01C5018D
:10393000B4010E945781FF90EF90DF90CF90BF902D
:10394000AF909F908F907F906F905F904F90089571
:103950004F925F926F927F928F929F92AF92BF929F
:10396000CF92DF92EF92FF922B013C0169017A0125
:1039700023EC35EF4CE851E4C701B6010E94D48333
:103980004B015C0128EB3EE143E753E4C701B6017C
:103990000E948D809B01AC01C501B4010E9457813A
:1039A0000E94C4814B015C0120E030E048EC52E40D
:1039B000C301B2010E945781A50194010E94D483E2
:1039C00020E030E040E251E40E948C8024EE38E3B5
:1039D0004EE05FE30E94D4839B01AC01C701B601B6
:1039E0000E948D80FF90EF90DF90CF90BF90AF90BE
:1039F0009F908F907F906F905F904F900895CF929F
:103A0000DF92EF92FF920F931F93CF93DF9380E8A3
:103A10000E9406598AEF0E9410598FE00E941059A7
:103A200065E375E080E090E00E94915881E80E9493
:103A300006590E942159C82F0E9421590E942159DC
:103A4000D82F0E9421590E942159182F0E942159D4
:103A50000E942B59082F0E942B5980E80E9406597A
:103A60008CEF0E94105989EC0E94105965E375E0B3
:103A700080E090E00E94915881E80E9406590E94DF
:103A80002159D82E0E942159C82E0E9421590E94E6
:103A90002159F82E0E942159E82E0E942B591F927D
:103AA000CF921F92DF921F920F931F921F931F922C
:103AB000DF931F92CF931F92EF921F92FF928FE09E
:103AC00094E09F938F930E94698B0E9408598DB751
:103AD0009EB742960FB6F8949EBF0FBE8DBF20E0F2
:103AE00030E040E050E060E070E080E090E0DF91A6
:103AF000CF911F910F91FF90EF90DF90CF9008959D
:103B00000F931F93CF93DF93EC0180E80E94065937
:103B1000209741F085EE0E94105961E077E980E03E
:103B200090E007C083EE0E94105969E97AEB81E0CA
:103B300090E00E94915881E80E9406590E94215904
:103B4000182F0E942159082F0E942B590E940859B2
:103B5000602F70E0712B6C7F80E090E0CD2B69F0DE
:103B60000E94F48120E030E04AEF5AE30E94D483BF
:103B700020E030E040EC50E40CC00E94F48122E5EB
:103B800038EB4FE25BE30E94D48326E636E64BE354
:103B900052E40E948C80DF91CF911F910F91089584
:103BA0000F931F93CF93DF93729A80914A0283FF02
:103BB00008C08EE40E94A458811195C0C0E5D0E0F1
:103BC00008C0C0E5D0E00E944B0921972097D9F7A3
:103BD000F0CF0E944B0921972097D9F78FE40E94DC
:103BE000A4580E942159982F929596959695937076
:103BF0009130A9F440918B2350918C2360918D23B7
:103C000070918E234F5F5F4F6F4F7F4F40938B2399
:103C100050938C2360938D2370938E2316C0923023
:103C2000A0F040918F235091902360919123709147
:103C300092234F5F5F4F6F4F7F4F40938F2350937F
:103C400090236093912370939223082F0F730E9407
:103C50002159182F0E942159D82F0E942B59C82F63
:103C60000E94085980914A0283FF7298602F70E089
:103C7000762F6627610F711D80E090E00E94F4812D
:103C800020E134E048EC5BE30E94D4836093711B35
:103C90007093721B8093731B9093741B6D2F70E055
:103CA000762F66276C0F711D7695679576956795CB
:103CB00080E090E00E94F48124EA3CEF44E25CE37F
:103CC0000E94D48320E030E040E252E40E948C80E5
:103CD0006093042870930528809306289093072802
:103CE00080E090E015C08091872390918823A09177
:103CF0008923B0918A230196A11DB11D809387234A
:103D000090938823A0938923B0938A2381E090E045
:103D1000DF91CF911F910F9108957298729A8EE45E
:103D20000E94A45880EA0E94105980E00E94105915
:103D300080E00E9410598FE40E94A4580E942159EB
:103D400082958695869583708130A9F440918B2366
:103D500050918C2360918D2370918E234F5F5F4F24
:103D60006F4F7F4F40938B2350938C2360938D2311
:103D700070938E2316C08230A0F040918F23509113
:103D8000902360919123709192234F5F5F4F6F4F0B
:103D90007F4F40938F235093902360939123709390
:103DA00092231F928F938EE394E09F938F930E94B0
:103DB000698B8EE40E94A45880E80E94105980E02C
:103DC0000E94105980E00E9410590E9408590F90DB
:103DD0000F900F900F9080E090E008958AE99DE0A9
:103DE0009F938F930E947B8B80916C020F900F901A
:103DF000882361F01F928F9387E99DE09F938F93B3
:103E00000E947B8B0F900F900F900F90089582E788
:103E10009DE09F938F930E947B8B8AE49DE09F930C
:103E20008F930E947B8B83E29DE09F938F930E94F0
:103E30007B8B88EE9CE09F938F930E947B8B86EB1D
:103E40009CE09F938F930E947B8B8AE79CE09F93DB
:103E50008F930E947B8B84E59CE09F938F930E94BD
:103E60007B8B8EE19CE09F938F930E947B8B809154
:103E70007D1F90917E1F827091702DB73EB7205F9D
:103E80003F4F0FB6F8943EBF0FBE2DBF892B41F0B8
:103E90008EEE9BE09F938F930E947B8B0F900F90F1
:103EA00082EC9BE09F938F930E947B8B89E99BE040
:103EB0009F938F930E947B8B8EE69BE09F938F93C3
:103EC0000E947B8B8FE39BE09F938F930E947B8B61
:103ED0008DE09BE09F938F930E947B8B8CED9AE00B
:103EE0009F938F930E947B8B85EA9AE09F938F9399
:103EF0000E947B8B85E79AE09F938F930E947B8B38
:103F000089E49AE09F938F930E947B8B8AE19AE0E9
:103F10009F938F930E947B8B81EE99E09F938F9369
:103F20000E947B8B88EA99E09F938F930E947B8B02
:103F300081E799E09F938F930E947B8B80E499E0C7
:103F40009F938F930E947B8B81E199E09F938F9346
:103F50000E947B8B82EE98E09F938F930E947B8BD5
:103F60008DB79EB780960FB6F8949EBF0FBE8DBFDB
:103F70008BEB98E09F938F930E947B8B85E898E072
:103F80009F938F930E947B8B8FE498E09F938F93F6
:103F90000E947B8B86E298E09F938F930E947B8B9D
:103FA0008BEE97E09F938F930E947B8B80EC97E042
:103FB0009F938F930E947B8B2DB73EB7245F3F4F1B
:103FC0000FB6F8943EBF0FBE2DBF08958EE494E067
:103FD0000C949F8B4F925F926F927F928F929F92E1
:103FE000AF92BF92CF92DF92EF92FF92CF93DF9387
:103FF000CDB7DEB728970FB6F894DEBF0FBECDBFA2
:104000008091832390918423A0918523B09186236E
:1040100089839A83AB83BC8340908323509084230D
:1040200060908523709086238091832390918423D0
:10403000A0918523B09186238D839E83AF83B8871B
:1040400060918323709184238091852390918623AE
:104050002CE3822E912CA12CB12CA50194010E945D
:10406000FD847F936F9330E1C32E3EE0D32EE12C8D
:10407000F12C6D817E818F819885A70196010E9428
:10408000FD84A50194010E94FD843F932F9340E895
:10409000842E41E5942EAA24A394B12CC301B2012D
:1040A000A50194010E94FD84A70196010E94FD8450
:1040B0003F932F9369817A818B819C81A501940123
:1040C0000E94FD843F932F938AE997E09F938F93FB
:1040D0000E947B8B0FB6F894DEBF0FBECDBF289633
:1040E0000FB6F894DEBF0FBECDBFDF91CF91FF902A
:1040F000EF90DF90CF90BF90AF909F908F907F9088
:104100006F905F904F900895E9ECF0E3808191818A
:104110008234924479F0E95CF043FF93EF938CE7AB
:1041200097E09F938F930E947B8B0F900F900F903F
:104130000F9008953A96E53F81E4F80738F3089523
:10414000CF93DF93EC018C9A0E942E0A9F938F935A
:104150007F936F9380E797E09F938F930E947B8B71
:104160000F900F900F900F900F900F90209719F0D5
:104170000E94480B08C08EE697E09F938F930E94A1
:104180007B8B0F900F9081E00E94DF0920917102DC
:104190003091720240917302509174020E94D48354
:1041A0009F938F937F936F9382E697E09F938F9374
:1041B0000E947B8B0F900F900F900F900F900F909D
:1041C000209719F00E94480B08C080E697E09F9363
:1041D0008F930E947B8B0F900F9082E00E94DF09EB
:1041E00020916D0230916E0240916F0250917002E9
:1041F0000E94D4839F938F937F936F9384E597E07E
:104200009F938F930E947B8B0F900F900F900F9036
:104210000F900F90209719F00E94480B08C082E57C
:1042200097E09F938F930E947B8B0F900F9083E07A
:104230000E94DF099F938F937F936F9383E497E0AE
:104240009F938F930E947B8B8C980F900F900F9071
:104250000F900F900F90209719F00E94480B08C004
:1042600081E497E09F938F930E947B8B0F900F9038
:1042700080917D1F87FF7FC021E042E161E080EDFA
:104280000E94685A9F938F937F936F9384E397E084
:104290009F938F930E947B8B0F900F900F900F90A6
:1042A0000F900F90209719F00E94480B08C082E3EE
:1042B00097E09F938F930E947B8B0F900F9021E04C
:1042C00042E162E080ED0E94685A9F938F937F9352
:1042D0006F9385E297E09F938F930E947B8B0F9063
:1042E0000F900F900F900F900F90209719F00E9451
:1042F000480B08C083E297E09F938F930E947B8BCB
:104300000F900F9021E042E163E080ED0E94685A37
:104310009F938F937F936F9386E197E09F938F9303
:104320000E947B8B0F900F900F900F900F900F902B
:10433000209719F00E94480B08C084E197E09F93F2
:104340008F930E947B8B0F900F9021E042E164E0FD
:1043500080ED0E94685A9F938F937F936F9387E0BD
:1043600097E09F938F930E947B8B0F900F900F90FD
:104370000F900F900F90CD2B21F4DF91CF910C94E3
:10438000480BDF91CF9108950F931F93CF93DF9345
:10439000882389F049E050E06FEF70E088EF97E202
:1043A0000E94D78A49E050E06AE070E088EF97E227
:1043B0000E94BE8C13C0C8EFD7E202E017E08991DB
:1043C0001F928F931F930F930E947B8B0F900F90E0
:1043D0000F900F9088E2C030D80789F7DF91CF9116
:1043E0001F910F910C94480BCF92DF92EF92FF92A6
:1043F000CF93DF936B017C0160FF11C089E694E0ED
:104400009F938F938FEA9DE09F938F930E947B8B66
:104410000F900F900F900F9081E090E002C080E02D
:1044200090E0C1FE09C0EC01219647EA58E06EE633
:1044300074E00E94A20FCE01C2FE09C0EC012196D9
:1044400047EA58E066E774E00E94A20FCE01C3FE7F
:1044500009C0EC01219647EA58E06EE774E00E943B
:10446000A20FCE01C4FE09C0EC01219647EA58E034
:1044700062E874E00E94A20FCE01C5FE09C0EC0103
:10448000219647EA58E065E874E00E94A20FCE0149
:10449000C6FE09C0EC01219647EA58E069E874E0DD
:1044A0000E94A20FCE01C7FE09C0EC01219647EA87
:1044B00058E06FE874E00E94A20FCE01D0FE09C060
:1044C000EC01219647EA58E067E974E00E94A20FE8
:1044D000CE01D1FE09C0EC01219647EA58E06FE910
:1044E00074E00E94A20FCE01D2FE09C0EC01219619
:1044F00047EA58E063EA74E00E94A20FCE012091DF
:104500007D1F30917E1F24703270232B59F0D3FE13
:1045100009C0EC01219647EA58E069EA74E00E947C
:10452000A20FCE0120917D1F23FF0BC0D4FE09C036
:10453000EC01219647EA58E06EEA74E00E94A20F6F
:10454000CE0120917D1F24FF0BC0D5FE09C0EC01D8
:10455000219647EA58E064EB74E00E94A20FCE0176
:10456000D6FE09C0EC01219647EA58E06CEB74E0F6
:104570000E94A20FCE01B701A60144275078452B17
:10458000462B472B61F047EA58E067EC74E0DF9177
:10459000CF91FF90EF90DF90CF900C94A20FCD2899
:1045A000CE28CF2841F48DEF96E09F938F930E9401
:1045B0007B8B0F900F90DF91CF91FF90EF90DF906A
:1045C000CF9008950F931F93CF93DF938C01C0E09A
:1045D000D0E00115110509F48AC068EF76E0C80142
:1045E0000E94B68A892B09F4C16060EF76E0C801A9
:1045F0000E94B68A892B09F4C26068EE76E0C80191
:104600000E94B68A892B09F4C46064EE76E0C80182
:104610000E94B68A892B09F4C86061EE76E0C80171
:104620000E94B68A892B09F4C0616DED76E0C8015D
:104630000E94B68A892B09F4C06267ED76E0C80152
:104640000E94B68A892B09F4C0646FEC76E0C80139
:104650000E94B68A892B09F4C06867EC76E0C8012D
:104660000E94B68A892B09F4D16063EC76E0C80118
:104670000E94B68A892B09F4D2606DEB76E0C801FE
:104680000E94B68A892B09F4D46068EB76E0C801F1
:104690000E94B68A892B09F4D86062EB76E0C801E3
:1046A0000E94B68A892B09F4D0616AEA76E0C801D3
:1046B0000E94B68A892B09F4D0626FE976E0C801BE
:1046C0000E94B68A892B09F4D0646EE876E0C801AE
:1046D0000E94B68A892B09F4D06860916A027091B1
:1046E0006B0280E090E00E94CA8A8C0172CFCE01FA
:1046F000DF91CF911F910F910895AF92BF92CF920A
:10470000DF92EF92FF920F931F93CF93DF93F22EDE
:10471000032F142FE52E5B016C01217030E040E087
:1047200050E060E070E080E090E0A0E00E9404874C
:1047300089F0E8EDF4E0FF93EF93EFEAFDE0FF93FB
:10474000EF930E947B8B0F900F900F900F90E1E002
:10475000F0E002C0E0E0F0E080917D1F80FF17C034
:104760002F2D247030E040E050E060E070E080E009
:1047700090E0A0E00E94048751F0EF01219647EA03
:1047800058E06CED74E0CF010E94A20FFE012F2DC6
:10479000227030E040E050E060E070E080E090E0C7
:1047A000A0E00E94048751F0EF01219647EA58E00B
:1047B00060EE74E0CF010E94A20FFE012F2D287041
:1047C00030E040E050E060E070E080E090E0A0E0A9
:1047D0000E94048751F0EF01219647EA58E068EF04
:1047E00074E0CF010E94A20FFE012F2D207130E056
:1047F00040E050E060E070E080E090E0A0E00E94E7
:10480000048751F0EF01219647EA58E063EE74E027
:10481000CF010E94A20FFE012F2D207230E040E058
:1048200050E060E070E080E090E0A0E00E9404874B
:1048300051F0EF01219647EA58E066EE74E0CF01AF
:104840000E94A20FFE012F2D207430E040E050E0C6
:1048500060E070E080E090E0A0E00E94048751F00A
:10486000EF01219647EA58E06CEE74E0CF010E9418
:10487000A20FFE012F2D207830E040E050E060E0F4
:1048800070E080E090E0A0E00E94048751F0EF012A
:10489000219647EA58E062EF74E0CF010E94A20F30
:1048A000FE0120E0302F317040E050E060E070E029
:1048B00080E090E0A0E00E94048751F0EF01219693
:1048C00047EA58E065EF74E0CF010E94A20FFE01B5
:1048D00020E0302F327040E050E060E070E080E097
:1048E00090E0A0E00E94048751F0EF01219647EA92
:1048F00058E06AEF74E0CF010E94A20FFE0120E0B1
:10490000302F347040E050E060E070E080E090E0F4
:10491000A0E00E94048751F0EF01219647EA58E099
:1049200061E075E0CF010E94A20FFE0120E0302F70
:10493000387040E050E060E070E080E090E0A0E09F
:104940000E94048751F0EF01219647EA58E064E0A5
:1049500075E0CF010E94A20FFE0120E0302F3071E0
:1049600040E050E060E070E080E090E0A0E00E9475
:10497000048751F0EF01219647EA58E069E075E0BD
:10498000CF010E94A20FFE0120E0302F307240E0E4
:1049900050E060E070E080E090E0A0E00E940487DA
:1049A00051F0EF01219647EA58E060E175E0CF0150
:1049B0000E94A20FFE0180917D1F81FF17C020E0A1
:1049C000302F307440E050E060E070E080E090E034
:1049D000A0E00E94048751F0EF01219647EA58E0D9
:1049E00067E175E0CF010E94A20FFE0180917D1F5B
:1049F00090917E1F90FF17C020E030E040E05E2DD8
:104A0000507160E070E080E090E0A0E00E940487D8
:104A100051F0EF01219647EA58E06AE175E0CF01D5
:104A20000E94A20FFE0180917D1F90917E1F90FF3A
:104A300017C020E030E040E05E2D507260E070E092
:104A400080E090E0A0E00E94048751F0EF01219601
:104A500047EA58E06DE175E0CF010E94A20FFE0128
:104A600080917D1F90917E1F90FF17C020E030E065
:104A700040E05E2D507460E070E080E090E0A0E0E7
:104A80000E94048751F0EF01219647EA58E063E263
:104A900075E0CF010E94A20FFE0120E0302F307898
:104AA00040E050E060E070E080E090E0A0E00E9434
:104AB000048751F0EF01219647EA58E06EE275E075
:104AC000CF010E94A20FFE0120E030E0412F417093
:104AD00050E060E070E080E090E0A0E00E94048799
:104AE00051F0EF01219647EA58E063E375E0CF010A
:104AF0000E94A20FFE0120E030E0412F427050E002
:104B000060E070E080E090E0A0E00E94048751F057
:104B1000EF01219647EA58E066E375E0CF010E9475
:104B2000A20FFE0120E030E0412F447050E060E031
:104B300070E080E090E0A0E00E94048751F0EF0177
:104B4000219647EA58E069E375E0CF010E94A20F81
:104B5000FE0180917D1F87FF17C020E030E0412FCC
:104B6000487050E060E070E080E090E0A0E00E94DB
:104B7000048751F0EF01219647EA58E06CE375E0B5
:104B8000CF010E94A20FFE0180917D1F87FF17C0F9
:104B900020E030E0412F407150E060E070E080E0C4
:104BA00090E0A0E00E94048751F0EF01219647EACF
:104BB00058E060E475E0CF010E94A20FFE018091F1
:104BC0007D1F87FF17C020E030E0412F407250E08A
:104BD00060E070E080E090E0A0E00E94048751F087
:104BE000EF01219647EA58E064E475E0CF010E94A6
:104BF000A20FFE0180917D1F87FF17C020E030E0EB
:104C0000412F407450E060E070E080E090E0A0E070
:104C10000E94048751F0EF01219647EA58E068E4CA
:104C200075E0CF010E94A20FFE0180917D1F82FFDF
:104C300017C020E030E0412F407850E060E070E0A5
:104C400080E090E0A0E00E94048751F0EF012196FF
:104C500047EA58E067E076E0CF010E94A20FFE012C
:104C600080917D1F82FF17C020E030E040E05E2D84
:104C7000517060E070E080E090E0A0E00E94048766
:104C800051F0EF01219647EA58E06CE475E0CF015E
:104C90000E94A20FFE0180917D1F90917E1F90FFC8
:104CA00017C020E030E040E05E2D527060E070E020
:104CB00080E090E0A0E00E94048751F0EF0121968F
:104CC00047EA58E06FE475E0CF010E94A20FFE01B1
:104CD00080917D1F90917E1F90FF17C020E030E0F3
:104CE00040E05E2D547060E070E080E090E0A0E075
:104CF0000E94048751F0EF01219647EA58E067E5EA
:104D000075E0CF010E94A20FFE0180917D1F90915E
:104D10007E1F91FF1EC020E030E040E05E2D587005
:104D200060E070E080E090E0A0E00E94048789F0FD
:104D300047EA58E060E675E0CF01DF91CF911F911F
:104D40000F91FF90EF90DF90CF90BF90AF900C94B9
:104D5000A20F2F2D302F412F5E2DB501C601A0E0EF
:104D60000E94048741F489E896E09F938F930E9404
:104D70007B8B0F900F90DF91CF911F910F91FF9040
:104D8000EF90DF90CF90BF90AF900895AF92BF9219
:104D9000DF92EF920F931F93CF93DF93EC015B01B0
:104DA000FB01108264E876E00E94B68A892B59F5EF
:104DB00080917D1F7DE4D72EE0E8EE2E82FD02C0BB
:104DC00004E001C004E810E081FF02C060ECE62EC0
:104DD00026E04AE250E06BE270E089E290E00E9457
:104DE000B85581E090E00E94D60A882311F05DE575
:104DF000D52E80917D1F90917E1F90FD16E091FF32
:104E000006C0186004C0D12CE12C00E010E062E87C
:104E100076E0CE010E94B68A892B61F481E0F5012B
:104E2000808360916A0270916B0280E090E00E9442
:104E3000CA8AEC0160E876E0CE010E94B68A892B2E
:104E400061F48FEFF501808360916A0270916B02CB
:104E500080E090E00E94CA8AEC01209709F41AC110
:104E60006CE776E0CE010E94B68A892B19F4FD2DFD
:104E7000F160DF2E68E776E0CE010E94B68A892BCA
:104E800019F48D2D8460D82E65E776E0CE010E945E
:104E9000B68A892B19F4ED2DE260DE2E63E776E009
:104EA000CE010E94B68A892B19F4FD2DF860DF2E01
:104EB00060E776E0CE010E94B68A892B19F48D2D29
:104EC0008061D82E6AE676E0CE010E94B68A892BF0
:104ED00019F4ED2DE062DE2E64E676E0CE010E944C
:104EE000B68A892B19F4FD2DF064DF2E61E676E099
:104EF000CE010E94B68A892B19F48D2D8068D82E98
:104F00006CE576E0CE010E94B68A892B19F4EE2D6D
:104F1000E160EE2E65E576E0CE010E94B68A892B2F
:104F200019F4FE2DF260EF2E62E576E0CE010E94CC
:104F3000B68A892B19F48E2D8460E82E6DE476E014
:104F4000CE010E94B68A892B19F4EE2DE860EE2E70
:104F500066E476E0CE010E94B68A892B19F4FE2D14
:104F6000F061EF2E6FE376E0CE010E94B68A892BC6
:104F700019F48E2D8062E82E6CE376E0CE010E945B
:104F8000B68A892B19F4EE2DE064EE2E67E376E005
:104F9000CE010E94B68A892B19F4FE2DF068EF2EFF
:104FA00064E376E0CE010E94B68A892B09F40160A1
:104FB00061E376E0CE010E94B68A892B09F4026093
:104FC0006EE276E0CE010E94B68A892B09F4046075
:104FD0006AE276E0CE010E94B68A892B09F4086065
:104FE00066E276E0CE010E94B68A892B09F4006160
:104FF00062E276E0CE010E94B68A892B09F4006253
:105000006EE176E0CE010E94B68A892B09F4006435
:105010006CE176E0CE010E94B68A892B09F4006823
:1050200069E176E0CE010E94B68A892B09F411600D
:1050300061E176E0CE010E94B68A892B09F4126004
:1050400068E076E0CE010E94B68A892B09F41460EC
:105050006FEF75E0CE010E94B68A892B09F41860C3
:105060006CEF75E0CE010E94B68A892B09F41061BD
:1050700066EF75E0CE010E94B68A892B09F41062B2
:105080006BEE75E0CE010E94B68A892B09F0DCCE6A
:105090001064DACE2D2D3E2DA80160E070E080E096
:1050A00090E0DF91CF911F910F91EF90DF90BF9033
:1050B000AF9008958BED95E09F938F930E947B8B2B
:1050C0000E94E61F82E99AE19F938F9383ED95E01A
:1050D0009F938F930E947B8B8FEC95E09F938F9390
:1050E0000E947B8B80E00E94C4218AEC95E09F9314
:1050F0008F930E947B8B0E94CA0F80917D1F2DB7DA
:105100003EB7265F3F4F0FB6F8943EBF0FBE2DBF90
:1051100080FF05C041E061E081E00E9474110E94BF
:10512000EA1F809149021F928F9381EC95E09F9333
:105130008F930E947B8B809145091F928F9388EB00
:1051400095E09F938F930E947B8B1F9280E48F93B7
:1051500080EA95E09F938F930E947B8B8091092832
:105160001F928F93809108281F928F938DE895E06E
:105170009F938F930E947B8B809148021F928F9305
:1051800084E895E09F938F930E947B8B80914A02E5
:1051900090914B022DB73EB72A5E3F4F0FB6F89461
:1051A0003EBF0FBE2DBF96FF03C089E695E002C04B
:1051B0008CE695E09F938F938AE795E09F938F937A
:1051C0000E947B8B809151028F93809150028F932C
:1051D00085E695E09F938F930E947B8B8DE595E00C
:1051E0009F938F930E947B8B2091520230915302A8
:1051F00040915402509155026091560270915702AD
:1052000080915802909159020E947D230E94480B80
:105210008DB79EB70A960FB6F8949EBF0FBE8DBF8E
:105220001D9B03C089E695E002C08CE695E09F9344
:105230008F9381E595E09F938F930E947B8B87E40A
:1052400095E09F938F930E947B8B80914A020F90F1
:105250000F900F900F900F900F9081FF09C081E485
:1052600095E09F938F930E947B8B0F900F9013C0BC
:1052700080FF03C089E695E002C08CE695E09F932D
:105280008F938DE395E09F938F930E947B8B0F907C
:105290000F900F900F9086E395E09F938F930E945D
:1052A0007B8B6091490970914A0980E090E00E94EF
:1052B000F4210E94480B0F900F90779903C089E664
:1052C00095E002C08CE695E09F938F938DE295E088
:1052D0009F938F930E947B8B0E94E50860915202FE
:1052E0007091530280915402909155020E94880A55
:1052F0000E94420A9F938F937F936F938FE195E073
:105300009F938F930E947B8B81E090E00E94A0206E
:105310008091E3279091E427A091E527B091E627BB
:10532000BF93AF939F938F9381E195E09F938F936A
:105330000E947B8B8091F3278F938091F2278F932C
:105340008091F1278F938091F0278F938DEF94E0D8
:105350009F938F930E947B8B8091E7279091E82702
:10536000A091E927B091EA27BF93AF939F938F93C2
:105370008FEE94E09F938F930E947B8B8091F72711
:105380008F938091F6278F938091F5278F9380914B
:10539000F4278F938BED94E09F938F930E947B8BE8
:1053A0002DB73EB72E5D3F4F0FB6F8943EBF0FBEF0
:1053B0002DBF61E070E080E090E00E94510B61E061
:1053C00070E081E090E00C94510BF894E0E0F0E0A4
:1053D00081E2809357008491E2E0F0E041E2409363
:1053E00057004491E4E0F0E091E290935700E4919B
:1053F00090E0A0E0B0E0DC019927882750E060E071
:1054000070E0762F652F542F4427840F951FA61F19
:10541000B71F8E0F911DA11DB11D8093281B909366
:10542000291BA0932A1BB0932B1B78940895DF921D
:10543000EF92FF920F931F93CF93DF93CDB7DEB719
:1054400069970FB6F894DEBF0FBECDBF48E050E0BD
:105450006AE170E0CE010B960E94A08CDB84EC84A4
:10546000FD840E851F85B889F989EA892D2D3E2D89
:105470004F2D502F612F7B2F8F2F9E2FAFEF0E942C
:10548000048749F448E050E06AE170E082E592E088
:105490000E94BE8C10C0D0925202E0925302F09251
:1054A00054020093550210935602B0935702F093A2
:1054B0005802E093590242E050E068E170E0CE010A
:1054C00047960E94A08C8F89988D8F3F2FEF92076F
:1054D00079F48CE390E0909351028093500242E083
:1054E00050E068E170E080E592E00E94BE8C04C06C
:1054F000909351028093500242E050E066E170E0E8
:10550000CE0147960E94A08C8F89988D8F3F2FEFF8
:10551000920779F48AE090E490934B0280934A02D8
:1055200042E050E066E170E08AE492E00E94BE8CC6
:1055300004C090934B0280934A0242E050E06EE236
:1055400070E0CE0147960E94A08C8F89988D8F3F86
:105550002FEF920769F410924A091092490942E02C
:1055600050E06EE270E089E499E00E94BE8C04C0D5
:1055700090934A098093490949E050E06AE070E05D
:1055800088EF97E20E94A08C0E94890C44E050E0D2
:1055900066E270E0CE0143960E94A08C8B899C89C4
:1055A000AD89BE8944E050E066E270E08F3F9F4FD6
:1055B000AF4FBF4F29F481E792E00E94BE8C04C038
:1055C00081E792E00E94A08C44E050E062E270E04B
:1055D000CE0143960E94A08C8B899C89AD89BE899F
:1055E00044E050E062E270E08F3F9F4FAF4FBF4F0B
:1055F00029F48DE692E00E94BE8C04C08DE692E014
:105600000E94A08C44E050E06AE270E0CE01439634
:105610000E94A08C8B899C89AD89BE8944E050E0B2
:105620006AE270E08F3F9F4FAF4FBF4F29F485E78D
:1056300092E00E94BE8C04C085E792E00E94A08C9C
:1056400041E050E065E170E0CE0149960E94A08CF7
:10565000898D41E050E065E170E08F3F29F485E4F9
:1056600099E00E94BE8C04C085E499E00E94A08C61
:1056700041E050E064E170E0CE0149960E94A08CC8
:10568000898D41E050E064E170E08F3F29F489E4C6
:1056900092E00E94BE8C04C089E492E00E94A08C3B
:1056A00041E050E063E170E0CE0149960E94A08C99
:1056B000898D41E050E063E170E08F3F29F488E498
:1056C00092E00E94BE8C04C088E492E00E94A08C0C
:1056D0004AE050E060E070E0CE0101960E94A08CAC
:1056E00089814AE050E060E070E08F3F29F482E970
:1056F0009AE10E94BE8C04C082E99AE10E94A08CCB
:1057000069960FB6F894DEBF0FBECDBFDF91CF9183
:105710001F910F91FF90EF90DF900895CF92DF924D
:10572000EF92FF9260916A0270916B0280E090E0CC
:105730000E94CA8A60E775E00E94DE8A892B09F020
:10574000C0C08DE48093520280E88093530284E0CD
:1057500080935402109255021092560210925702F2
:10576000109258021092590248E050E06AE170E04D
:1057700082E592E00E94BE8C8CE390E0909351020F
:105780008093500242E050E068E170E080E592E0F2
:105790000E94BE8C8AE090E490934B0280934A0270
:1057A00042E050E066E170E08AE492E00E94BE8C44
:1057B00010924A091092490942E050E06EE270E00E
:1057C00089E499E00E94BE8C32E2C32EDD24DA9493
:1057D0003CECE32E3BE3F32EC0927102D0927202B6
:1057E000E0927302F092740244E050E066E270E0EE
:1057F00081E792E00E94BE8CC0926D02D0926E0250
:10580000E0926F02F092700244E050E062E270E0D9
:105810008DE692E00E94BE8C87ED94E3AFEEBCE390
:105820008093750290937602A0937702B0937802EA
:1058300044E050E06AE270E085E792E00E94BE8CAE
:105840001092450980E090E00E94156341E050E02D
:1058500065E170E085E499E00E94BE8C8AE1809366
:1058600049028AE190E00E94CB6141E050E064E1AE
:1058700070E089E492E00E94BE8C8FE08093480241
:1058800041E050E063E170E088E492E00E94BE8C69
:105890008AE0E2E9FAE1DF011D928A95E9F74AE040
:1058A00050E060E070E0CF010E94BE8C81E00E9479
:1058B000C42180E090E0FF90EF90DF90CF900C94B7
:1058C0009D0CFF90EF90DF90CF9008952F923F9224
:1058D0004F925F926F927F928F929F92AF92BF9200
:1058E000CF92DF92EF92FF920F931F93CF93DF93AC
:1058F000CDB7DEB727970FB6F894DEBF0FBECDBF8A
:105900009F838E83FC0180819181892B11F00C94FF
:10591000C33C60916A0270916B0283EA93E20E9439
:10592000CA8A60E470E083EA93E20E94FD8A0097ED
:1059300059F46091C3307091C4308AE090E00E94C5
:10594000378B81E00C94C83C8130910549F420905C
:10595000A323312C412C512C612C712C4301BDC04F
:1059600082309105A1F48091A3232091A42390E09B
:10597000982F8827820F911D1C01892F880F880B73
:10598000482E582E682E782E882E982EA6C083304A
:105990009105D1F52091A3231091A423E091A52393
:1059A00030E040E050E060E070E080E090E000E156
:1059B0000E94A686522E632E742E852E962EB72F09
:1059C000A82FF92F212F30E040E050E060E070E098
:1059D00080E090E008E00E94A68659016A017B0100
:1059E0008C01252D362D472D582D692D7B2F8A2F83
:1059F0009F2F0E94DD86AE2EB12CC12CD12CE12C24
:105A0000F12C00E010E059C004970CF45DC0209127
:105A1000A3231091A423E091A523F091A62330E0C5
:105A200040E050E060E070E080E090E008E10E943B
:105A3000A68629013A014B01B82FA92F212F30E06A
:105A400040E050E060E070E080E090E000E10E9423
:105A5000A68659016A017B018C019201A301B40160
:105A60008B2F9A2F0E94DD86AF2EB12CC12CD12C0A
:105A7000E12CF12C00E010E00E94DD86522E632E16
:105A8000742E852E962EB72FA82FF92F2E2F30E0AB
:105A900040E050E060E070E080E090E008E00E94CC
:105AA000A68659016A017B018C01252D362D472DD3
:105AB000582D692D7B2F8A2F9F2F0E94DD8619017B
:105AC0002A013B014C0109C06AE0262E312C412CF1
:105AD000512C612C712C812C912C0E94480B91012E
:105AE000A201B301C4012736FFE63F07FCE64F07DA
:105AF0005105610571058105910511F40C94F53688
:105B00002736EFE63E07ECE64E07510561057105C5
:105B10008105910511F008F075C12936F2E73F07BC
:105B200041055105610571058105910511F40C943C
:105B30000B3A2936E2E73E0741055105610571053B
:105B40008105910511F008F097C02536F4E63F076E
:105B500041055105610571058105910509F42FC5C0
:105B60002536E4E63E0741055105610571058105CD
:105B7000910509F088F5A6E70E94048709F4D6C6C6
:105B80000E94048709F060F4A8E60E94048709F4E3
:105B90005CC5A5E70E94048709F4B2C60C94C13C19
:105BA0009101A201B301C4012A33F6E23F07410586
:105BB0005105610571058105910509F4CBC22436B3
:105BC000314641055105610571058105910511F4C5
:105BD0000C947A3A0C94C13C9101A201B301C40126
:105BE0002737FFE63F07410551056105710581052E
:105BF000910511F40C9430382737EFE63E07410544
:105C00005105610571058105910509F0C0F424363F
:105C1000F9E63F07410551056105710581059105CB
:105C200009F447C625363E46410551056105710513
:105C30008105910511F40C9464380C94C13C9101D8
:105C4000A201B301C4012333F1E73F074105510528
:105C5000610571058105910511F40C947A3A253698
:105C6000324741055105610571058105910511F422
:105C70000C941E390C94C13C9101A201B301C401E2
:105C80002236F5E63F07F4E64F0751056105710539
:105C90008105910509F493C42236E5E63E07E4E662
:105CA0004E075105610571058105910511F008F058
:105CB00051C02133F4E63F07F1E64F075105610576
:105CC00071058105910509F463C22133E4E63E07BD
:105CD000E1E64E075105610571058105910509F061
:105CE000C8F42337F2E73F07410551056105710507
:105CF0008105910511F40C94523A2337334741053D
:105D00005105610571058105910511F40C94663A00
:105D10000C94C13C9101A201B301C4012336F4E605
:105D20003F07F1E64F0751056105710581059105B2
:105D300011F40C947A3A28373446414651056105EE
:105D400071058105910511F00C94C13C0E94581514
:105D50000C94C33C9101A201B301C4012D36F5E7B7
:105D60003F07F8E64F07510561057105810591056B
:105D700011F40C94903A2D36E5E73E07E8E64E071D
:105D80005105610571058105910509F0E0F422379F
:105D9000F2E73F07F5E64F075105610571058105FB
:105DA000910511F40C94773723363D46484651054A
:105DB000610571058105910511F00C94C13C0E94AB
:105DC000D0150C94C33C9101A201B301C401233648
:105DD000F2E33F07F9E64F075105610571058105BB
:105DE000910509F4F5C1243633464C465105610549
:105DF00071058105910511F00C94C13C0E94195A5E
:105E00000C94C33C9101A201B301C4012037FCE60C
:105E10003F07F5E64F07F8E65F0761057105810565
:105E2000910509F412C42037ECE63E07E5E64E077B
:105E3000E8E65E07610571058105910511F008F03E
:105E4000C1C02437F8E73F07F4E74F075105610564
:105E500071058105910509F4D5C52437E8E73E07AA
:105E6000E4E74E075105610571058105910511F0C3
:105E700008F051C02133F1E33F07F1E74F07510527
:105E8000610571058105910511F40C94CA37213320
:105E9000E1E33E07E1E74E07510561057105810524
:105EA000910509F0D0F42537F3E63F07FDE64F07EB
:105EB0005105610571058105910511F40C94CA37EE
:105EC0002033314341475105610571058105910535
:105ED00011F40C9477370C94C13C9101A201B301E9
:105EE000C4012037F5E63F07F2E74F07510561058A
:105EF00071058105910511F40C941E392C36344737
:105F000044475105610571058105910511F40C9413
:105F1000FE3B0C94C13C9101A201B301C40129369E
:105F2000FCE63F07F1E64F07F3E65F076105710501
:105F30008105910509F481C12936ECE63E07E1E6C9
:105F40004E07E3E65E07610571058105910509F0DD
:105F5000E0F42437F4E63F07F7E74F075105610502
:105F600071058105910511F40C944C3C24373F4692
:105F70004F465246610571058105910511F00C945B
:105F8000C13C0C9400000C94C33C9101A201B301EC
:105F9000C4012E36F1E63F07F8E64F07F3E65F0748
:105FA000610571058105910509F401C5263339465E
:105FB00045475546610571058105910509F449C3B9
:105FC0000C94C13C9101A201B301C4012437F3E751
:105FD0003F07F5E64F07F2E75F07610571058105A9
:105FE000910511F40C94DE382437E3E73E07E5E62B
:105FF0004E07E2E75E07610571058105910511F025
:1060000008F053C02337F5E63F07F2E74F07F0E704
:106010005F07610571058105910511F40C94403B02
:106020002337E5E63E07E2E74E07E0E75E07610556
:1060300071058105910509F0D0F42136FDE63F0791
:10604000F5E74F07F8E65F076105710581059105E2
:1060500011F40C944E3822373747404750476105BA
:1060600071058105910509F4B7C00C94C13C9101FB
:10607000A201B301C4012337F2E73F07F7E74F0757
:10608000F0E75F07610571058105910511F40C9436
:10609000E13821363C464546524761057105810588
:1060A000910509F4F3C20C94C13C9101A201B30122
:1060B000C4012437F2E73F07F1E64F07F5E75F0732
:1060C000610571058105910509F469C32437E2E78B
:1060D0003E07E1E64E07E5E75E07610571058105CC
:1060E000910509F0C8F42437F3E73F07F5E64F07B9
:1060F000F4E75F07610571058105910509F4ABC4FB
:106100002737304748475447610571058105910598
:1061100009F422C40C94C13C9101A201B301C40151
:106120002237F7E63F07F0E74F07F5E75F0761051E
:1061300071058105910509F435C62C363146444771
:106140005847610571058105910511F40C94C83B10
:106150000C94C13C84E08093982385E0809399233C
:1061600010929A2310929B2310929C2381E080939B
:106170009D2310929E2310929F231092A02348E902
:1061800053E262E18AE292E00E943D4D0C94C33CEE
:1061900021E04CE061E080ED0E94685A21E04EE091
:1061A00061E080ED0E94685A21E040E161E080ED0D
:1061B0000E94685A21E042E161E080ED0E94685A45
:1061C00022E040E161E080ED0E94685A0C94C33CFB
:1061D0000E94CA0F0C94C33C60916A0270916B02DA
:1061E00080E090E00E94CA8A8C0169E675E00E9416
:1061F000DE8A892B19F477980C94C33C6CE675E021
:10620000C8010E94DE8A892B19F4779A0C94C33C4A
:10621000779903C089E695E002C08CE695E09F93EC
:106220008F9385EC94E09F938F930E947B8B0F90CC
:106230000F900F900F900C94C33C60916A02709184
:106240006B0280E090E00E94CA8A8C0163E375E0F3
:106250000E94DE8A892B09F077C060916A027091F2
:106260006B0280E090E00E94CA8A8C01009711F4D2
:106270000C94C33C67E775E00E94DE8A892BB1F479
:1062800082E29FEFACECBBE38093710290937202C9
:10629000A0937302B093740244E050E066E270E0B1
:1062A00081E792E00E94BE8C0C94C33C6DE775E0E0
:1062B000C8010E94DE8A892BB1F482E29FEFACEC28
:1062C000BAE38093710290937202A0937302B09329
:1062D000740244E050E066E270E081E792E00E94E0
:1062E000BE8C0C94C33CC8010E94B4892B013C01B4
:1062F00020E030E0A9010E9453818823D9F081E099
:106300000E94DF099B01AC01C301B2010E945781C9
:10631000609371027093720280937302909374027F
:1063200044E050E066E270E081E792E00E94BE8CBB
:106330000C94C33C84ED92E09F938F930E947B8BDF
:106340000F900F900C94C33C66E375E0C8010E9467
:10635000DE8A892B09F077C060916A0270916B0226
:1063600080E090E00E94CA8A8C01009711F40C949E
:10637000C33C67E775E00E94DE8A892BB1F482E2B4
:106380009FEFACECBBE380936D0290936E02A09301
:106390006F02B093700244E050E062E270E08DE67C
:1063A00092E00E94BE8C0C94C33C6DE775E0C8017E
:1063B0000E94DE8A892BB1F482E29FEFACECBAE353
:1063C00080936D0290936E02A0936F02B09370025F
:1063D00044E050E062E270E08DE692E00E94BE8C04
:1063E0000C94C33CC8010E94B4892B013C0120E0FD
:1063F00030E0A9010E9453818823D9F082E00E94F5
:10640000DF099B01AC01C301B2010E945781609377
:106410006D0270936E0280936F029093700244E05D
:1064200050E062E270E08DE692E00E94BE8C0C9437
:10643000C33C87EC92E09F938F930E947B8B0F90DD
:106440000F900C94C33C6EE275E0C8010E94DE8A96
:10645000892B09F073C060916A0270916B0280E031
:1064600090E00E94CA8A8C01009711F40C94C33CFE
:1064700067E775E00E94DE8A892BB1F487ED94E32B
:10648000AFEEBCE38093750290937602A0937702FF
:10649000B093780244E050E06AE270E085E792E071
:1064A0000E94BE8C0C94C33C6DE775E0C8010E944D
:1064B000DE8A892B51F488EB92E09F938F930E94A0
:1064C0007B8B0F900F900C94C33CC8010E94B48941
:1064D0002B013C0120E030E0A9010E945381882378
:1064E00019F180E00E94DF094B015C0121EE3AE7DF
:1064F00044E95EE3C301B2010E948C80A5019401CE
:106500000E945781609375027093760280937702A0
:106510009093780244E050E06AE270E085E792E010
:106520000E94BE8C0C94C33C8BEA92E09F938F93A5
:106530000E947B8B0F900F900C94C33C0E942E0AFC
:106540009F938F937F936F9384EA92E09F938F93AF
:106550000E947B8B82E00E94DF0920916D023091C6
:106560006E0240916F02509170020E94D483162FE8
:10657000072FF82EE92E81E00E94DF09EF92FF92AB
:106580000F931F9320917102309172024091730218
:10659000509174020E94D4839F938F937F936F9343
:1065A00088E992E09F938F930E947B8B0E94480B17
:1065B0000FB6F894DEBF0FBECDBF0C94C33C609104
:1065C0006A0270916B0280E090E00E94CA8A009794
:1065D000C1F00E94E2222091490930914A098217B4
:1065E000930709F190934A098093490942E050E0EA
:1065F0006EE270E089E499E00E94BE8C8EEB94E03C
:1066000002C087EB94E09F938F930E947B8B6091F5
:10661000490970914A0980E090E00E94F4210E94AB
:10662000480B0F900F908CEA94E09F938F930E94F9
:106630007B8B6FEF7FEF80E090E00E94F4210E945F
:10664000480B0F900F900C94C33C0E94071F0C94B2
:10665000C33C8091A723843329F440E061E080E0CB
:106660000E94741180916C02882311F40C94C33C35
:106670001F928F9389EA94E09F938F930E947B8B64
:106680000F900F900F900F900C94C33C8091A72314
:10669000893709F070C060916A0270916B0280E0E6
:1066A00090E00E94CA8A8C0169E675E00E94DE8A49
:1066B000892B31F480914A0290914B0290640CC076
:1066C0006CE675E0C8010E94DE8A892B91F4809106
:1066D0004A0290914B029F7B90934B0280934A0217
:1066E00042E050E066E170E08AE492E00E94BE8CF5
:1066F00042C062E875E0C8010E94DE8A892B21F55C
:106700008091AE1A8F938091AD1A8F938091AC1ABD
:106710008F938091AB1A8F938091AA1A8F93809157
:10672000A91A8F938091A81A8F938091A71A8F939B
:106730008DE692E09F938F930E947B8B0FB6F89427
:10674000DEBF0FBECDBF17C080914A0290914B02B1
:1067500096FF03C089E695E002C08CE695E09F9322
:106760008F9389E692E09F938F930E947B8B0F908B
:106770000F900F900F9080916C02882311F40C946D
:10678000C33C1F928F9386EA94E09F938F930E945D
:106790007B8B0F900F900F900F900C94C33C6091E7
:1067A0006A0270916B0280E090E00E94CA8A5C01EC
:1067B00068E875E00E94DE8A892B11F489E108C03F
:1067C0006CE875E0C5010E94DE8A892B49F480E1FE
:1067D0008093C4001092C50082E08093C00055C031
:1067E00060E975E0C5010E94DE8A892B11F488E01A
:1067F000EFCF65E975E0C5010E94DE8A892B39F08B
:106800006AE975E0C5010E94DE8A892B11F483E0F4
:10681000DFCF8091C400893141F484E692E09F93F8
:106820008F930E947B8B0F900F908091C4008031DA
:1068300041F48FE592E09F938F930E947B8B0F90A2
:106840000F908091C400883041F489E592E09F93D5
:106850008F930E947B8B0F900F908091C4008330A8
:1068600041F483E592E09F938F930E947B8B0F907E
:106870000F908091C400883041F48DE492E09F93A2
:106880008F930E947B8B0F900F9080916C028823D6
:1068900011F40C94C33C1F928F9383EA94E09F936E
:1068A0008F930E947B8B0F900F900F900F900C9402
:1068B000C33C60916A0270916B0280E090E00E949C
:1068C000CA8A67E775E00E94DE8A892B11F481E0AD
:1068D00001C080E00E94C42180916C02882311F4E1
:1068E0000C94C33C1F928F9380EA94E09F938F9304
:1068F0000E947B8B0F900F900F900F900C94C33CD5
:106900000E94EA1F80916C02882311F40C94C33C0E
:106910001F928F938DE994E09F938F930E947B8BBE
:106920000F900F900F900F900C94C33C0E94E61FA5
:1069300080916C02882311F40C94C33C1F928F93B6
:106940008AE994E09F938F930E947B8B0F900F9026
:106950000F900F900C94C33C60916A0270916B028F
:1069600080E090E00E94CA8A0E94B889803178F461
:106970008093450999270E94156341E050E065E145
:1069800070E085E499E00E94BE8C0C94C33C809139
:1069900045091F928F9383E492E09F938F930E9407
:1069A0007B8B0F900F900F900F900C94C33C6091D5
:1069B0006A0270916B0280E090E00E94CA8A0E9495
:1069C000B88925EF280F203170F480934902992768
:1069D0000E94CB6141E050E064E170E089E492E024
:1069E0000E94BE8CD0C7809149021F928F938AE388
:1069F00092E09F938F930E947B8B0F900F900F904C
:106A00000F90C1C760916A0270916B0280E090E0C4
:106A10000E94CA8A009781F04AE050E0BC0182E9F6
:106A20009AE10E94EE8A4AE050E060E070E082E97C
:106A30009AE10E94BE8CA7C782E99AE19F938F9347
:106A40008FE995E09F938F930E94698B0F900F9031
:106A50000F900F9098C760916A0270916B0280E06E
:106A600090E00E94CA8A5C0167E674E00E94DE8AB8
:106A7000892B99F4219A80914A0290914B0280616E
:106A800090934B0280934A0242E050E066E170E04E
:106A90008AE492E00E94BE8C76C767E375E0C50188
:106AA0000E94DE8A892B99F4229A80914A02909161
:106AB0004B02806290934B0280934A0242E050E086
:106AC00066E170E08AE492E00E94BE8C5CC763EBF2
:106AD00073E0C5010E94DE8A892B99F4239A809184
:106AE0004A0290914B02806490934B0280934A0239
:106AF00042E050E066E170E08AE492E00E94BE8CE1
:106B000042C76EED74E0C5010E94DE8A892B99F4BC
:106B1000239A80914A0290914B02806890934B0295
:106B200080934A0242E050E066E170E08AE492E03D
:106B30000E94BE8C28C760EF78E0C5010E94DE8A03
:106B4000892B09F040C081E0809398238091520204
:106B5000809399238091530280939A2380915402C9
:106B600080939B238091550280939C2380915602B1
:106B700080939D238091570280939E238091580299
:106B800080939F23809159028093A0231092A22387
:106B90001092A12380914A0290914B0291609093B0
:106BA0004B0280934A0242E050E066E170E08AE4E2
:106BB00092E00E94BE8C48E953E262E18AE292E0F0
:106BC0000E943D4DE0C66AED73E0C5010E94DE8A79
:106BD000892BD1F4E7EBFAE1119211929AE1E73DAA
:106BE000F907D1F780914A0290914B0292609093FD
:106BF0004B0280934A0242E050E066E170E08AE492
:106C000092E00E94BE8CBFC66CE675E0C5010E9492
:106C1000DE8A20914A0230914B02892BA9F42F7011
:106C20003C7F30934B0220934A022B9A42E050E083
:106C300066E170E08AE492E00E94BE8C8091EF27CA
:106C400090E00E94E0619FC624FF03C089E695E0C2
:106C500002C08CE695E09F938F938FE292E09F9322
:106C60008F930E947B8B80914A020F900F900F9020
:106C70000F9085FF03C089E695E002C08CE695E0A1
:106C80009F938F9384E292E09F938F930E947B8BDC
:106C900080914A020F900F900F900F9086FF03C0D3
:106CA00089E695E002C08CE695E09F938F9389E199
:106CB00092E09F938F930E947B8B80914A020F906A
:106CC0000F900F900F9087FF03C089E695E002C0F8
:106CD0008CE695E09F938F938EE092E09F938F9345
:106CE0000E947B8B80914A0290914B020F900F90F3
:106CF0000F900F9090FF03C089E695E002C08CE6EC
:106D000095E09F938F9383E092E09F938F930E94EF
:106D10007B8B80914A0290914B020F900F900F90C5
:106D20000F9091FF03C089E695E002C08CE695E0E4
:106D30009F938F9388EF91E09F938F930E947B8B1B
:106D400080914A0290914B020F900F900F900F90FC
:106D500091FF19C687EA95E00E949F8B47EBA42E0E
:106D60004AE1B42E0BE010E05FEA852E55E0952E47
:106D7000F50180819181F2E0AF0EB11C9F938F935A
:106D80001F930F939F928F920E94698B0F5F1F4FEB
:106D90000F900F900F900F900F900F900B311105E7
:106DA00039F7F1C586E994E09F938F930E947B8B1E
:106DB00080916C020F900F90882361F01F928F9347
:106DC00083E994E09F938F930E947B8B0F900F90A9
:106DD0000F900F9088E10FB6F894809360001092A6
:106DE00060000FBE0C94007CCEC560916A02709169
:106DF0006B0280E090E00E94CA8A8C0169E675E02F
:106E00000E94DE8A892BA9F40E94CA6080914A02FE
:106E100090914B028D7F816090934B0280934A0248
:106E200042E050E066E170E08AE492E00E94BE8CAD
:106E3000AAC56CE675E0C8010E94DE8A892BA1F420
:106E40000E94826080914A0290914B028C7F9093C5
:106E50004B0280934A0242E050E066E170E08AE42F
:106E600092E00E94BE8C8FC56AEB75E0C8010E945B
:106E7000DE8A892BA9F40E94826080914A02909157
:106E80004B028E7F826090934B0280934A0242E0D5
:106E900050E066E170E08AE492E00E94BE8C73C527
:106EA00080914A0281FF0FC08AEB95E09F938F93F8
:106EB00084EF91E09F938F930E947B8B0F900F90B4
:106EC0000F900F9060C580FF03C089E695E002C077
:106ED0008CE695E09F938F9380EF91E09F938F9343
:106EE0000E947B8B0F900F900F900F904CC589E6FE
:106EF00094E09F938F930E947B8B809192238F933A
:106F0000809191238F93809190238F9380918F23F1
:106F10008F9380918E238F9380918D238F93809177
:106F20008C238F9380918B238F9380918A238F93CF
:106F3000809189238F93809188238F9380918723D9
:106F40008F93809196238F93809195238F93809137
:106F500094238F93809193238F938BE494E09F935A
:106F60008F930E947B8B80916C020FB6F894DEBFEA
:106F70000FBECDBF882309F406C51F928F9388E406
:106F800094E09F938F930E947B8B0F900F900F90B4
:106F90000F90F9C4F89481E090E029E0FC0120937F
:106FA0005700C895E02C80E090E0FC01209357004A
:106FB000C895F02C7894F89483E090E0FC0120933D
:106FC0005700C895002D82E090E0FC012093570007
:106FD000C895102D789480912B1B8F9380912A1B3C
:106FE0008F938091291B8F938091281B8F932EE381
:106FF00034E03F932F930E947B8B1F92EF921F925E
:10700000FF921F920F931F921F9387E194E09F932B
:107010008F930E947B8B0E948420809166001F9238
:107020008F938BE094E09F938F930E947B8B0E94C1
:10703000480B80916C020FB6F894DEBF0FBECDBF37
:10704000882309F4A0C41F928F9388E094E09F9353
:107050008F930E947B8B0F900F900F900F9093C493
:1070600060E070E080E090E00E94510B60E070E032
:1070700081E090E00E94510B80916C02882309F41A
:1070800082C41F928F9385E094E09F938F930E9418
:107090007B8B0F900F900F900F9075C40E948D1EE8
:1070A0000E94480B80916C02882309F46CC41F92E3
:1070B0008F9382E094E09F938F930E947B8B0F903D
:1070C0000F900F900F905FC460916A0270916B02F5
:1070D00080E090E00E94CA8A6FEB75E00E94DE8A31
:1070E000892B31F5F89480E899E00E942A4E5C01E2
:1070F000009769F0C5010F960E942E51B50184E0FA
:1071000092E00E94E44DC5010E94D24EF0CF80E88B
:1071100099E00E94B74E892B29F080E899E00E94FF
:10712000634EF5CF80E899E00E94264E789434C0F3
:1071300080E899E00E942A4E5C0105EC15E0A1145C
:10714000B10451F1F50186811F928F9380851F92C2
:107150008F9385811F928F9381851F928F93878153
:107160001F928F9384811F928F9383811F928F939D
:1071700082811F928F9382851F928F931F930F930B
:107180000E94698BC5010E94D24E5C010FB6F89433
:10719000DEBF0FBECDBFD3CF80916C02882309F430
:1071A000F2C31F928F938FEF93E09F938F930E9470
:1071B0007B8B0F900F900F900F90E5C30E948E2B4A
:1071C000E2C360916A0270916B0280E090E00E94DD
:1071D000CA8A8C0164E076E00E94DE8A892B91F4F1
:1071E00080914A0290914B02977F90934B0280933B
:1071F0004A0242E050E066E170E08AE492E00E94D8
:10720000BE8CC1C36DE775E0C8010E94DE8A892B80
:1072100091F480914A0290914B02986090934B02B6
:1072200080934A0242E050E066E170E08AE492E036
:107230000E94BE8CA8C30E94E508A5C360916A02A3
:1072400070916B0280E090E00E94CA8A009709F476
:10725000A8C01982BE016F5F7F4F0E94C626390108
:107260004A01B62FA72FF82FE92F20905202309015
:1072700053024090540250905502309156023A8386
:10728000809157028B83909158029C8320915902E0
:107290002D839301A4016B2F7A2F8F2F9E2F5101E5
:1072A0006201EA80FB800C811D810E94FB8609F44B
:1072B0008CC0898181110FC060925202709253027A
:1072C0008092540290925502B0935602A0935702B6
:1072D000F09358023FC01816DCF462286092520204
:1072E00073287092530284288092540295289092B9
:1072F00055023A81B32BB09356028B81A82BA093F1
:1073000057029C81F92BF0935802FD81EF2B22C08C
:107310006094709480949094B095A095F095E095C9
:1073200062206092520273207092530284208092F5
:1073300054029520909255022A81B223B0935602AE
:107340003B81A323A09357028C81F823F09358022A
:10735000FD81EF23E093590248E050E06AE170E0DC
:1073600082E592E00E94BE8C87EF93E09F938F931B
:107370000E947B8B20915202309153024091540223
:1073800050915502609156027091570280915802B7
:10739000909159020E947D230E94480B0F900F90FC
:1073A00014C02091520230915302409154025091E6
:1073B0005502609156027091570280915802909147
:1073C00059020E947D230E94480B8BEE93E09F930D
:1073D0008F930E947B8B2FEF3FEF4FEF5FEF60E0CB
:1073E00070E080E090E00E947D230E94480B809135
:1073F0006C020F900F90882309F4C5C21F928F93DF
:1074000088EE93E09F938F930E947B8B0F900F9059
:107410000F900F90B8C260916A0270916B0280E089
:1074200090E00E94CA8A0097D9F04AE050E060E0FC
:1074300070E00E94A08860935002709351027F9385
:107440006F938BEC93E09F938F930E947B8B42E032
:1074500050E068E170E080E592E00E94BE8C0CC0D4
:10746000809151028F93809150028F938AEA93E02A
:107470009F938F930E947B8B0F900F900F900F9094
:1074800080916C02882309F47EC21F928F9387EA51
:1074900093E09F938F930E947B8B0F900F900F90A0
:1074A0000F9071C20E94675180916C02882309F489
:1074B0006AC21F928F9384EA93E09F938F930E94F6
:1074C0007B8B0F900F900F900F905DC20E945A28F7
:1074D00080916C02882309F456C21F928F9381EA2F
:1074E00093E09F938F930E947B8B0F900F900F9050
:1074F0000F9049C280E090E00E94A02080916C0231
:10750000882309F440C21F928F938EE993E09F93E2
:107510008F930E947B8B0F900F900F900F9033C230
:1075200080917D1F81FF2DC00E94D01D892B49F5C0
:107530008091741B8F938091731B8F938091721B2A
:107540008F938091711B8F9383E993E09F938F9327
:107550000E947B8B809107288F93809106288F93C0
:10756000809105288F93809104288F9386E893E07B
:107570009F938F930E947B8B0FB6F894DEBF0FBE54
:10758000CDBF0E94480B80917D1F90917E1F90FF80
:1075900063C081E090E00E94801D3B014C0180E0CF
:1075A00090E00E94801D1B012C010E94FF1C9F92F5
:1075B0008F927F926F9285E793E09F938F930E94C3
:1075C0007B8B5F924F923F922F9285E693E09F9341
:1075D0008F930E947B8B222D332D442D552D662DAC
:1075E000772D882D992D0E94E61B9F938F937F9373
:1075F0006F938AE593E09F938F930E947B8B222D5C
:10760000332D442D552D662D772D882D992D0E94D3
:10761000471C9F938F937F936F938CE493E09F938A
:107620008F930E947B8B222D332D442D552D662D5B
:10763000772D882D992D0E94A81C9F938F937F935F
:107640006F9389E393E09F938F930E947B8B0FB698
:10765000F894DEBF0FBECDBF0E94480B80916C0234
:10766000882309F490C11F928F9386E393E09F9340
:107670008F930E947B8B0F900F900F900F9083C180
:1076800080917D1F82FF2BC021E048E061E083E014
:107690000E94E91280916F1B8F9380916E1B8F93D4
:1076A00080916D1B8F9380916C1B8F9380916B1BCE
:1076B0008F9380916A1B8F938091691B8F93809128
:1076C000681B8F938FE193E09F938F930E947B8B36
:1076D0000E94480B0FB6F894DEBF0FBECDBF80915D
:1076E0007D1F90917E1F91FF41C00E943317B62EDF
:1076F000A72E982E892E20E030E048EC52E4D501E8
:10770000F4016B2F7A2F8F2F9E2F0E94D48320E8B5
:1077100036EE45EC57E40E94578121E03EED42E40D
:107720005EE30E9437849B01AC0160E070E080E87A
:107730009FE30E948C802BE43AE34DEB57E30E94D9
:1077400057819F938F937F936F938F929F92AF9266
:10775000BF9286E093E09F938F930E947B8B0E9461
:10776000480B0FB6F894DEBF0FBECDBF80916C0200
:10777000882309F408C11F928F9383E093E09F93BD
:107780008F930E947B8B0F900F900F900F90FBC0F8
:1077900060916A0270916B0280E090E00E94CA8A58
:1077A00069E076E00E94DE8A892BB1F460916A027A
:1077B00070916B0280E090E00E94CA8A009709F401
:1077C000E2C00E94B889803108F0DDC0909152017A
:1077D000982B90935201D7C0809152018F701F92C5
:1077E0008F9383EE91E09F938F930E947B8B0E94F7
:1077F000480B0F900F900F900F90C5C060916A02D8
:1078000070916B0280E090E00E94CA8A009711F1AB
:107810004AE050E060E070E00E946C87603198F4CC
:10782000609348021F926F9386EF92E09F938F932D
:107830000E947B8B41E050E063E170E088E492E0DD
:107840000E94BE8C11C0809148021F928F938DEED2
:1078500092E006C0809148021F928F9384EE92E0DE
:107860009F938F930E947B8B0F900F900F900F90A0
:107870000E94480B80916C02882309F484C01F92F7
:107880008F9381EE92E09F938F930E947B8B0F905A
:107890000F900F900F9077C060916A0270916B0209
:1078A00080E090E00E94CA8A8C0169E675E00E943F
:1078B000DE8A892BA1F40E94335F80914A02909165
:1078C0004B02906190934B0280934A0242E050E059
:1078D00066E170E08AE492E00E94BE8C54C06CE6DF
:1078E00075E0C8010E94DE8A892B41F5F8940E9458
:1078F000415F88E10FB6F8948093600010926000B9
:107900000FBE84B7877F84BF8091600088618093B9
:10791000600010926000789480914A0290914B022E
:107920009F7E90934B0280934A0242E050E066E1D2
:1079300070E08AE492E00E94BE8C25C06EE076E0A2
:10794000C8010E94DE8A20914A0230914B02892BA5
:1079500021F434FF18C0F894FFCF34FF03C089E648
:1079600095E002C08CE695E09F938F938FED91E0B8
:107970009F938F930E947B8B0F900F900F900F908F
:1079800002C00E94EE1EEE81FF811182108283E010
:1079900027960FB6F894DEBF0FBECDBFDF91CF9113
:1079A0001F910F91FF90EF90DF90CF90BF90AF901D
:1079B0009F908F907F906F905F904F903F902F900F
:1079C00008950E94275F6C9A6B9A6A9A6F9A729ACE
:1079D000749A739A779A809880B3897F80BB8398D2
:1079E000849887E080937E00549A0E94E5290E9443
:1079F000172A81E00E94530980E090E00E949D0CCC
:107A00000E949E5880914A0286FD239A0895CF9342
:107A1000DF93EC0188819981009741F0853F9E407A
:107A200009F47EC01982188283E083C00E94E13C81
:107A300080914A0280FD05C081FF01C01D9B0E940C
:107A40008260809170008C7F809370008091B6007E
:107A500080628093B6001092B20082E08093B10001
:107A60008091B6008770E1F780917000816080930B
:107A700070006FEF78E080E090E00E94115F0E945C
:107A8000E61F80E00E94C42181E29EE09F938F93D5
:107A90000E947B8B0E94CA0F80917D1F0F900F90D8
:107AA00086FD0E94C5598091450990E00E941563AA
:107AB0008091490290E00E94CB610E94C86180934E
:107AC00070098091490290E00E94CB618091450944
:107AD0001F928F93809170091F928F9383E196E09C
:107AE0009F938F930E94698B109272091092710973
:107AF0000F900F900F900F900F900F908EE392E0E9
:107B0000909302288093012883E290E09093831160
:107B10008093821185EF9EE09983888381E009C07C
:107B20006332E1F760E070E081E799E00E94662C43
:107B3000E5CFDF91CF9108958436910514F19F939D
:107B40008F9385E296E09F938F930E94698B80913B
:107B5000932390919423A0919523B091962301961D
:107B6000A11DB11D8093932390939423A0939523FB
:107B7000B09396230F900F900F900F9081E090E0BC
:107B8000089580E090E008952F923F924F925F9287
:107B90006F927F928F929F92AF92BF92CF92DF921D
:107BA000EF92FF920F931F93CF93DF93CDB7DEB782
:107BB000C559D1090FB6F894DEBF0FBECDBFC4576B
:107BC000DF4F99838883CC58D040633871F485E7C0
:107BD00099E0CB56DF4F6883C559D0400E94804B57
:107BE000CB56DF4F6881C559D040C457DF4FE8817D
:107BF000F981CC58D04020813181293AFEE03F07FD
:107C0000F9F040F42115310581F027313D4009F4A8
:107C100085C079C02A3B8EE0380709F455C0213C65
:107C20003E4011F40C94C3486EC04FED52E061E841
:107C300070E085E799E00E94664B87E19DE058C0BF
:107C400000E010E020914A0230914B0230FF1EC04C
:107C50007398809169098F5F809369098A83B8015D
:107C60006F5F7F4FCE0101960E94AF5485E799E088
:107C70000E94824B40E050E065E88091861190912F
:107C800087110E943D4D89EA9EE032C08D2D90E023
:107C90000E94E061F0925102E0925002739A80914A
:107CA000460990914709892B11F00E9482608091CA
:107CB00069098F5F809369098091490990914A0908
:107CC00082FFBBCF739AB9CF81E699E00E94E34F60
:107CD000892BB1F00E94CA6080914A0287FD2B98DF
:107CE00060E470E081E699E00E94BC4F81EC9EE088
:107CF000C457DF4FE881F981CC58D040918380830D
:107D000081E00C94D648C457DF4FE881F981CC5804
:107D1000D0401182108283E00C94D648623181F702
:107D200080914A0290914B0291FD87CF80919823D8
:107D3000813039F58090992390909A23A0909B23CD
:107D4000B0909C23F0919D23C257DF4FF883CE580B
:107D5000D04020919E23C157DF4F2883CF58D04079
:107D600030919F23C057DF4F3883C059D040409196
:107D7000A023CF56DF4F4883C159D040212C312C4E
:107D80002FC0823049F58090992390909A23A0903B
:107D90009B23B0909C2350919D23C257DF4F588363
:107DA000CE58D04080919E23C157DF4F8883CF5853
:107DB000D04090919F23C057DF4F9883C059D04047
:107DC000E091A023CF56DF4FE883C159D0402090E7
:107DD000A1233090A22304C0843009F02ECFAACF73
:107DE000FA2DF470C657DF4FF883CA58D04020E010
:107DF00030E04F2F50E060E070E080E090E0A0E0E5
:107E00000E94048709F08C9AB401C5010E94880A77
:107E1000292D2074C557DF4F2883CB58D04020E050
:107E2000C557DF4F3881CB58D04040E050E060E08C
:107E300070E080E090E0A0E00E94048711F00E94D2
:107E4000D01D392D3078CE56DF4F3883C259D040FF
:107E500020E040E050E060E070E080E090E0A0E0F2
:107E60000E94048751F00E942E0A6093EB277093C2
:107E7000EC278093ED279093EE27282D217030E09A
:107E800040E050E060E070E080E090E0A0E00E9420
:107E90000487F1F082E99AE19F938F9389E396E05A
:107EA0009F938F931F9287E78F93CE0103969F93A3
:107EB0008F930E94CC8B7C010E949C3D0FB6F8945E
:107EC000DEBF0FBECDBF892B09F0B7CE870102C040
:107ED00000E010E0282D227030E040E050E060E04B
:107EE00070E080E090E0A0E00E940487C9F1C80142
:107EF000029661E476E0E1E0F0E0EC0FFD1F8E0F0A
:107F00009F1F0E94E78A0D5F1F4FA8EFCA2EA7E2AE
:107F1000DA2EB3EEEB2EB3E0FB2E87E7782EF601D8
:107F200081916F011F928F93FF92EF921F927F9228
:107F3000C801029621E030E02C0F3D1F820F931FF5
:107F40009F938F930E94CC8B080F191F0FB6F89444
:107F5000DEBF0FBECDBF50E0C51658E2D506F9F61C
:107F6000282D247030E040E050E060E070E080E0D8
:107F700090E0A0E00E94048709F446C0C801029680
:107F800065E476E0E1E0F0E0EC0FFD1F8E0F9F1F4F
:107F90000E94E78A0C5F1F4F6E01FAE7CF0ED11CDB
:107FA00080E1F60111928A95E9F728E0A60168E9D7
:107FB00080EB0E942D113601F8E06F0E711CE3EE8C
:107FC000EE2EE3E0FE2EF7E75F2EF60181916F01C2
:107FD0001F928F93FF92EF921F925F92C8010296B9
:107FE00021E030E02C0F3D1F820F931F9F938F9352
:107FF0000E94CC8B080F191F0FB6F894DEBF0FBE7E
:10800000CDBFC614D70409F75B2D5078CD56DF4F8E
:108010005883C359D04020E030E040E060E070E099
:1080200080E090E0A0E00E94048701F5809146097D
:10803000909147099F938F938AE496E09F938F9343
:108040001F9287E78F93C8010296E1E0F0E0EC0F02
:10805000FD1F8E0F9F1F9F938F930E94CC8B080F45
:10806000191F0FB6F894DEBF0FBECDBF20E030E081
:1080700040E050E0C257DF4F6881CE58D040617079
:1080800070E080E090E0A0E00E94048709F1E3E066
:10809000F0E0EC0FFD1FE00FF11F80E28083E6EAC5
:1080A000F3E280810F5F1F4F882359F08081A1E0A8
:1080B000B0E0AC0FBD1FA00FB11F12968C9331968C
:1080C000F0CFE3E0F0E0EC0FFD1FE00FF11F1082B6
:1080D000282D287030E040E050E060E070E080E063
:1080E00090E0A0E00E940487C1F127E04AE250E05E
:1080F0006BE270E089E290E00E94B85588EF97E269
:108100000E942658BC01882777FD8095982F0E94F1
:10811000F68120E030E048EC52E40E9457819F93C2
:108120008F937F936F9381E596E09F938F931F9238
:1081300087E78F93C801029641E050E04C0F5D1F26
:10814000840F951F9F938F930E94CC8B080F191F4C
:108150000FB6F894DEBF0FBECDBF282D207130E0E2
:1081600040E050E060E070E080E090E0A0E00E943D
:108170000487F1F126E04AE250E06BE270E089E228
:1081800090E00E94B85581E090E00E94D60A80936A
:10819000440980EE9AE10E942658BC01882777FDA9
:1081A0008095982F0E94F68120E030E048EC52E460
:1081B0000E9457819F938F937F936F938BE596E0F7
:1081C0009F938F931F9287E78F93C8010296E1E0F8
:1081D000F0E0EC0FFD1F8E0F9F1F9F938F930E9467
:1081E000CC8B080F191F0FB6F894DEBF0FBECDBFA2
:1081F000282D207230E040E050E060E070E080E048
:1082000090E0A0E00E94048731F180919F1A8F9343
:1082100080919E1A8F9380919D1A8F9380919C1AC2
:108220008F9386E696E09F938F931F9287E78F93B5
:10823000C801029641E050E04C0F5D1F840F951F6E
:108240009F938F930E94CC8B080F191F0FB6F89441
:10825000DEBF0FBECDBF282D207430E040E050E0DF
:1082600060E070E080E090E0A0E00E94048731F1DF
:10827000809182238F93809181238F93809180239B
:108280008F9380917F238F9384E796E09F938F93C2
:108290001F9287E78F93C8010296E1E0F0E0EC0FB0
:1082A000FD1F8E0F9F1F9F938F930E94CC8B080FF3
:1082B000191F0FB6F894DEBF0FBECDBF282D207852
:1082C00030E040E050E060E070E080E090E0A0E06E
:1082D0000E94048741F1F8948091E3279091E4276C
:1082E000A091E527B091E6277894BF93AF939F9331
:1082F0008F9382E896E09F938F931F9287E78F93E7
:10830000C801029641E050E04C0F5D1F840F951F9D
:108310009F938F930E94CC8B080F191F0FB6F89470
:10832000DEBF0FBECDBF20E0392D317040E050E000
:1083300060E070E080E090E0A0E00E94048709F433
:1083400077C08091500290915102892B09F470C03E
:10835000F894C090E327D090E427E090E527F090D0
:10836000E62778948091D81A9091D91AA091DA1AB8
:10837000B091DB1AA7019601281B390B4A0B5B0B46
:10838000CA01B9010E94F4812B013C0160915002A5
:108390007091510280E090E00E94F4819B01AC0159
:1083A000C301B2010E9457813C017F928F937F935A
:1083B0006F938DE896E09F938F931F9287E78F933B
:1083C0009E01200F311F2D5F3F4F3F932F93CB56C0
:1083D000DF4F6883C559D040CC56DF4F7883C459EE
:1083E000D0400E94CC8B080F191FCB56DF4F6881FD
:1083F000C559D040CC56DF4F7881C459D040862F24
:10840000972FA62DB72D8093F0279093F127A09357
:10841000F227B093F327C092D81AD092D91AE092DB
:10842000DA1AF092DB1A0FB6F894DEBF0FBECDBF9A
:1084300020E0392D327040E050E060E070E080E0F4
:1084400090E0A0E00E94048791F180915002909109
:108450005102892B61F1F8948091AF1A9091B01A72
:10846000A091B11AB091B21A78949F938F93809192
:108470004F028F9380914E028F938AE996E09F93EB
:108480008F931F9287E78F93C8010296E1E0F0E097
:10849000EC0FFD1F8E0F9F1F9F938F930E94CC8B1D
:1084A000080F191F0FB6F894DEBF0FBECDBF20E036
:1084B000392D347040E050E060E070E080E090E002
:1084C000A0E00E94048771F1F8948091E7279091D1
:1084D000E827A091E927B091EA277894BF93AF935A
:1084E0009F938F938AEA96E09F938F931F9287E7DB
:1084F0008F93C801029641E050E04C0F5D1F840F3E
:10850000951F9F938F930E94CC8B080F191FC80152
:108510000E949C3D0FB6F894DEBF0FBECDBF892BE5
:1085200009F08BCB20E0392D387040E050E060E05E
:1085300070E080E090E0A0E00E94048709F477C03A
:108540008091500290915102892B09F470C0F894E7
:10855000C090E727D090E827E090E927F090EA273D
:1085600078948091DC1A9091DD1AA091DE1AB09176
:10857000DF1AA7019601281B390B4A0B5B0BCA01B6
:10858000B9010E94F4812B013C016091500270916D
:10859000510280E090E00E94F4819B01AC01C30194
:1085A000B2010E9457813C017F928F937F936F931A
:1085B00085EB96E09F938F931F9287E78F939E01A1
:1085C000200F311F2D5F3F4F3F932F93CB56DF4F2F
:1085D0006883C559D040CC56DF4F7883C459D0400A
:1085E0000E94CC8B080F191FCB56DF4F6881C559ED
:1085F000D040CC56DF4F7881C459D040862F972F7A
:10860000A62DB72D8093F4279093F527A093F627F6
:10861000B093F727C092DC1AD092DD1AE092DE1AEE
:10862000F092DF1A0FB6F894DEBF0FBECDBF20E088
:10863000392D307140E050E060E070E080E090E083
:10864000A0E00E94048791F1809150029091510224
:10865000892B61F1F8948091B31A9091B41AA0918A
:10866000B51AB091B61A78949F938F9380914D026A
:108670008F9380914C028F9382EC96E09F938F931F
:108680001F9287E78F93C8010296E1E0F0E0EC0FBC
:10869000FD1F8E0F9F1F9F938F930E94CC8B080FFF
:1086A000191F0FB6F894DEBF0FBECDBF20E0392DE5
:1086B000307240E050E060E070E080E090E0A0E0E8
:1086C0000E94048761F18091832390918423A0917B
:1086D0008523B0918623BF93AF939F938F9382EDB1
:1086E00096E09F938F931F9287E78F93C80102961E
:1086F00041E050E04C0F5D1F840F951F9F938F93B7
:108700000E94CC8B080F191FC8010E949C3D0FB618
:10871000F894DEBF0FBECDBF892B09F08ECA20E0D2
:10872000C557DF4F3881CB58D04040E050E060E083
:1087300070E080E090E0A0E00E94048761F1809109
:10874000741B8F938091731B8F938091721B8F93F7
:108750008091711B8F938DED96E09F938F931F9265
:1087600087E78F93C801029621E030E02C0F3D1F70
:10877000820F931F9F938F930E94CC8B080F191F1A
:10878000C8010E949C3D0FB6F894DEBF0FBECDBF5E
:10879000892B09F052CA20E0CE56DF4F3881C259EA
:1087A000D04040E050E060E070E080E090E0A0E089
:1087B0000E94048761F18091EE278F938091ED27CD
:1087C0008F938091EC278F938091EB278F9388EE86
:1087D00096E09F938F931F9287E78F93C80102962D
:1087E000E1E0F0E0EC0FFD1F8E0F9F1F9F938F9332
:1087F0000E94CC8B080F191FC8010E949C3D0FB628
:10880000F894DEBF0FBECDBF892B09F016CA20E059
:1088100030E04A2D417050E060E070E080E090E090
:10882000A0E00E94048789F181E00E94DF09209185
:1088300071023091720240917302509174020E9451
:10884000D4839F938F937F936F9385EF96E09F934D
:108850008F931F9287E78F93C801029641E050E003
:108860004C0F5D1F840F951F9F938F930E94CC8B9D
:10887000080F191FC8010E949C3D0FB6F894DEBF77
:108880000FBECDBF892B09F0D8C920E030E04A2DBA
:10889000427050E060E070E080E090E0A0E00E9474
:1088A000048789F182E00E94DF0920916D023091F6
:1088B0006E0240916F02509170020E94D4839F9388
:1088C0008F937F936F9382E097E09F938F931F9294
:1088D00087E78F93C801029621E030E02C0F3D1FFF
:1088E000820F931F9F938F930E94CC8B080F191FA9
:1088F000C8010E949C3D0FB6F894DEBF0FBECDBFED
:10890000892B09F09AC920E030E0C657DF4F488133
:10891000CA58D04050E060E070E080E090E0A0E015
:108920000E94048741F183E00E94DF099F938F93A7
:108930007F936F938FE097E09F938F931F9287E7CA
:108940008F93C8010296E1E0F0E0EC0FFD1F8E0F5F
:108950009F1F9F938F930E94CC8B080F191F8C9899
:10896000C8010E949C3D0FB6F894DEBF0FBECDBF7C
:10897000892B09F062C920E030E04A2D487050E0B0
:1089800060E070E080E090E0A0E00E94048771F178
:1089900080917D1F87FF2AC021E042E161E080EDE8
:1089A0000E94685A9F938F937F936F938CE197E017
:1089B0009F938F931F9287E78F93C801029641E0A0
:1089C00050E04C0F5D1F840F951F9F938F930E9463
:1089D000CC8B080F191FC8010E949C3D0FB6F8945C
:1089E000DEBF0FBECDBF892B09F027C920E030E0E4
:1089F0004A2D407150E060E070E080E090E0A0E03F
:108A00000E94048771F180917D1F87FF2AC021E0B9
:108A100042E162E080ED0E94685A9F938F937F93BA
:108A20006F938AE297E09F938F931F9287E78F93CC
:108A3000C801029621E030E02C0F3D1F820F931FEA
:108A40009F938F930E94CC8B080F191FC8010E941F
:108A50009C3D0FB6F894DEBF0FBECDBF892B09F049
:108A6000ECC820E030E04A2D407250E060E070E059
:108A700080E090E0A0E00E94048771F180917D1F6A
:108A800087FF2AC021E042E163E080ED0E94685A3E
:108A90009F938F937F936F9388E397E09F938F9338
:108AA0001F9287E78F93C8010296E1E0F0E0EC0F98
:108AB000FD1F8E0F9F1F9F938F930E94CC8B080FDB
:108AC000191FC8010E949C3D0FB6F894DEBF0FBE6F
:108AD000CDBF892B09F0B1C820E030E04A2D4074A9
:108AE00050E060E070E080E090E0A0E00E94048749
:108AF00071F180917D1F87FF2AC021E042E164E08F
:108B000080ED0E94685A9F938F937F936F9386E4C2
:108B100097E09F938F931F9287E78F93C8010296E8
:108B200041E050E04C0F5D1F840F951F9F938F9382
:108B30000E94CC8B080F191FC8010E949C3D0FB6E4
:108B4000F894DEBF0FBECDBF892B09F076C8FA2D91
:108B5000F078EF2E20E030E04F2F50E060E070E042
:108B600080E090E0A0E00E94048749F080917D1FA2
:108B700082FF05C046E061E083E00E94E9122B2DF0
:108B80002170F22E20E030E040E05F2D60E070E0E8
:108B900080E090E0A0E00E94048751F080917D1F6A
:108BA00082FF06C021E046E061E083E00E94E91216
:108BB00020E030E04E2D50E060E070E080E090E09A
:108BC000A0E00E94048789F180917D1F82FF2DC063
:108BD00080916B1B8F9380916A1B8F938091691B8F
:108BE0008F938091681B8F9384E597E09F938F9379
:108BF0001F9287E78F93C801029641E050E04C0F27
:108C00005D1F840F951F9F938F930E94CC8B080F3D
:108C1000191FC8010E949C3D0FB6F894DEBF0FBE1D
:108C2000CDBF892B11F00C941D3E20E030E040E0D8
:108C30005F2D60E070E080E090E0A0E00E9404879B
:108C400089F180917D1F82FF2DC080916F1B8F93D2
:108C500080916E1B8F9380916D1B8F9380916C1B05
:108C60008F938CE597E09F938F931F9287E78F9365
:108C7000C801029621E030E02C0F3D1F820F931FA8
:108C80009F938F930E94CC8B080F191FC8010E94DD
:108C90009C3D0FB6F894DEBF0FBECDBF892B11F0FF
:108CA0000C941D3E20E030E040E05B2D527060E00F
:108CB00070E080E090E0A0E00E94048779F180916C
:108CC0007D1F90917E1F90FF29C080E090E00E9460
:108CD000801D9F938F937F936F9387E697E09F9379
:108CE0008F931F9287E78F93C8010296E1E0F0E02F
:108CF000EC0FFD1F8E0F9F1F9F938F930E94CC8BB5
:108D0000080F191FC8010E949C3D0FB6F894DEBFE2
:108D10000FBECDBF892B11F00C941D3E20E030E03A
:108D200040E05B2D547060E070E080E090E0A0E0F7
:108D30000E94048779F180917D1F90917E1F90FFA2
:108D400029C081E090E00E94801D9F938F937F93C4
:108D50006F9387E797E09F938F931F9287E78F9397
:108D6000C801029641E050E04C0F5D1F840F951F33
:108D70009F938F930E94CC8B080F191FC8010E94EC
:108D80009C3D0FB6F894DEBF0FBECDBF892B11F00E
:108D90000C941D3E20E030E040E05B2D507160E01F
:108DA00070E080E090E0A0E00E940487D9F180911B
:108DB0007D1F90917E1F90FF35C081E090E00E9462
:108DC000801D6B017C0180E090E00E94801D9B0172
:108DD000AC01C701B6010E94E61B9F938F937F935E
:108DE0006F9388E897E09F938F931F9287E78F9305
:108DF000C801029621E030E02C0F3D1F820F931F27
:108E00009F938F930E94CC8B080F191FC8010E945B
:108E10009C3D0FB6F894DEBF0FBECDBF892B11F07D
:108E20000C941D3E20E030E040E05B2D507260E08D
:108E300070E080E090E0A0E00E940487D9F180918A
:108E40007D1F90917E1F90FF35C081E090E00E94D1
:108E5000801D6B017C0180E090E00E94801D9B01E1
:108E6000AC01C701B6010E94471C9F938F937F936B
:108E70006F9383E997E09F938F931F9287E78F9378
:108E8000C8010296E1E0F0E0EC0FFD1F8E0F9F1F7E
:108E90009F938F930E94CC8B080F191FC8010E94CB
:108EA0009C3D0FB6F894DEBF0FBECDBF892B11F0ED
:108EB0000C941D3E20E030E040E05B2D507460E0FB
:108EC00070E080E090E0A0E00E940487D9F18091FA
:108ED0007D1F90917E1F90FF35C081E090E00E9441
:108EE000801D6B017C0180E090E00E94801D9B0151
:108EF000AC01C701B6010E94A81C9F938F937F937A
:108F00006F9381EA97E09F938F931F9287E78F93E8
:108F1000C801029641E050E04C0F5D1F840F951F81
:108F20009F938F930E94CC8B080F191FC8010E943A
:108F30009C3D0FB6F894DEBF0FBECDBF892B11F05C
:108F40000C941D3E20E030E040E05B2D587060E066
:108F500070E080E090E0A0E00E94048769F18091D9
:108F60007D1F90917E1F91FF27C00E9433179F9312
:108F70008F937F936F9384EB97E09F938F931F92D0
:108F800087E78F93C801029621E030E02C0F3D1F48
:108F9000820F931F9F938F930E94CC8B080F191FF2
:108FA000C8010E949C3D0FB6F894DEBF0FBECDBF36
:108FB000892B11F00C941D3E20E030E040E0CD56AE
:108FC000DF4F5881C359D04060E070E080E090E00E
:108FD000A0E00E94048771F1F10186811F928F93B6
:108FE00085811F928F9383811F928F9382811F921D
:108FF0008F9385EC97E09F938F931F9287E78F93D2
:10900000C801029621E030E02C0F3D1F820F931F14
:109010009F938F930E94CC8B080F191FC8010E9449
:109020009C3D0FB6F894DEBF0FBECDBF892B11F06B
:109030000C941D3E779A8091490990914A0992FDBE
:10904000749A9401A501C257DF4F6881CE58D04071
:10905000C157DF4F7881CF58D040C057DF4F88814C
:10906000C059D040CF56DF4F9881C159D040A0E0C1
:10907000FE0133967F010E94048751F180914909D6
:1090800090914A0982FD08C080914A0280FD04C087
:1090900081FF1EC01D9B1CC0FF92EF928CED97E0DC
:1090A0009F938F930E94698B80916C020F900F9019
:1090B0000F900F90882361F01F928F938EE19EE0B6
:1090C0009F938F930E947B8B0F900F900F900F9028
:1090D0008091480280618983809169098A83F701C0
:1090E000E00FF11F10828091490990914A0998017F
:1090F0002D5F3F4F790180FF0CC0FF922F9383EECD
:1091000097E09F938F930E94698B0F900F900F9021
:109110000F90B701CE0101960E94AF5480914A0290
:1091200082FF0AC023EE33E2A701BE016F5F7F4FCB
:109130008AE592E00E9435598091490990914A0947
:1091400082FD73980E94CA6085E799E00E94824B75
:1091500080914A0290914B0290FD02C00C944F3EC8
:109160000F5F1F4FE0905002F09051020E94C861C3
:10917000D82E109251021092500289E190E00E9484
:10918000E0610C94223E81E699E00E94E34F892B36
:1091900011F40C94803E0E94826080914A0287FD07
:1091A00002C00C941D3E2B9A0C941D3ECB56DF4FF3
:1091B0000FB6F894DEBF0FBECDBFDF91CF911F91E8
:1091C0000F91FF90EF90DF90CF90BF90AF909F9066
:1091D0008F907F906F905F904F903F902F90089569
:1091E0000C94A94B4F925F926F927F928F929F92B5
:1091F000AF92BF92CF92DF92EF92FF920F931F93A5
:10920000CF93DF93CDB7DEB760970FB6F894DEBF8C
:109210000FBECDBF6B010E94C861FC01EE0FFF1FA6
:10922000EE7FF170EF55F54E80819181019691832B
:1092300080838091490990914A0981FD74988090BA
:109240004A0290904B020E9403547C01FC018081F1
:10925000982F92959F70913099F48F7051F480916E
:10926000AD1A9091AE1A01969093AE1A8093AD1AF2
:1092700008C1B60188E098E20E941F4B892B51F08B
:109280008091AB1A9091AC1A01969093AC1A80938E
:10929000AB1AF7C0C40184E0989F812D992711244F
:1092A000F82FF1708F2E80E899E00E942A4E8C01F1
:1092B000009709F448C0B601C80102960E941F4BEE
:1092C000892BE9F1980149E159E060E074E6C801B1
:1092D0000F960E94AA50F7019181F801848198139A
:1092E00021C082858F5F82878091A91A9091AA1AE6
:1092F00001969093AA1A8093A91A84E00E9420559F
:10930000F801208530E02817390708F074C184E09F
:109310000E942055F8018087F70180818F70F80145
:109320008187AFC0F801128684E00E942055F801C1
:109330008087F70180818F70F80181875DC1C80146
:109340000E94D24EB4CF84E092E00E94BF4D8C01C7
:10935000009709F496C0B601C80102960E94164B08
:10936000F70181818150F801848380E091E0A0E0E1
:10937000B0E083879487A587B687128684E00E9431
:109380002055F8018087F70180818F70F80181876F
:10939000B80180E899E00E948A4E980149E159E0BD
:1093A00060E074E6C8010F960E94AA509924939435
:1093B000F7018181F8018483F70180818F70F801C2
:1093C000878384E00E942055F801858383E00E9412
:1093D00020555C01F801868387818F3009F0912C3C
:1093E000F7014180F8018481481A512C612C712CBD
:1093F00046E0440C551C661C771C4A95D1F7238522
:10940000348545855685A0ECB0E00E94B284BB2728
:10941000A92F982F872F480E591E6A1E7B1E438640
:109420005486658676868091490990914A0981FD26
:1094300032C080914A0280FD2EC081FD2AC0992051
:1094400001F182E08093982381E080939923109228
:109450009A2310929B2380E880939C2310929D2353
:1094600010929E2310929F231092A0231093A22368
:109470000093A12348E953E262E18AE292E00E946C
:109480003D4D8091490990914A0981FFB7C0749A76
:10949000B5C01D9BD4CFA4E6B0E0A30192010E9409
:1094A000B284672F782F892F992724E630E040E097
:1094B00050E00E94FD847F936F93452C562C672CBF
:1094C00077245F924F92BB24BF92AF92F8018581BF
:1094D0001F928F93F70180818F701F928F938181EC
:1094E0001F928F93F60181811F928F9380811F922B
:1094F0008F93C70102969F938F9384EF97E09F937A
:109500008F930E94698B80916C020FB6F894DEBF36
:109510000FBECDBF882361F01F928F938BE19EE039
:109520009F938F930E947B8B0F900F900F900F90C3
:1095300080914A0290914B0296FF2DC0882059F1EC
:10954000F7012081322F3F70832F90E00297D4F0F3
:109550008FEF830F207F822B808385E799E00E9425
:10956000F0488091A71A9091A81A01969093A81A92
:109570008093A71A8091490990914A0996FF0BC0E0
:10958000739809C08091AD1A9091AE1A019690938C
:10959000AE1A8093AD1A80917D1F86FF50CF0E9436
:1095A000B759C70105960E948359F70181811F921F
:1095B0008F93F80186811F928F9385811F928F93DD
:1095C00088E398E09F938F931F9280E18F939E0191
:1095D0002F5F3F4F7901FF922F930E94CC8B82E047
:1095E0000E949D59C7010E9483590FB6F894DEBFAF
:1095F0000FBECDBF24CF812C912CDACE60960FB652
:10960000F894DEBF0FBECDBFDF91CF911F910F91B8
:10961000FF90EF90DF90CF90BF90AF909F908F9092
:109620007F906F905F904F9008950895FB01208187
:10963000FC012083FB012181FC0121830895FC01B1
:109640009081DB018C91981309C081E090E0318119
:1096500011962C91321721F080E0089580E090E07F
:109660000895BC0188E098E20C94164BDC01199631
:10967000ED91FC911A970280F381E02D309709F06B
:10968000099408950F931F93CF93DF9300D0CDB724
:10969000DEB78C0188E10E943355BC01CE010196F2
:1096A0000E94164BD8011996ED91FC911A970190E2
:1096B000F081E02DBE016F5F7F4FC80109950F90CB
:1096C0000F90DF91CF911F910F910895EF92FF922C
:1096D0000F931F93CF93DF93EC018B017A0143EF3C
:1096E00052E00E948F4BFA86E98667EF72E0C8016C
:1096F000DF91CF911F910F91FF90EF900C94E84B69
:109700000C94A74BCF93DF93EC0168E078E288E1FB
:109710000E942955CE01DF91CF910C94A94BEF9275
:10972000FF920F931F93CF93DF93EC018B017A018C
:109730000E94C44BF886EF826BEF72E0C801DF91A4
:10974000CF911F910F91FF90EF900C94E84B0C94E8
:10975000CC4B0C943566DC011796ED91FC91189773
:109760000190F081E02D0994DC011796ED91FC91B8
:1097700018970280F381E02D309709F0099408953D
:1097800084E891E10C94264EFC0173836283BC0152
:1097900084E891E10C948A4EBC0184E891E10C9438
:1097A0006F4ECF93DF93EC0184E891E10E942A4E43
:1097B000009749F0FC01228133812C173D0729F0E5
:1097C0000E94D24EF5CF80E090E0DF91CF910895D6
:1097D0000F931F93CF93DF938B010E94D14BEC012A
:1097E000009731F01D830C83C8010E9466688E8348
:1097F000DF91CF911F910F9108951F93CF93DF9326
:10980000EC01162FEC81FD813097D1F090938711F8
:109810008093861182E08887CE0106960995992764
:1098200087FD90950297029710F0133839F4BE0126
:10983000CE01DF91CF911F910C942A4C81E0888753
:10984000DF91CF911F910895FC01208520FD0C949C
:10985000FD4B0895CF92DF92EF92FF920F931F93EB
:10986000CF93DF93EC016B01E0908611F0908711AC
:109870000091881110918911F801EC17FD0739F05A
:10988000309709F44AC00190F081E02DF6CF20977F
:1098900009F443C08885882309F11886011511054C
:1098A00061F0C017D10729F0AE0167E8C8010E9436
:1098B000244CF80100811181F1CFEC81FD813097BA
:1098C00069F0CC15DD0551F0D0938711C093861156
:1098D00040E050E063E8CE0106960995E0918811DA
:1098E000F0918911CE17DF0769F4888199819093EF
:1098F0008911809388110DC0808191818C179D07FB
:1099000021F0FC013097C1F704C0888199819183CF
:109910008083F0928711E0928611DF91CF911F91A1
:109920000F91FF90EF90DF90CF9008951F93CF930A
:10993000DF9310929211C0918811D091891111E09A
:10994000209779F08985882341F01887198640E0AF
:1099500050E062E8CE010E94FD4B0990D881C02DF5
:10996000EFCFDF91CF911F9108958091351291E053
:10997000980F909335120895609186117091871118
:109980000C942A4C8AE8809335121092331210926C
:10999000341210928911109288111092871110922E
:1099A000861108958091921181110E94964C7091B8
:1099B0003412772309F451C0E09133122E2F30E096
:1099C00085E0E89FF0011124ED56FE4E6081609322
:1099D0009111418152815093901140938F11838155
:1099E000948190938E1180938D112F5F3F4F2F7133
:1099F000332720933312715070933412009731F54E
:109A0000809188119091891190938C1180938B1182
:109A100080918B1190918C11892BF9F0809192118A
:109A200081110E94964C40918F115091901160913C
:109A3000911180918B1190918C110E94244CE09196
:109A40008B11F0918C1180819181DECF613819F4F6
:109A500021E0FC0120870E94244C809192112091EA
:109A6000341290E0820F911D0895809192112091FF
:109A7000341290E0820F911D08952091341220320B
:109A8000B9F0E0913312E20FEF71E0938A1135E003
:109A9000E39FF0011124ED56FE4E60835283418313
:109AA000948383832F5F2093341280E090E00895A5
:109AB00081E090E00895CF93DF93C0918611D0911B
:109AC00087110E94244CD0938711C0938611DF9197
:109AD000CF910895AB013091881120918911E32F26
:109AE000F22FE817F907B1F0309721F00190F081DB
:109AF000E02DF7CF009771F0FC0130832183909324
:109B000089118093881121E020871782168261E8ED
:109B10000C945B4D0895009749F0FC01208521507D
:109B2000223020F421E0218720939211089521E032
:109B300030E0FC018085811102C020E030E0C901E5
:109B40000895CF93DF93EC014A815B8160E070E080
:109B50008C819D810E94D78A2A813B81888199814D
:109B6000289FA001299F500D389F500D112460E0BF
:109B700070E08E819F81DF91CF910C94D78AFC0198
:109B80008281938120E030E028173907D1F0A48149
:109B9000B581A20FB31F4C91411110C081E08C938D
:109BA00080819181289FA001299F500D389F500DE1
:109BB000112486819781840F951F08952F5F3F4F51
:109BC000E3CF80E090E00895FC0126813781428157
:109BD000538180E090E084179507C9F02617370776
:109BE00081F4A481B581A80FB91F2C91121614F429
:109BF00021502C930480F581E02DE80FF91F80811E
:109C00000895A081B1812A0F3B1F0196E4CF8FEF09
:109C10000895FC018681978168177907A0F0A081DB
:109C2000B18142815381A49F9001A59F300DB49FC3
:109C3000300D1124280F391F81E090E0621773075F
:109C400020F080E0089580E090E00895FC0111820A
:109C500010820895FC01808191810895FB0120818B
:109C60003181FC01318320830895DC01ED91FC9169
:109C7000309731F080819181009729F0FC01FACF73
:109C800080E090E00895CF010895DC01ED91FC9112
:109C900011973097A9F020813181232B21F41D9257
:109CA0001C92CF010895A081B1818D919C91119753
:109CB000892B11F0FD01F7CF11821082CD0108959B
:109CC00080E090E00895DC01ED91FC9111973097D0
:109CD00021F0208131812D933C93CF010895DC0147
:109CE000ED91FC913097A9F0A0E0B0E020813181A6
:109CF000E617F70741F4109709F4DC012D933C9324
:109D00001182108208952115310519F0DF01F90142
:109D1000EDCF08950F931F93CF93DF938C01EB0149
:109D20000E946F4E19821882C8010E94354E00971A
:109D300011F4F80101C0FC01D183C083DF91CF9100
:109D40001F910F9108950F931F93CF93DF93EC0111
:109D50008B010E946F4E88819981F80191838083E5
:109D600019830883DF91CF911F910F910895DC0132
:109D7000ED91FC9180E090E0309729F00196019000
:109D8000F081E02DF9CF0895FB01309719F4BA0165
:109D90000C94A34E80819181DA018D939C93518321
:109DA00040830895009721F0FC01808191810895FE
:109DB00080E090E008958091381290913912892BBB
:109DC00029F4109237121092361208950E94CF5D36
:109DD000E0913812F0913912228133814081518112
:109DE000240F351F281B390B0480F581E02D309797
:109DF00069F04281538160817181460F571F481B72
:109E0000590B4217530780F79A01EECF280F391FDD
:109E1000309337122093361208958BE792E00C941A
:109E20008B4DEF92FF920F931F93CF93DF938C0193
:109E3000FC0180819181009799F08A359105D9F0D4
:109E4000F8011182108283E068C0868197818417AF
:109E5000950709F049C00480F581E02D3097A9F7F6
:109E600010923912109238128AE590E0F80191832D
:109E7000808381E052C0673891F16238A9F7C091C0
:109E80003812D0913912E12CF12C209769F3CE01D0
:109E90000E94376C892BF1F0AE0168E88E819F81BA
:109EA0000E943D4D892BA1F41F821E828C819D81D1
:109EB000E114F10421F0F7019583848304C09093A9
:109EC0003912809338121D821C820E94DB4ED7CF3C
:109ED0000E940D4F7E010C80DD81C02DD6CFE09118
:109EE0003812F0913912BACFF0933912E093381248
:109EF000A481B581109709F4B7CF16968D919C91E6
:109F000017978417950711F0FD01F2CF14968D91E4
:109F10009C91159795838483EBCFDF91CF911F910F
:109F20000F91FF90EF900895CF93DF93EC010E9483
:109F30000D4F8E819F813091381220913912892BDB
:109F400059F0E32FF22F309739F0EC17FD0781F02D
:109F50000480F581E02DF7CF8091861190918711D3
:109F60009F838E833C832D83D0933912C093381204
:109F7000DF91CF910C94DB4ECF93DF93EC010E94E5
:109F8000176CCE01DF91CF910C94944FCF93DF9358
:109F9000EC010E94236CCE01DF91CF910C94944F81
:109FA000CF93DF93EC010E942D6CCE01DF91CF9116
:109FB0000C94944FFC0120813181260F371F31838F
:109FC00020830C94DB4E21E030E0FC0186819781F8
:109FD000892B11F020E030E0C9010895FC012281B5
:109FE000338180819181820F931F0895FC018081CC
:109FF0009181089581E090E02091381230913912DA
:10A00000232B11F480E090E0089580913812909114
:10A010003912892B29F080913612909137120895C8
:10A0200080E090E00895CF93DF93EC01E091381247
:10A03000F09139128E179F0769F48C819D8190935E
:10A040003912809338120DC0848195818C179D0739
:10A0500021F0FC013097C1F706C08C819D8195836A
:10A0600084830E94DB4E1D821C821F821E82DF9130
:10A07000CF910895EF92FF920F931F93CF93DF93A9
:10A080008C017A01FC0180819181009741F08B3431
:10A09000910501F1F8011182108283E048C08BE341
:10A0A00092E10E942A4EEC01209751F06C817D8153
:10A0B000CE0102960E94BC4F0990D881C02DF4CFEA
:10A0C00081E080933A128BE490E0F80191838083E1
:10A0D00081E02DC06838E1F78BE392E10E942A4EBF
:10A0E000EC01209781F3CE010296E816F906D9F427
:10A0F000BE018BE392E10E946F4EE0908611F090DA
:10A1000087118A859B859093871180938611EC85B2
:10A11000FD85309719F08E859F850995F0928711FE
:10A12000E0928611D0CF0990D881C02DDACFDF918F
:10A13000CF911F910F91FF90EF90089510923A12D6
:10A140008BE392E10E94264E60E070E085E892E0A9
:10A150000C946A4D0F931F93CF93DF93EC01009102
:10A160008611109187111B870A875D874C873F876F
:10A170002E8780913A12882379F085E892E09093B7
:10A18000871180938611CE0102960E94BC4F1093D6
:10A1900087110093861102C07D836C83BE018BE31F
:10A1A00092E10E946F4EBE018BE392E1DF91CF916D
:10A1B0001F910F910C948A4E0F931F93CF93DF93AF
:10A1C000EC0180913A12882391F000918611109150
:10A1D000871185E892E09093871180938611CE01D4
:10A1E00002960E94C64F1093871100938611BE01FC
:10A1F0008BE392E10E946F4EBE018BE392E1DF910F
:10A20000CF911F910F910C948A4E0F931F93CF9370
:10A21000DF93EC0180913A12882391F0009186112E
:10A220001091871185E892E09093871180938611B1
:10A23000CE0102960E94D04F109387110093861191
:10A24000BE018BE392E10E946F4EBE018BE392E16F
:10A25000DF91CF911F910F910C948A4ECF93DF9392
:10A26000EC0180913A12882329F0CE0102960E94D7
:10A27000135004C01F821E8219861886BE018BE30C
:10A2800092E1DF91CF910C946F4ECF93DF93EC016D
:10A2900080913A12882331F0CE010296DF91CF915E
:10A2A0000C94E34F8BE392E10E942A4E009739F021
:10A2B0008C179D0739F0FC0180819181F7CF81E0F7
:10A2C00090E002C080E090E0DF91CF9108952F925E
:10A2D0003F924F925F926F927F928F929F92AF9236
:10A2E000BF92CF92DF92EF92FF920F931F93CF9383
:10A2F000DF93CDB7DEB7E8970FB6F894DEBF0FBE99
:10A30000CDBFEFE3FAE22081318142815381EBE35B
:10A31000FAE25080418032802380E7E3FAE28081D4
:10A32000898391819A83A281AB836380E3E3FAE21C
:10A33000B081BC8381818D8392819E83A381AF8311
:10A34000EFE2FAE2B081B8878181898792819A87AA
:10A35000A381AB87EBE2FAE2B081BC8781818D8774
:10A3600092819E87A381AF87E7E2FAE2B081B88B42
:10A370008181898B92819A8BA381AB8BE3E2FAE294
:10A38000B081BC8B81818D8B92819E8BA381AF8BA1
:10A39000EFE1FAE2B081B88F8181898F92819A8F43
:10A3A000A381AB8FEBE1FAE2B081BC8F81818D8F0D
:10A3B00092819E8FA381AF8FE7E1FAE2B081B8A3CB
:10A3C000818189A392819AA3A381ABA3E3E1FAE2FD
:10A3D000B081BCA381818DA392819EA3A381AFA3F1
:10A3E000EFE0FAE2B081B8A7818189A792819AA7AC
:10A3F000A381ABA7EBE0FAE2B081BCA781818DA776
:10A4000092819EA7A381AFA7E7E0FAE2B081B8AB43
:10A41000818189AB92819AAB7380E3E0FAE2B080EC
:10A42000A18092808380EFEFF9E2F080E180D2801A
:10A43000C380EBEFF9E2A081AFABB181B8AF12817D
:10A4400003812BAB3CAB4DAB5EAB0E94FD5D5EA9C7
:10A450005F934DA94F933CA93F932BA92F932F9224
:10A460003F924F925F926F922B812F932A812F936D
:10A4700029812F932F812F932E812F932D812F931D
:10A480002C812F932B852F932A852F9329852F930A
:10A4900028852F932F852F932E852F932D852F93EE
:10A4A0002C852F932B892F932A892F9329892F93DA
:10A4B00028892F932F892F932E892F932D892F93BE
:10A4C0002C892F932B8D2F932A8D2F93298D2F93AA
:10A4D000288D2F932F8D2F932E8D2F932D8D2F938E
:10A4E0002C8D2F932BA12F932AA12F9329A12F934A
:10A4F00028A12F932FA12F932EA12F932DA12F931E
:10A500002CA12F932BA52F932AA52F9329A52F9309
:10A5100028A52F932FA52F932EA52F932DA52F93ED
:10A520002CA52F937F922AA92F9329A92F9328A98D
:10A530002F938F929F92AF92BF92CF92DF92EF9222
:10A54000FF920F931F9328AD2F932FA92F939F93C3
:10A550008F937F936F93A9E0B8E28C911F928F93B2
:10A56000E8E0F8E280811F928F9386E99EE09F9356
:10A570008F930E947B8BEFE6FAE22081318142814A
:10A580005381EBE6FAE25080418032802380EFE590
:10A59000FAE29080818072806380EBE5FAE280814C
:10A5A000898391819A83A281AB83B381BC83E7E5E0
:10A5B000FAE280818D8391819E83A281AF83B381F2
:10A5C000B887E3E5FAE28081898791819A87A28141
:10A5D000AB87B381BC87EFE4FAE280818D879181FC
:10A5E0009E87A281AF87B381B88BEBE4FAE28081CA
:10A5F000898B91819A8BB280A380E7E4FAE2F080A4
:10A60000E180D280C380E3E4FAE2A081AB8BB18128
:10A61000BC8B128103810FB6F894DEBF0FBECDBF95
:10A620002BAB3CAB4DAB5EAB0E94FD5D5EA95F9377
:10A630004DA94F933CA93F932BA92F932F923F9263
:10A640004F925F926F927F928F929F922C812F9365
:10A650002B812F932A812F9329812F9328852F9344
:10A660002F812F932E812F932D812F932C852F9324
:10A670002B852F932A852F9329852F9328892F9314
:10A680002F852F932E852F932D852F93AF92BF92D9
:10A690002A892F9329892F93CF92DF92EF92FF92ED
:10A6A0000F931F932C892F932B892F939F938F9315
:10A6B0007F936F93A9E0B8E28C911F928F93E8E0AB
:10A6C000F8E280811F928F9387E29EE09F938F93A1
:10A6D0000E947B8B0FB6F894DEBF0FBECDBFE8960D
:10A6E0000FB6F894DEBF0FBECDBFDF91CF911F91A3
:10A6F0000F91FF90EF90DF90CF90BF90AF909F9021
:10A700008F907F906F905F904F903F902F90089523
:10A7100080E38093F1120895CF93DF936091F1125B
:10A7200070E0C0E3D0E0C61BD70B615C7D4EAE018C
:10A730000E94CE8ACE01DF91CF910895CF92DF9211
:10A74000EF92FF920F931F93CF93DF937C01C09002
:10A75000F412D090F5126091F11270E0E601E096EB
:10A76000C61BD70BC138D105D8F400E310E0061B97
:10A77000170B615C7D4EA8010E94CE8A60913D124C
:10A7800070913E128091F2129091F312680F791F2E
:10A79000A601C701800F911F0E94CE8ACE0102C080
:10A7A00080E090E0DF91CF911F910F91FF90EF90AB
:10A7B000DF90CF9008959091F112980F9093F1123D
:10A7C00008954091F4125091F5124817590798F0E6
:10A7D0002091F2123091F312280F391F3093F312A7
:10A7E0002093F212481B590B5093F5124093F41228
:10A7F00081E090E0089580E090E008959093F51254
:10A800008093F41208958091F2129091F31281597D
:10A810009D4E08958091F11290E0815C9D4E0895C7
:10A8200081E090E020913D1230913E122F5632414E
:10A8300011F480E090E008950E941054892B61F09B
:10A8400060913D1270913E124091F4125091F512B8
:10A850008FE692E10C94CE8A2091F2123091F3129D
:10A8600021153105B9F08091F4129091F512C0963E
:10A87000EFE6F2E1AF014F5352414817590734F464
:10A88000DF01A20FB31F4C914193F4CF1092F3124A
:10A890001092F212089580913D1290913E12089507
:10A8A0008091F4129091F51208959091F11280E345
:10A8B000891B089520E38091F112281B8091F412E6
:10A8C0009091F512820F911D08951F93CF93DF93FE
:10A8D000EC011091F112812F90E08C179D076CF024
:10A8E0000E945A548C0F9D1F8138910530F41C1B17
:10A8F0001093F11281E090E002C080E090E0DF91DF
:10A90000CF911F910895CF93DF93E2E1F8E2119286
:10A91000119288E2E234F807D1F7CAE0D8E261EF99
:10A9200072E0CE010E94164B229688E2C231D8070F
:10A93000B1F7DF91CF9108951092F3121092F212B5
:10A940001092F5121092F41280E38093F1128FE6C8
:10A9500092E190933E1280933D120C948354EF92B7
:10A96000FF920F931F93CF93DF9300D0CDB7DEB745
:10A970008C0169837A830E949C546981E62E7A81D6
:10A98000F72E81E8E816F10418F080E8E82EF12CA3
:10A99000A701B80180913D1290913E120E94CE8A8B
:10A9A000F092F512E092F412C7010F900F90DF9130
:10A9B000CF911F910F91FF90EF9008950F931F93E8
:10A9C000CF93DF938C01EB010E949C5410933E12B5
:10A9D00000933D12D093F512C093F412DF91CF9102
:10A9E0001F910F91089520E3E2E1F8E2DC0101906C
:10A9F0000D922A95E1F788E0EAE0F8E2DB010190A8
:10AA00000D928A95E1F7089520E3FC01A2E1B8E2F6
:10AA100001900D922A95E1F788E0FB01AAE0B8E2E7
:10AA200001900D928A95E1F70895E82FF0E0EE0F7E
:10AA3000FF1FEE5EF74D7183608381E090E0089523
:10AA4000E82FF0E0EE0FFF1FEE5EF74D8081918161
:10AA5000089590E0880F991F8652984D0E94164BDA
:10AA600081E090E0089590E0880F991F8652984DFC
:10AA700008958115910511F00197F1F70895E0917E
:10AA80004528F09146289081809144288923089593
:10AA9000E0914228F0914328808190914428892BAD
:10AAA0008083E0914728F091482880819091442844
:10AAB000892B80830895E0914228F091432890816A
:10AAC00080914428809589238083E0914728F091E4
:10AAD0004828908180914428809589238083089517
:10AAE0001F93CF93DF93E0914228F0914328908108
:10AAF00080914428809589238083E0914728F091B4
:10AB00004828808190914428892B80838FEB93E0A3
:10AB10000E9439551FB7F894E0914728F0914828D2
:10AB200090818091442880958923808383E890E0F8
:10AB30000E943955E0914528F0914628D081C09176
:10AB400044281FBF78948BE393E00E943955E0912D
:10AB50004528F0914628908180914428982319F047
:10AB60008D2F8C2301C081E0DF91CF911F9108953B
:10AB70005093482840934728709343286093422875
:10AB8000909346288093452881E001C0880F2A953C
:10AB9000EAF7809344280C947055CF93DF93C82F25
:10ABA000DFB7F894E0914728F09148288081909190
:10ABB0004428892B808383E090E00E943955CC2380
:10ABC00051F0E0914728F0914828808190914428E5
:10ABD00090959823908387E190E00E943955E09109
:10ABE0004528F0914628808190914428892309F4D2
:10ABF000C0E089E590E00E943955E0914728F09146
:10AC00004828808190914428909598239083DFBFB5
:10AC10008BE390E00E9439558C2FDF91CF910895FE
:10AC2000CF93DF93C82FD8E08C2F81700E94CD5531
:10AC3000C6958111C068D150B9F78C2FDF91CF91A3
:10AC400008958FEF0C941056DF92EF92FF920F93BE
:10AC50001F93CF93DF93E82EEB010E947055811173
:10AC60002FC080EF0E941056F12C10E488EFD82EF0
:10AC7000D10E81E00E94CD55082F81E00E94CD5574
:10AC8000882319F0002361F01DC0011109C01E15B1
:10AC900028F0888180FF04C0E11611F0F12E01E058
:10ACA000802F0E94CD5598819695011190689883C8
:10ACB00011501D11DECF21961111D8CF8F2D03C059
:10ACC0008FEF01C08EEFDF91CF911F910F91FF9019
:10ACD000EF90DF900895FF920F931F93CF93DF9330
:10ACE000F82EEB010E947055209769F085E50E94CF
:10ACF00010568E01085F1F4F89910E941056C01791
:10AD0000D107D1F703C08CEC0E9410568F2DDF9134
:10AD1000CF911F910F91FF900C9410560F931F939A
:10AD2000CF93DF93DB01EC9111969C911197F0E0AA
:10AD3000F92B803181F4BF016E7FE3E0660F771F4E
:10AD4000EA95E1F716969C911697ECE0F0E0E91B86
:10AD5000F109E60FF71FF7FF07C091E0EA019883BA
:10AD6000F195E195F10902C0EA011882883279F47F
:10AD700014968C91982F9076903649F086FF02C0F9
:10AD8000EE7F05C085FF02C0EC7F01C0E87FCF01E8
:10AD900044E0969587954A95E1F7D9018C93EF7039
:10ADA000E801E88380E0DF91CF911F910F91089532
:10ADB0000F931F93CF93DF93EC018B01B801888130
:10ADC0000E942456888381508D3F30F4F8018081A1
:10ADD000883211F0803191F7DF91CF911F910F915F
:10ADE0000895CF93DF93EC010E947055BE0184EB70
:10ADF0000E946B5681E00E94CD55C82F0E9470556D
:10AE000081E0C11101C080E0DF91CF9108951F93CF
:10AE1000CF93DF9300D0CDB7DEB7182F69837A8345
:10AE20000E9470550E943F5569817A81882341F0C4
:10AE300084E40E946B56113029F00E94485502C0EC
:10AE400082E001C080E00F900F90DF91CF911F91C1
:10AE500008954F925F926F927F928F929F92AF92DE
:10AE6000BF92CF92DF92EF92FF920F931F93CF93F7
:10AE7000DF93CDB7DEB729970FB6F894DEBF0FBECC
:10AE8000CDBF6C015B014A0189010E947055B6017A
:10AE90008EEB0E946B56CE0101967C013E019AE03A
:10AEA000690E711C27010E942156F70181937F01D1
:10AEB000E615F705C1F769E070E0C2010E94A870CD
:10AEC000811109C09401A501B201F60180810E949F
:10AED0008E5680E001C083E029960FB6F894DEBF5D
:10AEE0000FBECDBFDF91CF911F910F91FF90EF90DB
:10AEF000DF90CF90BF90AF909F908F907F906F909A
:10AF00005F904F9008955F926F927F928F929F9281
:10AF1000AF92BF92CF92DF92EF92FF920F931F9367
:10AF2000CF93DF93CDB7DEB729970FB6F894DEBF86
:10AF30000FBECDBF582E6B015A01890160E070E051
:10AF40008EEB0E946B56CE0101967C014E019AE079
:10AF5000890E911C37010E942156F70181937F01D0
:10AF6000E815F905C1F769E070E0C3010E94A87017
:10AF7000811108C09501A601B301852D0E948E564E
:10AF800080E001C083E029960FB6F894DEBF0FBEC3
:10AF9000CDBFDF91CF911F910F91FF90EF90DF9088
:10AFA000CF90BF90AF909F908F907F906F905F9069
:10AFB00008950F931F93CF93DF93CDB7DEB72897F4
:10AFC0000FB6F894DEBF0FBECDBF182F062F98E046
:10AFD000EDEFF2E0DE01119601900D929A95E1F706
:10AFE000242F332727FD309541E752E0249FC001ED
:10AFF000259F900D349F900D112464E670E00E940F
:10B00000E984CB0144E6049F800D911D1124FE01CB
:10B010003196AE01475F5F4F619170E026173707A9
:10B0200011F4019603C0E417F507B1F7112319F0E5
:10B0300091958195910928960FB6F894DEBF0FBEC1
:10B04000CDBFDF91CF911F910F910895EF92FF92A5
:10B050000F931F93CF93DF93CDB7DEB72B970FB628
:10B06000F894DEBF0FBECDBFF82EE92E682F792FE2
:10B0700088E08F0D0E940757882319F084E391E23E
:10B0800043C066E471E48FE090E00E9491588E0125
:10B09000075F1F4F9801AE01465F5F4FBE01655FBE
:10B0A0007F4F8F2D9E2D0E9429578111E7CF88E079
:10B0B000EDEFF2E0DE01119601900D928A95E1F735
:10B0C000498521E732E0429FC001439F900D112442
:10B0D00064E670E00E94E9848A8594E6899F600DA9
:10B0E000711D1124FE0131968191481303C06F5FD9
:10B0F0007F4F03C0E017F107B9F78B85882319F05C
:10B10000719561957109CB012B960FB6F894DEBF4E
:10B110000FBECDBFDF91CF911F910F91FF90EF90A8
:10B120000895DC01CB0181159105A105B10529F038
:10B1300081509040A040B040D9F708951092B900D6
:10B1400080E28093B800089594EA9093BC0040EAAE
:10B1500056E861E070E09091BC0097FD0BC0415053
:10B16000510961097109411551056105710599F789
:10B1700081E008959091B900987F983011F0903156
:10B18000B9F78093BB0084E88093BC0080EA96E81E
:10B19000A1E0B0E02091BC0027FD08C00197A10903
:10B1A000B1090097A105B105A9F7E2CF8091B900D7
:10B1B000887F883111F08034D9F680E0089524EA40
:10B1C00034E844E92093BC009091BC0097FFFCCF89
:10B1D0009091B900987F983011F0903199F7809351
:10B1E000BB003093BC009091BC0097FFFCCF9091C6
:10B1F000B900987F903211F0983539F44093BC0033
:10B200009091BC0094FDFCCFDDCF08950C94A45820
:10B2100084E98093BC008091BC0084FDFCCF08953C
:10B220008093BB0084E88093BC008091BC0087FFC2
:10B23000FCCF9091B900987F81E0983209F480E0CA
:10B24000089584EC8093BC008091BC0087FFFCCF04
:10B250008091BB00089584E88093BC008091BC007D
:10B2600087FFFCCF8091BB000895E0E1DC01FD91F8
:10B27000CD01F0933F01E150C9F780913C018F7DF2
:10B2800080933C0180913C01877F80933C01FB01CE
:10B2900080E1919190933E018150D9F780913C01DA
:10B2A000806880933C0180913D0180FFFCCF40513C
:10B2B000510980913C01806280933C0180913C0166
:10B2C000877F80933C01141615069CF4FB0180E1F6
:10B2D000919190933E018150D9F780913C01806813
:10B2E00080933C0180913D0180FFFCCF405151098A
:10B2F000EACFF90180E190913E0191938150D9F715
:10B3000081E090E008950F931F93CF93DF93EC01BA
:10B310008CE70E94DF588CE70E9410598E01005F75
:10B320001F4F89910E941059C017D107D1F7DF91A3
:10B33000CF911F910F910C940859813019F440E07E
:10B3400050E002C040EC50E060E070E08CE790E03C
:10B350000C941611813019F44EE050E002C048E020
:10B3600050E060E070E08CE790E00C94161141E052
:10B3700050E060E070E08CE790E00E9416116AE611
:10B380007AE080E090E00C94915848E350E060E06F
:10B3900070E08CE790E00E94161149E350E060E015
:10B3A00070E08CE790E00E94161144E150E060E00C
:10B3B00070E08CE790E00E94161148E750E060E0F2
:10B3C00070E08CE790E00E9416114EE550E060E0DE
:10B3D00070E08CE790E00E9416114DE650E060E0CE
:10B3E00070E08CE790E00E9416116CE17AE186E053
:10B3F00090E00E9491584CE050E060E070E08CE7F3
:10B4000090E00E94161141E050E060E070E08CE7AF
:10B4100090E00E94161146E050E060E070E08CE79A
:10B4200090E00E9416116AE67AE080E090E00C94C9
:10B430009158CF93DF93CDB7DEB7A2970FB6F894AC
:10B44000DEBF0FBECDBF81E1E4ECF8E0DE01529635
:10B4500001900D928A95E1F781E1E5EDF8E0DE01DA
:10B46000119601900D928A95E1F70E94C559CE017F
:10B4700042960E94835982E00E949D596AE67AE0D2
:10B4800080E090E00E949158CE0101960E9483597D
:10B4900060E17EEA88E290E00E94915880E00E949C
:10B4A000AA5960E17EEA88E290E00E9491584EE05D
:10B4B00050E060E070E08CE790E00E941611A296E8
:10B4C0000FB6F894DEBF0FBECDBFDF91CF910895C8
:10B4D000CF92DF92EF92FF920F931F93CF93DF9360
:10B4E00000D01F92CDB7DEB7F82E042F122F2130D7
:10B4F00031F0223031F0243031F0283031F090E05A
:10B5000005C091E003C092E001C093E00C3059F017
:10B510000E3011F4946007C0003111F4986003C03C
:10B52000023109F49C60613059F0623011F490628C
:10B5300007C0633011F4906403C0643009F490666E
:10B540009068692F70E023E030E0AE014F5F5F4FFD
:10B550008F2D90E00E942D1169E07AE180E090E06B
:10B560000E9491588F2D8160F82E0E94A4580E944D
:10B57000215989830E9421598A83023119F40E943A
:10B5800021598B830E94215987FDF1CF0E942B59AD
:10B590000E94085969E07AE180E090E00E949158A9
:10B5A0008F2D0E94A4580E94215989830E942159FD
:10B5B0008A83023119F40E942B598B830E942B59E4
:10B5C0000E94085939812A81023149F5832F90E080
:10B5D000A0E0B0E04B817727662731FF0EC030E056
:10B5E000322F2227620F731F811D911D640F711D61
:10B5F000811D911D8C6F9F6F0BC030E0322F222771
:10B60000620F731F811D911D640F711D811D911D9E
:10B610000E94F68120E83FEF4FEF57E420C0632FF0
:10B6200070E0762F6627620F711D882777FD809561
:10B63000982F0E94F6810C3029F420E030EE4FEF75
:10B6400054E40DC00E3029F420E038EF4FEF55E4FC
:10B6500006C0003131F420E03EEF4FEF56E40E9487
:10B6600057812FE632E143E050E40E94D4836B011E
:10B670007C01612F70E080E090E00E94F6819B01E8
:10B68000AC01C701B6010E9457810F900F900F9037
:10B69000DF91CF911F910F91FF90EF90DF90CF90AE
:10B6A0000895E6E4F1E080812081908130818295E7
:10B6B00086958695837022952F70822B832B929589
:10B6C0009F70892B08950F931F93CF93DF9300D022
:10B6D000CDB7DEB746E06CE080E00E94935E89E182
:10B6E0008093C4001092C50082E08093C00080E087
:10B6F0000E941E5F0E94BF5D84B784B784B784B781
:10B7000084B7E9ECF0E322E432E4318320833A9613
:10B710008DB79EB70A97E817F907B8F386EE98E059
:10B720009F938F9383EE9FE09F938F930E947B8BD9
:10B730000E94EB6C0E94C24C60E070E08BE792E0EC
:10B740000E946A4D0E949E50E0910503F09106030D
:10B7500009950E94515B90E00E94276DCE010196F1
:10B760000E94F45C0F900F900F900F90882341F08F
:10B7700083EC9FE09F938F930E947B8B0F900F90A1
:10B78000CE0101960E94314B0E94025D8C010E9405
:10B79000FE5CAE014F5F5F4FB8010E94EA610E94FC
:10B7A0006E5C0E94CB610E94065D0E94156386EB71
:10B7B0009FE09F938F930E947B8B8A811F928F9330
:10B7C00002EB1FE01F930F930E947B8B89811F92D6
:10B7D0008F931F930F930E947B8B80EB9FE09F932F
:10B7E0008F930E947B8B0E942B6DE0914203F0911E
:10B7F00043030995E0913403F09135030995E091F5
:10B800001B03F0911C0309950E941C63182F0E94D2
:10B81000C8611F921F931F928F93809141038F9352
:10B82000809140038F93809133038F9380913203F3
:10B830008F9385E99FE09F938F930E947B8BE0918C
:10B840004C03F0914D030FB6F894DEBF0FBECDBF91
:10B85000309791F00995BC0180E890E00E94D58472
:10B860007F936F9382E89FE09F938F930E947B8BDF
:10B870000F900F900F900F9080E89FE09F938F9311
:10B880000E947B8B60E070E081ED92E00E946A4D47
:10B8900083EE92E00E94FB6B88E79FE09F938F937B
:10B8A0000E947B8B0F900F900F900F900F900F9036
:10B8B000DF91CF911F910F9108957F936F939F9385
:10B8C0008F9382E79FE09F938F930E947B8B0F90D3
:10B8D0000F900F900F900F900F9008951F93CF939C
:10B8E000DF93CDB7DEB7A0970FB6F894DEBF0FBEDB
:10B8F000CDBF85E390E00E94B88C182F282F35EF3C
:10B90000380F303108F0982F9095291709F461C04D
:10B910008EEF9FE09F938F930E947B8BE3E4F0E197
:10B920000F900F90DE01119684918D93319680E1F6
:10B93000EB34F807C9F7F89448E050E061E570E0AF
:10B94000CE0101960E94BE8CE5E3F0E1DE01119686
:10B9500084918D93319680E1E334F807C9F74EE086
:10B9600050E063E470E0CE0101960E94BE8CEBE2F1
:10B97000F0E1DE01119684918D93319680E1E533FB
:10B98000F807C9F74AE050E069E370E0CE0101969C
:10B990000E94BE8C6DEC7BEA83E390E00E94D68C23
:10B9A00060E070E081E390E00E94D68C60E080E38C
:10B9B00090E00E94C88C60E070E087E390E00E9415
:10B9C000D68C1AE16AE175EE85E390E00E94D68C90
:10B9D0007894812FA0960FB6F894DEBF0FBECDBF2E
:10B9E000DF91CF911F910895F89442E050E061E516
:10B9F00070E00E94A08C789480E0089583E390E04A
:10BA00000C94B88C81E390E00C94B88C80E390E0C7
:10BA10000C94B08C40915728509158286091592827
:10BA200070915A2890E0A0E0B0E0480F591F6A1FBB
:10BA30007B1F409357285093582860935928709340
:10BA40005A2840915328509154286091552870915C
:10BA50005628480F591F6A1F7B1F40935328509345
:10BA6000542860935528709356282091F729222353
:10BA7000A1F040914F285091502860915128709129
:10BA80005228480F591F6A1F7B1F40934F2850931D
:10BA90005028609351287093522808951F920F9256
:10BAA0000FB60F9211240BB60F922F933F934F9323
:10BAB0005F936F937F938F939F93AF93BF93EF9316
:10BAC000FF938091F8129091F91201969093F912D8
:10BAD0008093F8128091F7128F5F8093F71280386D
:10BAE000A9F41092F7128091572890915828A091AC
:10BAF0005928B0915A280196A11DB11D809357284D
:10BB000090935828A0935928B0935A288091F729E8
:10BB10008823E1F08091F6128F5F8093F6128038CF
:10BB2000A9F41092F61280914F2890915028A0917C
:10BB30005128B09152280196A11DB11D80934F2824
:10BB400090935028A0935128B09352280E94FA4F06
:10BB5000892B11F00E940D4FFF91EF91BF91AF9192
:10BB60009F918F917F916F915F914F913F912F9115
:10BB70000F900BBE0F900FBE0F901F901895F8946A
:10BB80001092B60016BC83EF87BD82E084BD94E0BE
:10BB900095BD95B395BB80936E0078940895809180
:10BBA000F8129091F9122091F8123091F91282173F
:10BBB0009307A9F70895009751F022E330E00000C1
:10BBC0002150310921153105D1F70197F4CF08959E
:10BBD0000F931F93CF93DF93EC010E94CF5D8C01F5
:10BBE0000E94CF5D801B910B8C179D07C8F3DF91DE
:10BBF000CF911F910F91089508950F931F93609116
:10BC00005728709158288091592890915A2800916E
:10BC10005728109158282091592830915A28601798
:10BC200071078207930759F71F910F9108951F928B
:10BC30000F920FB60F9211241092A7020F900FBE11
:10BC40000F901F9018951F920F920FB60F9211240C
:10BC50000BB60F922F933F934F935F936F937F9306
:10BC60008F939F93AF93BF93EF93FF93E0919D02C8
:10BC7000F0919E028081E091A802F091A902309794
:10BC800009F00995FF91EF91BF91AF919F918F912D
:10BC90007F916F915F914F913F912F910F900BBECC
:10BCA0000F900FBE0F901F9018951F920F920FB616
:10BCB0000F9211241092B4020F900FBE0F901F909C
:10BCC00018951F920F920FB60F9211240BB60F9278
:10BCD0002F933F934F935F936F937F938F939F9394
:10BCE000AF93BF93EF93FF93E091AA02F091AB0261
:10BCF0008081E091B502F091B602309709F0099584
:10BD0000FF91EF91BF91AF919F918F917F916F9133
:10BD10005F914F913F912F910F900BBE0F900FBEEF
:10BD20000F901F9018959DE0899FF0011124E35614
:10BD3000FD4FA281B3811C92A481B5816C93A68131
:10BD4000B78188ED8C93A085B1854C9312861486BB
:10BD5000138608959DE0899FF0011124E356FD4F5D
:10BD600081E08287A081B1816C933A9680818111B4
:10BD7000FDCF08951F93CF93DF93182FEB01FE01A2
:10BD80006491662329F0812F0E94AA5E2196F7CF45
:10BD9000DF91CF911F9108951F93CF93DF93182FB9
:10BDA000EB018881882369F08A3021F46DE0812FCE
:10BDB0000E94AA5E69916D30A1F3812F0E94AA5E54
:10BDC000F0CFDF91CF911F910895CF93DF93CDB73F
:10BDD000DEB79E01285F3F4F4E815F8160E470E0D7
:10BDE0008AEF92E10E94098C6AEF72E18D810E94D4
:10BDF000CC5EDF91CF910895CF93C82F8A3031F474
:10BE00006DE080913A130E94AA5E02C08D3029F045
:10BE10006C2F80913A130E94AA5E80E090E0CF914F
:10BE200008959DE0899FF0011124E356FD4F74872A
:10BE300063870895682F80E00C94AA5E80933A137C
:10BE40008FE892E09093C4308093C330089584B714
:10BE5000877F84BF88E10FB6F894809360001092CA
:10BE600060000FBE08952FE088E190E00FB6F894CF
:10BE7000A895809360000FBE209360000895A89558
:10BE8000089588E10FB6F8948093600010926000E6
:10BE90000FBE0895F89428E088E190E00FB6F8947A
:10BEA000A895809360000FBE20936000FFCF809123
:10BEB00062288091622890E0089540E06FE181E47B
:10BEC00091E00C94B164E9E3F1E0808180818D7FA1
:10BED00080838DE090E00197F1F723E040E06FE18F
:10BEE00082E491E00E94BB6483E090E00197F1F767
:10BEF00008959091390191FD0AC0282F803108F0F2
:10BF00002FE040E06FE085E491E00C94BB6408957D
:10BF10008091390181FD0EC040E06FE181E491E044
:10BF20000E94B164282F2F7E81E090E0213021F023
:10BF300080E0089580E090E008958091390181FDCE
:10BF400010C040E06FE181E491E00E94B1648F3164
:10BF500031F0982F9F7E915081E0923018F480E06C
:10BF6000089581E008950E949D5F8823E1F308957C
:10BF7000CF93DF93C82F0E94B35F0E945D5FD82FDD
:10BF8000C81789F1C83019F40E94635F25C0C93110
:10BF900021F4863189F429E005C0C63169F489317C
:10BFA00059F426E040E06FE182E491E00E94BB6436
:10BFB000E3E0F0E03197F1F72C2F40E06FE182E40D
:10BFC00091E00E94BB64D83019F4E9E6F1E002C0C8
:10BFD000E3E0F0E03197F1F70E945D5F8C1719F014
:10BFE00083E490E002C080E490E0DF91CF91089577
:10BFF0000E94B35F1092F7290E94635F809139011C
:10C0000082608093390180917A2A8823D9F18091C6
:10C0100094009091950040918B2A50918C2A84171E
:10C020009507A0F48091572A9091582AA091592AF7
:10C03000B0915A2A8C57914EAF4FBF4F8093572AD9
:10C040009093582AA093592AB0935A2A2091940089
:10C0500030919500241B350B8091572A9091582AD6
:10C06000A091592AB0915A2A820F931FA11DB11D88
:10C070008093572A9093582AA093592AB0935A2A0A
:10C0800010927A2A80917C2A8823D9F18091940099
:10C090009091950040918F2A5091902A841795078E
:10C0A000A0F480915F2A9091602AA091612AB091BA
:10C0B000622A8C57914EAF4FBF4F80935F2A909367
:10C0C000602AA093612AB093622A20919400309153
:10C0D0009500241B350B80915F2A9091602AA091D6
:10C0E000612AB091622A820F931FA11DB11D809316
:10C0F0005F2A9093602AA093612AB093622A1092DB
:10C100007C2A08958091F729882381F08091BE13BD
:10C11000811104C00E949D5F811106C081E080935F
:10C12000BC1381E090E008950E94F85F80E090E009
:10C13000089580919400909195009093902A809317
:10C140008F2A21E020937C2A8091390181FD08C04B
:10C150008091390181FD1AC086E10E94B85F16C046
:10C160002093F629809194009091950090938C2AC9
:10C1700080938B2A20937A2A809139018D7F809336
:10C1800039018091F6298111FCCFE2CF81E08093C3
:10C19000F72908958091F72981110AC08091BE1373
:10C1A000882321F081E08093BD1302C00E94996032
:10C1B00081E090E008951F93CF93DF931F92CDB756
:10C1C000DEB78FB789838091BE13811126C0F894A2
:10C1D0008091F729882351F08091390181FD1BC09E
:10C1E0000E949D5F8823B9F080E003C00E94CA606E
:10C1F00081E02091470191E02E3008F090E0192F66
:10C20000119581110E948260107429F089818FBF7D
:10C2100081E090E004C089818FBF80E090E00F90C2
:10C22000DF91CF911F9108958091BD13882321F054
:10C230000E9499601092BD138091BC13882321F055
:10C240000E94F85F1092BC131092BE1308950F93D2
:10C250001F93AB0121E02093BE1300913B2A109164
:10C260003C2A20913D2A30913E2A0F5F1F4F2F4FCD
:10C270003F4F00933B2A10933C2A20933D2A309352
:10C280003E2A22E0260F27FF0CC08091F4299091CE
:10C29000F52901969093F5298093F4290FEF1FEF6C
:10C2A00007C0BC018BE393E10E94CE8A00E010E05E
:10C2B0000E941461C8011F910F9108958093C013CB
:10C2C00008950E945D5F823011F0823111F480E0A8
:10C2D000089581E0089508958FEF80934E0122E044
:10C2E00044E060EF8CE691E00E94BB6425E041E011
:10C2F0006EE08CE290E00E94BB6480E880936F0166
:10C300008091460180936D0121E045E060E284E484
:10C3100091E00C94BB648DEF93E00197F1F70E94DC
:10C32000A76410926B281092ED2810926F2910923A
:10C330006A2810926928E9E3F1E080818E7F80838A
:10C3400080818D7F80838DE090E00197F1F7E9E3B4
:10C35000F1E080818160808323E040E06FE182E44E
:10C3600091E00E94BB648DEF93E00197F1F780911B
:10C370005D0180915E010E946C6160E070E087EB7E
:10C3800092E00E946A4D0E94996081E090E00895D9
:10C390008091BF130895CF93DF931F92CDB7DEB77F
:10C3A00089830E94B35F89818093BF13282F40E067
:10C3B0006FE188E491E00F90DF91CF910C94BB6422
:10C3C0000E94CB618091390181FD03C086E00C940D
:10C3D000B85F0895FA0180936201909363016093BE
:10C3E0006001709361013097C1F0808180936B018F
:10C3F000818180936A018281809369018381809326
:10C4000068018481809367018581809366018681BC
:10C4100080936501878180936401089587EB92E0A2
:10C420000E948B4D81E080936228809163289091D7
:10C4300064280196909364288093632881E090E0BB
:10C4400008951F93CF93DF9320916A2812E8129FDB
:10C4500090011124D901A559B74D4C91442309F4F9
:10C46000A6C05091390151FDA2C05091F729552322
:10C4700009F49DC047FF15C01C9280912B2A909112
:10C480002C2AA0912D2AB0912E2A0196A11DB11D12
:10C4900080932B2A90932C2AA0932D2AB0932E2A96
:10C4A00086C04330A8F41C928091272A9091282AB4
:10C4B000A091292AB0912A2A0196A11DB11D80932D
:10C4C000272A9093282AA093292AB0932A2A6FC05A
:10C4D00050E0EA0122976C177D07A8F41C92809126
:10C4E000232A9091242AA091252AB091262A0196E8
:10C4F000A11DB11D8093232A9093242AA093252A5D
:10C50000B093262A54C0B9016459774D0E94CE8A4F
:10C5100080916A28189FF0011124E559F74DDF0139
:10C52000A058BF4F9C9190935B2810828F5F8330FF
:10C5300018F480936A2802C010926A28E0916A2851
:10C5400082E8E89FF0011124E559F74D80818111BF
:10C550000E940E628091470180935C28909161282F
:10C56000992311F0891710F48093612860915C2859
:10C5700070E084E00E94155560915B2870E083E0D4
:10C580000E94155540913F2A5091402A6091412ABE
:10C590007091422A4F5F5F4F6F4F7F4F40933F2A0A
:10C5A0005093402A6093412A7093422A02C0C0E00F
:10C5B000D0E0CE01DF91CF911F910895CF93DF930B
:10C5C000EC01888199810097E9F08B3F944021F03C
:10C5D0001982188283E026C06238C1F41092622862
:10C5E0000E949C540E94035460E870E00E94216203
:10C5F000181619066CF40E94FE53E0914603F09160
:10C60000470309958BEF94E09983888381E00AC002
:10C6100080915F2890916028019690936028809384
:10C620005F28F0CFDF91CF91089591E09093BE13F2
:10C630000E94795F0C9414618091390181FD06C0DC
:10C6400040E06FE085E491E00C94B16480E10895EE
:10C650000F931F93CF93DF93182F21E02093BE13E6
:10C660000091F7298091390181FF16C080919400D3
:10C670009091950090938C2A80938B2A20937A2A0C
:10C680002093F629809139018D7F80933901809123
:10C69000F6298111FCCF00E00E94B35F8091F72959
:10C6A000882309F43FC080917C2A8823D9F18091A6
:10C6B000940090919500E0918F2AF091902A8E1726
:10C6C0009F07A0F440915F2A5091602A6091612AEF
:10C6D0007091622A4C57514E6F4F7F4F40935F2AA3
:10C6E0005093602A6093612A7093622A209194008B
:10C6F000309195002E1B3F0B40915F2A5091602A8C
:10C700006091612A7091622A420F531F611D711D51
:10C7100040935F2A5093602A6093612A7093622A43
:10C7200010927C2A8091390181FD03C089E10E9429
:10C73000B85F86E00E942055892B51F00E941C634F
:10C74000C82F86E00E94205581500E94795F02C068
:10C75000C0E0D0E0209194003091950030938E2A73
:10C7600020938D2A81E080937B2AF894809139016F
:10C77000826080933901809139018D7F80933901E6
:10C7800062E0610F8BE393E10E94EC647894209166
:10C79000F1293091F2292F5F3F4F3093F2292093F6
:10C7A000F1290E94B35F45E060EE82E491E00E94CF
:10C7B000B164182F86E00E942055892B19F08C2F28
:10C7C0000E94795F002319F00E94996002C00E94C4
:10C7D000F85F80917B2A8823D9F180919400909111
:10C7E0009500E0918D2AF0918E2A8E179F07A0F474
:10C7F00040915B2A50915C2A60915D2A70915E2A7B
:10C800004C57514E6F4F7F4F40935B2A50935C2A99
:10C8100060935D2A70935E2A209194003091950078
:10C820002E1B3F0B40915B2A50915C2A60915D2A40
:10C8300070915E2A420F531F611D711D40935B2A48
:10C8400050935C2A60935D2A70935E2A10927B2A33
:10C850008091F729882361F0209194003091950010
:10C860003093902A20938F2A81E080937C2A07C0FE
:10C8700023E040E06FE182E491E00E94BB640E940B
:10C8800014611130E9F01330A9F48091332A9091AA
:10C89000342AA091352AB091362A0196A11DB11DE6
:10C8A0008093332A9093342AA093352AB093362A62
:10C8B00012E009C0153031F0173029F411E003C03F
:10C8C00010E001C013E0812F90E0DF91CF911F9124
:10C8D0000F910895CF93DF93EB010E94276100979A
:10C8E00029F4CE010E942863009751F02091F42989
:10C8F0003091F5292F5F3F4F3093F5292093F4298C
:10C90000DF91CF910895CF93DF938091F729811123
:10C9100004C00E94CA60D1E001C0D0E00E945D5F07
:10C92000863111F0813119F4C091470109C040E00E
:10C930006FE186E491E00E94B164C82FCC0FC80F6C
:10C94000D1110E9482608C2FDF91CF9108951092B7
:10C95000C2131092C113EFE6F0E080818062808301
:10C960000895FC018081862390E002C0959587950B
:10C970004A95E2F70895F894FC015081362F3095DE
:10C980005323042E01C0220F0A94EAF72623522BC8
:10C9900050837894089540917B01FC014193A0E875
:10C9A000B1E050E8540F9D012F5F3F4F6C916193B0
:10C9B000521711F0D901F7CF4150E42FF0E0E058C1
:10C9C000FE4F2181FC01E058FF4F2083FC01EF570F
:10C9D000FF4F21E02083089560938001E1E8F1E0BA
:10C9E00061589F012F5F3F4FDC014D91CD01408386
:10C9F000621711F0F901F5CF08951F920F920FB64B
:10CA00000F9211240BB60F922F933F934F935F9386
:10CA10006F937F938F939F93AF93BF93EF93FF9306
:10CA20008091470180935C288091692822E8829F49
:10CA3000C00111248559974D0E94CB6480916928CB
:10CA40008F5F833018F48093692802C010926928A0
:10CA50000E940E62FF91EF91BF91AF919F918F91D4
:10CA60007F916F915F914F913F912F910F900BBEEE
:10CA70000F900FBE0F901F9018951F920F920FB638
:10CA80000F9211240F900FBE0F901F9018951F92B8
:10CA90000F920FB60F9211240F900FBE0F901F90A0
:10CAA00018951F920F920FB60F9211240F900FBE80
:10CAB0000F901F9018951F920F920FB60F9211248E
:10CAC0001092F6290F900FBE0F901F9018951F928D
:10CAD0000F920FB60F9211241092F6290F900FBEED
:10CAE0000F901F9018951F920F920FB60F9211245E
:10CAF0008F9381E0809362288F910F900FBE0F90EB
:10CB00001F9018951F920F920FB60F92112410923A
:10CB1000F6290F900FBE0F901F9018951F920F923D
:10CB20000FB60F9211248F939F938091C113909110
:10CB3000C21301969093C2138093C1139F918F915A
:10CB40000F900FBE0F901F901895CF92DF92EF922B
:10CB5000FF920F931F93CF93DF937C018B016A01A8
:10CB600083EC93E10E942A4EEC01009751F0EC8196
:10CB7000FD81309711F0C8010995CE010E94D24E77
:10CB8000F3CFA601B801C701DF91CF911F910F919B
:10CB9000FF90EF90DF90CF900C94B44B0F931F93C6
:10CBA000CF93DF9300D0CDB7DEB78091FF2990916E
:10CBB000002AA091012AB091022A0196A11DB11D5F
:10CBC0008093FF299093002AA093012AB093022A10
:10CBD0000E9438688C0183EC93E10E942A4E0097F2
:10CBE00079F0DC011296ED91FC911397309729F0C2
:10CBF00089839A8309959A8189810E94D24EEFCFC9
:10CC00000115110549F0C8010F900F90DF91CF91E8
:10CC10001F910F910C94AB4B0F900F90DF91CF9120
:10CC20001F910F9108950E942B6D0E949C540E94A9
:10CC30005F6682E393E09093FA298093F9290E943A
:10CC400036682FEF31E040E05EE160E074E082E0C2
:10CC500090E00C94FF67BC0183EC93E10C948A4E46
:10CC6000BC0183EC93E10C946F4ECF93DF93EC0106
:10CC70004091FB295091FC296091FD297091FE297A
:10CC80004F5F5F4F6F4F7F4F4093FB295093FC29BD
:10CC90006093FD297093FE290E944B68009761F014
:10CCA0000E941C54E0913603F0913703BE0185EADF
:10CCB00095E6099581E090E0DF91CF91089589ECA8
:10CCC00093E10C94264E0F93CF93DF93EC017B837B
:10CCD0006A8318865F834E83BC0189EC93E10E94CE
:10CCE0008A4EE091C513F091C613309749F04C81FC
:10CCF0005D8101E020E030E068858A819B810995B3
:10CD0000DF91CF910F910895BC0189EC93E10C94D0
:10CD10006F4E0F93DC0118961C921897E091C51383
:10CD2000F091C613309759F000E020E030E040E089
:10CD300050E060E012968D919C91139709950F91A8
:10CD400008950F93DC01AB0114962D913C9115973A
:10CD500081E018968C93189715967C936E93149790
:10CD6000E091C513F091C613309739F000E061E00F
:10CD700012968D919C91139709950F9108950F9399
:10CD8000DC01E091C513F091C613309771F0149651
:10CD90004D915C91159701E09A0118966C91189746
:10CDA00012968D919C91139709950F910895E0919A
:10CDB000C713F091C813309709F009940895909320
:10CDC000C8138093C71308959093C6138093C51317
:10CDD000089589EC93E10C942A4EEF92FF920F9301
:10CDE0001F93CF93DF938C01EB017A0189EC93E1E0
:10CDF0000E942A4E0097D9F0DC0112962D913C91A9
:10CE000013972C173D0781F41696ED91FC91179717
:10CE1000309769F09701AE01B801DF91CF911F9172
:10CE20000F91FF90EF9009940E94D24EE3CFDF91D3
:10CE3000CF911F910F91FF90EF9008950895CF9398
:10CE4000DF93CCEFD3E16881798120E030E04EE3DD
:10CE500057E686EE93E10E94AA500E94296D6881F0
:10CE600079810E94D58420E030E042E557E6BC019C
:10CE700086ED93E1DF91CF910C94AA508091FC1341
:10CE80009091FD132091FA133091FB13880F991F95
:10CE90002817390708F4C9019093FD138093FC13F8
:10CEA0000C941F67CF93DF930E949C540E940354FD
:10CEB000EC01198218820E94E96628813981009765
:10CEC00019F1FC0140854423F9F0FC0142815381B2
:10CED000F901EE0FFF1FEE0FFF1FEC0FFD1F538335
:10CEE0004283FC01448155812F5F3F4FF901EE0FD2
:10CEF000FF1FEE0FFF1FEC0FFD1F5183408339838F
:10CF000028830E94D24ED9CFC901880F991F880F5C
:10CF1000991F02960E94FE5388819981892B31F0D6
:10CF20008BEC93E1DF91CF910C94824BDF91CF9109
:10CF30000895AF92BF92CF92DF92EF92FF920F933C
:10CF40001F93CF93DF9300D0CDB7DEB76B010E9464
:10CF50000354FC01008111811A8309830C301105EF
:10CF600018F4E12CF12C0DC01F930F9384E099E08D
:10CF70009F938F930E94698B0F900F900F900F904B
:10CF800021C0E016F106F1F00E940354F701EE0F04
:10CF9000FF1FEE0FFF1FE80FF91FA280B3800E9452
:10CFA0000354FFEFEF1AFF0AF701EE0FFF1FEE0F1A
:10CFB000FF1FE80FF91F40815181B501C6010E9492
:10CFC000ED66DFCF0F900F90DF91CF911F910F9102
:10CFD000FF90EF90DF90CF90BF90AF9008950F93A8
:10CFE000013059F48091F6139091F7139093FD134B
:10CFF0008093FC130F910C941F670F910895EF928B
:10D00000FF920F931F93CF93DF938B01EA01790176
:10D010004FE153E0BC018BEC93E10E94664B10930F
:10D02000F7130093F613D093F913C093F813F0920B
:10D03000FB13E092FA138FEE97E6DF91CF911F91E9
:10D040000F91FF90EF900C94E46686EE93E10E94BE
:10D050002E5186ED93E10E942E518BEC93E10C94BE
:10D06000804B8091FC139091FD1308950C94C04B5C
:10D07000CF93DF93E0912303F09124030995EC0112
:10D08000009729F06A817B8181E00E941555CE01CD
:10D09000DF91CF9108950F931F93CF93DF93EC010E
:10D0A000E0912503F091260309958C016A817B812B
:10D0B00081E00E94155581E090E0012B11F480E0A1
:10D0C00090E0DF91CF911F910F910895E091270398
:10D0D000F0912803099420E030E00296FC01329799
:10D0E0004081442331F0FC0131974081240F311DF0
:10D0F000F4CFC9010895FC01208130E0322F2227AE
:10D100008181282B02C0220F331F6A95E2F7832FFB
:10D110009927FA01E75DFC4F208130E082239323B9
:10D1200028E030E0241B350B02C0969587952A95A0
:10D13000E2F708956F927F928F929F92AF92BF9283
:10D14000CF92DF92EF92FF920F931F93CF93DF93D3
:10D150008C01EB016A0179012830310524F4A90121
:10D16000B601CE014AC0590123E0B594A7942A958F
:10D17000E1F74115510521F04801612C712C03C0E4
:10D18000D801FB0120C048E050E0B601CE01860D79
:10D19000971D0E947B68F40181934F01FFEF6F1A86
:10D1A0007F0A6A147B047CF3C501B7FE02C080E0ED
:10D1B00090E0A701477055274115510511F1080F5F
:10D1C000191FB60118C0CF018C1B9D0B8A159B053A
:10D1D0001CF481918D93F7CFC501B7FE02C080E0AA
:10D1E00090E0A701477055274115510551F0080FF0
:10D1F000191F60E070E08C0F9D1F0E947B68F80192
:10D200008083DF91CF911F910F91FF90EF90DF907E
:10D21000CF90BF90AF909F908F907F906F90089528
:10D220008F929F92AF92BF92CF92DF92EF92FF9236
:10D230000F931F93CF93DF9300D0CDB7DEB70E943B
:10D2400003548C0182E090E00E94E153892B19F491
:10D2500080E090E05DC0F801818190E0982F882700
:10D260002081820F911D0E94D14B7C01009781F398
:10D270000E9403544C01F7012681822F86958695E2
:10D28000869590E0422F477021E030E011F420E0D5
:10D2900030E0820F931F0E94E153892BC9F2F701FE
:10D2A00004811581C12CD12CF8018081882379F16A
:10D2B000F801A180B12CB60133E0759567953A95D8
:10D2C000E1F7A60147705527680D791D883168F090
:10D2D0009501CE0101960E949A68BE016F5F7F4F53
:10D2E000F80180810E9429550DC01A82198295018A
:10D2F000CE0101960E949A6869817A81F801808145
:10D300000E941555CA0CDB1C0E5F1F4FCDCFC70105
:10D310000F900F90DF91CF911F910F91FF90EF90A1
:10D32000DF90CF90BF90AF909F908F900895DC01D9
:10D3300050E0E0E1F0E0E61BF70BE21BF30B02C06C
:10D34000440F551FEA95E2F78C91852B8C9311962B
:10D350008C911197842B11968C9308956F927F92E4
:10D360008F929F92AF92BF92CF92DF92EF92FF92F5
:10D370000F931F93CF93DF938C016B01EA01790127
:10D38000283031051CF44881C8015CC0390153E0E4
:10D39000759467945A95E1F76115710521F04E0176
:10D3A000A12CB12C03C0D801FE0127C0F40141918A
:10D3B0004F0128E030E0B601C8018A0D9B1D0E9494
:10D3C0009769FFEFAF1ABF0AA614B7047CF3C30135
:10D3D00077FE02C080E090E0970127703327211587
:10D3E000310509F43FC0C80FD91F488150E0B6018C
:10D3F000621B730B685F7F4F1CC0CF018C1B9D0BA2
:10D40000861597051CF481918D93F7CFC30177FEA4
:10D4100002C080E090E09701277033272115310585
:10D4200009F1C80FD91F488150E068E070E0621B25
:10D43000730B02C0559547956A95E2F760E070E07E
:10D44000800F911FDF91CF911F910F91FF90EF906F
:10D45000DF90CF90BF90AF909F908F907F906F9014
:10D460000C949769DF91CF911F910F91FF90EF90EE
:10D47000DF90CF90BF90AF909F908F907F906F90F4
:10D4800008956F927F928F929F92AF92BF92CF92A8
:10D49000DF92EF92FF920F931F93CF93DF9300D011
:10D4A000CDB7DEB78C01FC018681E82EE694E694C8
:10D4B000E694F12C282F277081E090E011F480E0B1
:10D4C00090E0E80EF91EC70102960E94655400978D
:10D4D00009F445C00E940A54F8012281FC0120830E
:10D4E000F8012381FC0121830E940A5402965C0109
:10D4F000A70160E070E00E94D78AF80104811581DD
:10D50000E12CF12CF8018081882339F1F801818028
:10D51000912C670163E0D594C7946A95E1F73701D0
:10D52000F7E06F227724CA0CDB1C883128F00E94B8
:10D5300033559401AC0108C00E9420559A83898319
:10D540009401AE014F5F5F4FB301C6010E94AE6907
:10D55000E80CF91C0E5F1F4FD5CF81E090E00F90D3
:10D560000F90DF91CF911F910F91FF90EF90DF907F
:10D57000CF90BF90AF909F908F907F906F900895C5
:10D58000E0914403F09145030994E0911D03F0916B
:10D590001E030994E0914803F09149030994E09136
:10D5A0004A03F0914B03099480E090E008950895B8
:10D5B000E0911503F0911603099480E090E008953E
:10D5C0000F931F93CF93DF93CDB7DEB7E0970FB6DE
:10D5D000F894DEBF0FBECDBF0E9450548C010E9454
:10D5E0000354AE014F5F5F4F602F0E94B0728823DB
:10D5F00009F446C088A99801281B3109C9010E9475
:10D60000E153892BE9F12E8121110CC0BE016A5E24
:10D610007F4F88E10E942955E0913803F09139034A
:10D6200009952EC08A859B858D3C3BEA930711F0B6
:10D63000019631F5223019F088E090E002C082E0D6
:10D6400090E001979C012F5F3F4F12161306F4F6EE
:10D65000E1E0F0E0EC0FFD1FE80FF91F23852F3FFD
:10D6600081F3BE01645F7F4F89E10E94295589E102
:10D670000E94335568E078E20E941F4B892B31F6F7
:10D68000E0960FB6F894DEBF0FBECDBFDF91CF910D
:10D690001F910F910895AF92BF92CF92DF92EF92B8
:10D6A000FF920F931F93CF93DF93CDB7DEB7E09731
:10D6B0000FB6F894DEBF0FBECDBF8C016B01CE015B
:10D6C00001967C0180E3F70111928A95E9F781E0E8
:10D6D00089838CE00E9420558C831D821F8280915B
:10D6E000001491E0980F90930014898783E0B82E7E
:10D6F000B8868DEC9BEA9B878A8789E10E94335527
:10D7000061EF72E00E941F4B892B31F082E08E8323
:10D710008FEF8C878D8709C089E10E943355BC014A
:10D72000CE010C960E94164BBE828DEC9BEA9D8B1F
:10D730008C8B68E078E2CE0146960E94164B0E94E0
:10D7400003549FA78EA70E94505488ABC7010E9424
:10D75000A971B82E90E00E946554892B31F10E9486
:10D760000A54BC014B2DC7010E94C771E0900B0306
:10D77000F0900C030E945A545C010E940A54B501B7
:10D78000F70109950115110581F0009739F001970E
:10D7900061F441E050E064E070E004C041E050E03A
:10D7A00060E070E0C601F8010995E0960FB6F894C4
:10D7B000DEBF0FBECDBFDF91CF911F910F91FF90C4
:10D7C000EF90DF90CF90BF90AF9008950E94296DA9
:10D7D00080930014E0911503F09116030994892BAE
:10D7E00029F0E0911503F091160304C0E0911703AE
:10D7F000F09118030994CF93DF93EC0189919991EB
:10D80000009729F060E070E00E946A4DF7CFDF9149
:10D81000CF910895CF93DF93EC018991999100976F
:10D8200019F00E94BC4CF9CFDF91CF910895CF93AE
:10D83000DF93EC017B836A830E94CF5D99838883A9
:10D84000DF91CF910895FC01808191812281338104
:10D85000820F931F918380830895CF93DF93EC0110
:10D860000E94CF5D99838883DF91CF910895CF93F4
:10D87000DF93EC010E94CF5D28813981821B930BDD
:10D880009C012F5F3F4F81E090E04A815B8142170E
:10D89000530710F080E090E0DF91CF910895CF938F
:10D8A000DF93FC01C281D38180819181C80FD91F90
:10D8B0000E94CF5D9E01281B390BC901DF91CF91DA
:10D8C0000895CF93DF93E1E8FAE2C3E4DAE2A5E753
:10D8D000BAE21192119219921992199219921D920B
:10D8E0008AE2E939F807A9F7DF91CF910895CF933C
:10D8F000DF93FC01EB58F54D40819C01220F331F53
:10D90000220F331F442301F1A0919400B0919500A0
:10D91000FC01EE0FFF1FEF57F54D80819181AD01A6
:10D92000481B590BCA01E901CD5BD54D488159818E
:10D930006A817B81480F591F611D711D488359837E
:10D940006A837B83B183A083F901ED5BF54D608130
:10D95000718182819381DF91CF91089560E070E0C1
:10D96000CB010895FC01EE0FFF1FEE0FFF1FED5BD3
:10D97000F54D40835183628373830895CF93DF9382
:10D9800025E73AE2C3E4DAE2E1E8FAE2D9018D916F
:10D990009D018823B9F040919400509195008081B9
:10D9A0009181BA01681B790B88819981AA81BB8119
:10D9B000860F971FA11DB11D88839983AA83BB83FE
:10D9C0005183408324963296BAE221383B07F1F620
:10D9D000DF91CF9108950C9438710F931F93FC0140
:10D9E000CB0140910114509102143383228315839B
:10D9F000048371836083F0930214E0930114452B38
:10DA000011F40E94527180E090E01F910F910895EF
:10DA100080910114909102140097C1F010920214A9
:10DA200010920114DC0114966D917C911597129659
:10DA3000ED91FC9113970995E0910114F091021476
:10DA4000309721F0808191810C94527108950C944B
:10DA500061870C945D8789EC92E00E94A14D81EC76
:10DA600092E00C94A14DCF93DF930E941054892B28
:10DA7000A9F081EC92E00E94BF4DEC01009721F1EA
:10DA80000E945054998388830E944B549B838A83BD
:10DA9000CE0104960E948C538CAB14C089EC92E0AA
:10DAA0000E94BF4DEC01009779F002960E949E53B0
:10DAB00099838883BE016E547F4FCE018E579F4F4E
:10DAC0000E94F354CE0102C080E090E0DF91CF913C
:10DAD0000895BC016E547F4F8E579F4F0C94F354A2
:10DAE000CF93DF93EC01BC0189EC92E00E94094ED8
:10DAF000BE01892B19F089EC92E009C081EC92E01B
:10DB00000E94094E892B39F0BE0181EC92E0DF9131
:10DB1000CF910C94E44DDF91CF9108950F931F9313
:10DB2000CF93DF93EC01BC0189EC92E00E94094E97
:10DB3000892B91F0FE0161917191CF010E94AF5448
:10DB4000BE016E547F4FCE018E579F4FDF91CF9114
:10DB50001F910F910C940455BE0181EC92E00E943C
:10DB6000094E892BD1F00E949C54688179818A8169
:10DB70009B810E94AF548CA990E00E9465540CA92F
:10DB800010E00E940A54BE016C5F7F4FA801DF9134
:10DB9000CF911F910F910C94CE8ADF91CF911F915D
:10DBA0000F910895CF93DF93EC01BC0189EC92E0D3
:10DBB0000E94094E892B19F0CE0102960CC0BE01BD
:10DBC00081EC92E00E94094E892B19F08A819B8199
:10DBD00002C080E090E0DF91CF910895FC01808148
:10DBE00091810895860F911D860F911D8E579F4F2D
:10DBF0000895860F911D860F911D8E579F4FFC0132
:10DC0000808191810895089580E69AE10E94E34F12
:10DC1000892B21F080E69AE10C94D04F0895E09191
:10DC20004C1AF0914D1A309709F0099480E008954C
:10DC3000EF92FF920F931F93CF93DF937C01EA0142
:10DC4000FC0180819181009741F08C30934071F10B
:10DC5000F7011182108283E0F2C080E024E0829F0D
:10DC6000F0011124E25BF54E118210828F5F843047
:10DC7000A8F380934B1A809186119091871190930D
:10DC80005F1A80935E1A0E94B54C8093992A60E4D3
:10DC900070E080E69AE10E94BC4F0E9426748CE0FE
:10DCA00093E0F7019183808381E0C9C06230D9F4A9
:10DCB00080919A2A90919B2A892B89F38091AB2A93
:10DCC000863029F48091C32A81FD0E94046E81E090
:10DCD0000E94647580919A2A90919B2A892BF9F26F
:10DCE0000E942870DCCF633060F5611114C020976A
:10DCF000B1F2D093A82FC093A72F83E00E94647540
:10DD000080919A2A90919B2A892B11F00E940F6E84
:10DD10000E94046EC4CF613011F6209709F4BFCF82
:10DD2000D093A42FC093A32F85E00E9464758091A7
:10DD30009A2A90919B2A892B09F4B1CF0E940F6EE9
:10DD4000AECF6738E9F510924A1A0EE41AE18091D5
:10DD50004A1A8430B8F4F801828193818C179D07A8
:10DD600049F4808191810E943175F80111821082FD
:10DD7000138212820C5F1F4F80914A1A8F5F80932B
:10DD80004A1AE5CFE2ECFFE2838194818C179D076C
:10DD900019F4148213821082B09620E3E234F20761
:10DDA00099F7EFE3F0E3818592858C179D0711F4D5
:10DDB000158214823D9680E3E13CF807A1F76FCF0E
:10DDC000683809F06CCFC056DA4109F068CF80E6B8
:10DDD0009AE10E94E34F892B09F461CF10924A1A0D
:10DDE000E0914A1AE43008F05ACF20E2E29FF001B5
:10DDF0001124E755F04D818D8823D9F080E69AE112
:10DE00000E94D04F80914A1AE0E28E9FC0011124F7
:10DE10008755904D9093A82F8093A72F82E00E9462
:10DE2000647580919A2A90919B2A892B11F00E9407
:10DE30000F6E80914A1A8F5F80934A1AD1CFDF917B
:10DE4000CF911F910F91FF90EF90089590934D1AED
:10DE500080934C1A0895209186113091871160E0CB
:10DE6000EEE4FAE1643098F4408151814817590793
:10DE700059F4428153814217530731F46093491A90
:10DE8000118210820C94317534966F5FEBCF6093E2
:10DE9000491A089540E0EEE4FAE14430A8F451E074
:10DEA000540F20813181232B61F44093481A9183D0
:10DEB00080832091861130918711338322830C94C3
:10DEC0004B753496452FE9CF4093481A0895209119
:10DED000861130918711FC01358F248F778F668FE3
:10DEE00008952091861130918711FC013287218796
:10DEF000748763870895CF93DF93EA010E94D474F7
:10DF0000009749F02091861130918711FC013287EA
:10DF10002187D487C387DF91CF9108950F931F93F3
:10DF2000CF93DF9300D000D0CDB7DEB78C01AB012B
:10DF30008FEF89838A838B838C83B801CE0101960E
:10DF40000E947B6F009719F0FC01158304830F90EA
:10DF50000F900F900F90DF91CF911F910F91089527
:10DF600040E050E062E081ED92E00E945B4D109253
:10DF70009B2A10929A2A0895AC0161E081ED92E00B
:10DF80000C943D4DAC0160E081ED92E00C943D4D70
:10DF90000F931F93CF93DF938A010E945274EC0179
:10DFA000009759F080918611909187119D8F8C8FE9
:10DFB0001F8F0E8FCE010E94C26FCE01DF91CF91D5
:10DFC0001F910F910895CF93DF93A091A72FB09148
:10DFD000A82F109719F0ED016C9605C0C091A32FE2
:10DFE000D091A42F29968091A22F86FF22C0109253
:10DFF000471A40E0EEE4FAE14430B8F42081318180
:10E0000014968D919C9115972817390759F48281A0
:10E010009381009739F04093471A998388831B8234
:10E020001A8205C034964F5FE7CF4093471A0E948B
:10E03000046E88819981009741F04A815B816091EB
:10E04000992ADF91CF910C945B4DDF91CF91089588
:10E050000F931F93CF93DF938091AB2A863009F003
:10E0600071C080919A2A90919B2A8115954009F060
:10E0700069C0C4E9D2E0D0939B2AC0939A2A02E0F7
:10E080000093A42A14E91093A52A1092C72A10928B
:10E09000C62A0E942074809590959093C72A8093F9
:10E0A000C62A1092AD2A1092AC2A0E940F74809555
:10E0B00090959093AD2A8093AC2A0E940F6ED093D6
:10E0C0009B2AC0939A2A0093A42A1093A52AA09170
:10E0D000A52FB091A62FFD01E459FD4F8CE692E0EB
:10E0E00001900D920197E1F76CE672E08AEB9AE2FB
:10E0F0000E94CE7380919E2A8093BA2A80919F2A93
:10E100008093BB2A8091A02A8093BC2A8091A12A67
:10E110008093BD2A1092C72A1092C62A0E942074AA
:10E12000809590959093C72A8093C62A1092AD2A25
:10E130001092AC2A0E940F74809590959093AD2A0E
:10E140008093AC2ADF91CF911F910F910C940F6EA9
:10E15000FC01680F791F80E048E1E617F70781F0BE
:10E16000219198E0322F3827532F517030FD8427AA
:10E170008695513009F480682695915099F7EDCF36
:10E1800008951F920F920FB60F9211240BB60F92A3
:10E190002F933F934F935F936F937F938F939F93AF
:10E1A000AF93BF93EF93FF9380919400909195006C
:10E1B0009093862A8093852A81E08093772A8091A4
:10E1C0007100807D809371000E94086D8091772A94
:10E1D0008823D9F180919400909195004091852AEF
:10E1E0005091862A84179507A0F480914B2A90912C
:10E1F0004C2AA0914D2AB0914E2A8C57914EAF4F88
:10E20000BF4F80934B2A90934C2AA0934D2AB093F2
:10E210004E2A2091940030919500241B350B80915B
:10E220004B2A90914C2AA0914D2AB0914E2A820FF0
:10E23000931FA11DB11D80934B2A90934C2AA0934C
:10E240004D2AB0934E2A1092772AFF91EF91BF91F9
:10E25000AF919F918F917F916F915F914F913F917E
:10E260002F910F900BBE0F900FBE0F901F9018951F
:10E270009FB7F894E1E7F0E08081807D808388B3E8
:10E280008F6288BB10929000E1E9F0E0108210925A
:10E290009200109295001092940080818560808396
:10E2A0009FBF08952FB7F89490939900809398009A
:10E2B00088B38F6288BBE1E7F0E080818260808371
:10E2C0002FBF0895CF93DF93FC01DB0185E0EB01C5
:10E2D00019928A95E9F78581837011F082E08C9319
:10E2E0008781837021F082E012968C93129785814A
:10E2F000837081F08781837069F0238934898185F7
:10E3000092852817390731F481E0848312961C9294
:10E31000129701C0148285818370823021F083308E
:10E3200021F080E003C082E001C088E011968C9368
:10E33000119787818370823021F0833021F080E053
:10E3400003C082E001C088E013968C93DF91CF91E7
:10E350000895CF93DF9300D000D01F92CDB7DEB7E2
:10E36000BE016F5F7F4F0E94627189819A81890F20
:10E370008D5F9B81890F9C81890F9D81890F0F90F3
:10E380000F900F900F900F90DF91CF9108954F92C3
:10E390005F926F927F928F929F92AF92BF92CF9235
:10E3A000DF92EF92FF920F931F93CF93DF9300D0F2
:10E3B00000D000D0CDB7DEB78C017B01BE016F5F0E
:10E3C0007F4F4E830E946271B981AA815B804C802D
:10E3D0008B2F90E003962A2F30E0820F931F850D3C
:10E3E000911D642D70E0860F971F5D81850F911D33
:10E3F0004E8150E0481759070CF49AC0F80181810A
:10E4000080FB662460F8712C43E0660C771C4A950B
:10E41000E1F7828180FB882480F8912C54E0880CFD
:10E42000991C5A95E1F7862880818770882A838114
:10E4300080FBAA24A0F8B12C85E0AA0CBB1C8A950D
:10E44000E1F78A28848180FBCC24C0F8D12C96E0A7
:10E45000CC0CDD1C9A95E1F78C28F7018082F8013D
:10E4600045814370F4E04F9FA0011124F80186819B
:10E470008370F0E18F9FC0011124482BF801878140
:10E48000F0E48F9FC0011124482BF7014183F8016C
:10E490008085F7018283B23059F4F8018185F70154
:10E4A0008383F8018285F701848395E0C92E02C039
:10E4B00083E0C82EB0E080E090E0200F311FDB2E1B
:10E4C000DC0C0197BA1761F0A901480F591FFA0136
:10E4D000B384A7014D0D511DFA01B082BF5FEFCF8C
:10E4E0009D2DF2E05F120EC0D701AD0DB11DF801F8
:10E4F00083898C9381E08D0DD701A80FB11D9E5F9C
:10E5000084898C9340E020E030E0060F171F842FB1
:10E51000890F21503109441561F0D801A20FB31FB2
:10E5200055965C91D701A80FB11D5C934F5FEFCF5B
:10E5300080E026960FB6F894DEBF0FBECDBFDF9108
:10E54000CF911F910F91FF90EF90DF90CF90BF90F0
:10E55000AF909F908F907F906F905F904F900895B5
:10E56000BF92CF92DF92EF92FF920F931F93CF93C0
:10E57000DF937C01D62EEA0182E0861708F0B2C054
:10E58000F701808186FBBB24B0F89181292F269565
:10E5900026952370C92EC294C694C69453E0C52212
:10E5A000382F3770388383FB332730F9398384FB66
:10E5B000332730F93A8385FB882780F98B83BC8227
:10E5C0002D83892F829583708E83CF828281888765
:10E5D000222391F13381848190E0982F8827830F43
:10E5E000911D9A87898787010B5F1F4F223079F42D
:10E5F00061EF72E0CE010B960E94164BF701868107
:10E600008B8785818C878701095F1F4F20C023304E
:10E61000F1F4F7013D9680E090E03E2F2F2F4291DC
:10E62000DE01A80FB91F1B964C9301968830910507
:10E63000B1F7032F122F0BC087010D5F1F4F61EF42
:10E6400072E0CE010B960E94164B1A861986CC20DA
:10E65000B9F1B1100DC0F8012081818190E0982FAF
:10E660008827820F911D9C8B8B8B0E5F1F4F04C0E0
:10E6700089859A859C8B8B8BF2E0CF120EC061EF5F
:10E6800072E0CE0145960E94164BF80181818D8B78
:10E6900080818E8B0E5F1F4F1BC0F3E0CF1218C01E
:10E6A000085F1F4FF80180E090E02291DE01A80F83
:10E6B000B91F55962C93019688309105B1F708C083
:10E6C00061EF72E0CE0145960E94164B1C8A1B8AB0
:10E6D000C8018E199F092D2D281B2FA71EA70DA736
:10E6E000D81608F480E0DF91CF911F910F91FF9031
:10E6F000EF90DF90CF90BF900895FB0141505109FA
:10E70000460F571FE417F50778F4208130E0322FC9
:10E7100022276181260F311D820F931F82179307D5
:10E7200008F401963296EECFE417F50751F42081F4
:10E7300030E0322F2227820F931F8217930708F4AD
:10E7400001960895CF93DF93C091A52AD0E06497F6
:10E750002091A42A30E0322F2227C20FD31F48E095
:10E7600050E06EEA7AE29E01280F311DC9010E9435
:10E770007D73AE0166EB7AE20E947D73009721F013
:10E7800098278927982702C08FEF9FEFDF91CF91BD
:10E7900008959093791A8093781A0895FC01538113
:10E7A000560F5093A12A872F99274281480F4093F3
:10E7B000A02AA181A0939F2AE081E0939E2A242F82
:10E7C00030E02817390748F481E08A0F80939F2AA8
:10E7D000811103C0EF5FE0939E2A852F90E0772799
:10E7E0008617970788F44F5F4093A02A41110CC009
:10E7F00080919F2A8F5F80939F2A811105C080910D
:10E800009E2A8F5F80939E2A0895AB01BC0180E011
:10E8100090E00E947D73982789279827089544E106
:10E8200050E062EA7AE280E090E00E947D73009717
:10E8300021F098278927982708958FEF9FEF089553
:10E8400086E00C94A27381E10C94A27380E0E82F1F
:10E85000F0E0EE0FFF1FE75DFF4C118210828F5F2B
:10E860008430A8F380E090E2899FF0011124E755FD
:10E87000F04D118E8F5F8430B0F380E094E0909380
:10E88000731A8093721A80E09DE0989FF001112422
:10E89000E15CFF4C158214828F5F8A30B0F3809365
:10E8A000711A0895CF932091721A3091731A2F5FC5
:10E8B0003F4F21154DE7340710F020E030E1522F93
:10E8C000432FE9EAFFE2C0E0C43059F0A18DAA234A
:10E8D00029F0A481B581A417B50749F3CF5FB0969D
:10E8E000F3CF3093731A2093721A1092711A20E0AA
:10E8F000E0E0F0E02430E8F430E2239FD00111247E
:10E90000A755B04D59963C915997311104C02093A9
:10E91000711AFD0110C0373041F4309739F05A9622
:10E920004C915A97328D341708F0DF012F5FFD01AB
:10E93000E1CF2093711A3097A1F122E0218F20912D
:10E94000741A24872091751A25872091761A2687B4
:10E950002091771A278728ED34E0338B228B358B73
:10E96000248B21E030E0318B208B138E21E0228F2D
:10E9700023E0208F168A20E1278B2091721A309194
:10E98000731A3227232732273583248377836683BC
:10E99000DC014D915D916D917C9140835183628347
:10E9A0007383CF01CF910895CF93DF932091721A93
:10E9B0003091731A2F5F3F4F21154DE7340710F048
:10E9C00020E030E1522F432FE3E4F0E3C0E0CA300F
:10E9D00041F0A081B181CF5F3D96A417B507B9F78B
:10E9E000E9CF3093731A2093721A40E05DE04A3009
:10E9F000A0F4A1E0A40F549FF0011124E15CFF4CAE
:10EA000024813581232B39F44093711A309741F4D6
:10EA100080E090E023C04A2FEACF4093711AF8CFEC
:10EA20002091721A3091731A3227232732273583A7
:10EA3000248377836683009729F4108211821282DF
:10EA4000138209C0EC0188819981AA81BB818083EE
:10EA50009183A283B38380E48087CF01DF91CF913C
:10EA6000089540E04430A0F4E42FF0E051E0540F6A
:10EA7000EE0FFF1FE75DFF4C20813181281739071A
:10EA800029F44093711A118210820895452FEACF1C
:10EA90004093711A089540E0443098F4E42FF0E078
:10EAA00051E0540FEE0FFF1FE75DFF4C20813181D5
:10EAB000232B29F44093711A918380830895452F65
:10EAC000EBCF4093711A0895AF92BF92CF92DF922D
:10EAD000EF92FF920F931F93CF93DF93C091A72FD5
:10EAE000D091A82F843009F4DCC12AEC3AE23093AB
:10EAF000A62F2093A52F30939D2A20939C2A833004
:10EB000059F4898D8F70833009F06BC08889998999
:10EB1000892B09F0DFC67FC0823009F080C0809168
:10EB2000771A8F5F8093771A811113C08091761ABC
:10EB30008F5F8093761A81110CC08091751A8F5F58
:10EB40008093751A811105C08091741A8F5F80932C
:10EB5000741A10929B2A10929A2A10923E301092A8
:10EB60003D30298D822F8D7F853041F48A8D8F5FD6
:10EB70008A8F843109F0AEC6198EACC6222309F4FF
:10EB8000A9C688899989892B09F441C08A8D9FEF8C
:10EB9000980F9A8F81119EC68B8D883031F09FEF30
:10EBA000920F923048F4853039F4198E80E88093C2
:10EBB000A22F0E94E36F47C5853038F493E0082EFA
:10EBC00001C0990F0A94EAF701C090E39A8F8F5F12
:10EBD0008B8F822F8F708330A1F048F4813009F43D
:10EBE0004FC3823009F076C61092C32A4CC38630D8
:10EBF00009F4C8C4883009F4C5C4843009F06AC671
:10EC0000C1C484E08093A22F0E94E36F4EC52F7091
:10EC1000233009F05FC688E08093A22F09C58530B4
:10EC200019F5E091A32FF091A42F84819581892B70
:10EC300009F450C61092A82F1092A72F8EEB9AE2DB
:10EC40009093A62F8093A52F90939D2A80939C2A22
:10EC500010923E3010923D3010929B2A10929A2AC8
:10EC600088E08093A22F1BC18091A22A853409F0ED
:10EC700031C60091A42A10E0102F00278091A52A08
:10EC8000080F111D80919A2A90919B2A8017910755
:10EC900008F420C610939B2A00939A2A8091A82AF0
:10ECA0008F7309F017C68091A92A811113C680912C
:10ECB000393090913A30C0914E03D0914F038C1768
:10ECC0009D0759F440913B3050913C3020915003C6
:10ECD0003091510342175307A1F02091B22A30918D
:10ECE000B32A2817390709F0F5C52091B42A3091C5
:10ECF000B52A80913B3090913C302817390709F0B4
:10ED0000E9C50E940F74019609F0E4C58091AB2A11
:10ED1000863009F429C18131E9F1813009F0DAC581
:10ED20008091B62A883009F0D5C51092B62A809114
:10ED3000B82A9091B92A873F3FEF930710F00996C0
:10ED400001C008969093B92A8093B82A8091AE2A80
:10ED50009091AF2AA091B02AB091B12A8093B22AA3
:10ED60009093B32AA093B42AB093B52A80913930F6
:10ED700090913A30A0913B30B0913C308093AE2AD4
:10ED80009093AF2AA093B02AB093B12A80E48093E5
:10ED9000AA2A7DC50C51110910939B2A00939A2A27
:10EDA0008EEB9AE29093A62F8093A52F8091BC2A98
:10EDB0009091BD2A892B29F00E942374019609F0B5
:10EDC00089C52091B82A3091B92A2115310509F455
:10EDD00081C58FE390E39093A42F8093A32FA090FD
:10EDE000B62AB090B72A40915003509151036091D8
:10EDF000520370915303A0915403B09155030091B5
:10EE0000AE2A1091AF2AE090B02AF090B12AE0919A
:10EE1000A32FF091A42F80E3E13CF80708F05AC536
:10EE200084819581009721F12817390709F586819A
:10EE30009781009719F0A816B906D1F480819181C5
:10EE40008C179D0729F4C280D380C416D506B1F073
:10EE50008617970729F4C280D380CA16DB0671F0A3
:10EE60000817190729F482819381E816F90631F011
:10EE70003D96F093A42FE093A32FC9CF1092A82F13
:10EE80001092A72F82E08093A22F8EEB9AE29093AC
:10EE90009D2A80939C2A10923E3010923D300E9411
:10EEA000E36F80913D3090913E30009709F412C598
:10EEB0009C01245E3F4F30939B2A20939A2A3093E3
:10EEC000A42A2093A52AE091A32FF091A42F2085B6
:10EED0002093AA2A21E12093AB2A08969827892714
:10EEE00098279093BB2A8093BA2A1092BD2A109239
:10EEF000BC2A848195819093B72A8093B62A868113
:10EF000097819093B92A8093B82A80913930909153
:10EF10003A30A0913B30B0913C308093AE2A909330
:10EF2000AF2AA093B02AB093B12A80819181A281A7
:10EF3000B3818093B22A9093B32AA093B42AB0935A
:10EF4000B52A8AEC9AE29093A62F8093A52F0E946F
:10EF5000237480959095009711F48FEF9FEF909315
:10EF6000BD2A8093BC2A93C40E942074019609F0A4
:10EF7000B1C48091B82A9091B92A009709F4AAC423
:10EF80002091B62A3091B72A2115310509F4A2C47F
:10EF90004091AE2A5091AF2A6091B02A7091B12A67
:10EFA000E2ECFFE2C9EADFE2F080FF20A9F0AC81E9
:10EFB000BD818A179B0781F4AE81BF812A173B0769
:10EFC00059F4A881B9814A175B0731F4AA81BB8142
:10EFD0006A177B0709F46FC1A096B096A0E3C93207
:10EFE000DA0711F72091C32A2F732230D9F49093B6
:10EFF0006F1A80936E1A40E0443090F4E42FF0E0F2
:10F00000EE0FFF1FE75DFF4C208131814F5F8217BC
:10F01000930791F71092711A20E0C0E0D0E07EC013
:10F020004093711A8091C32A82FD54C484E1809375
:10F03000C32A88E290E090939B2A80939A2A80E5E5
:10F040008093C22A8091BD2A9091C12A9093BD2AB3
:10F050003091BC2A9091C02A9093BC2A3093C02A48
:10F060002091BB2A9091BF2A9093BB2A2093BF2A5C
:10F070009091BA2A9093711A4091BE2A4093BA2A6D
:10F080009093BE2A8F5F8093C12A81110FC081E0C7
:10F09000830F8093C02A811109C081E0820F809381
:10F0A000BF2A811103C09F5F9093BE2A8091B62A28
:10F0B0009091B72A90936F1A80936E1A2091B82A74
:10F0C0003091B92A3093B72A2093B62A9093B92A5F
:10F0D0008093B82A8091AE2A9091AF2AA091B02A4D
:10F0E000B091B12A8093B22A9093B32AA093B42A04
:10F0F000B093B52A8091393090913A30A0913B304D
:10F10000B0913C308093AE2A9093AF2AA093B02A5E
:10F11000B093B12AA1C3373089F02F5F2430C0F4F7
:10F1200030E2239FC0011124FC01E755F04D318DE1
:10F130003111F1CF2093711AEF010CC0209721F00B
:10F14000428D3A8D341748F7EC01C755D04DE5CFC5
:10F150002093711A209709F4BDC3D093A82FC093B0
:10F16000A72F83E08A8F888F1E8A84E08F8B1B8E67
:10F170008091B82A9091B92A9D838C838091B62A78
:10F180009091B72A9F838E838091AE2A9091AF2A67
:10F19000A091B02AB091B12A88839983AA83BB83B6
:10F1A00081E0898F8091741A8C878091751A8D8780
:10F1B0008091761A8E878091771A8F8781E090E010
:10F1C000998B888B8091BD2A8B878091BC2A8A87F6
:10F1D0008091BB2A89878091BA2A888781E090E054
:10F1E0000E94CE7C8091C22A282F207F30E02135DA
:10F1F00031050CF445C082958F7090E00597880F1B
:10F20000991F880F991F3091701A20E0E22FF0E0CB
:10F21000E817F9078CF5EE55F54D30A5311105C00D
:10F220002093711A1092701A2BC0313011F42F5F95
:10F23000EDCF3230E1F441A54430C9F42093711A86
:10F240003093701A82A590E0982F882723A5822BEF
:10F2500090936F1A80936E1A893DA4E09A0710F07C
:10F2600088ED94E09B8B8A8B9D8B8C8B09C041A58C
:10F27000442311F0240FCACF2093711A3093701ACF
:10F2800080E18093C32A8091C32A82608093C32A3D
:10F2900082E08093CA2A84E08093CB2A8093CC2A90
:10F2A00088ED8093CD2A8CE290E090939B2A809306
:10F2B0009A2A80E67EC2D093A82FC093A72F1092DF
:10F2C000A22F9091C32A92FF03C0198E80E21AC226
:10F2D0008091C22A82958F70880F880F8093711A4F
:10F2E000081B11090451110910939B2A00939A2AB3
:10F2F0008F2D8F70823029F4892F8F73823139F4EA
:10F300001FC0813021F4892F8F738230C9F0012B07
:10F3100019F4892F8370A1F02091BA2A88852813C7
:10F320003EC22091BB2A8985281339C22091BC2A6C
:10F330008A85281334C22091BD2A8B8528132FC2B9
:10F3400094FF4AC0688979896115710509F444C040
:10F35000CE010C960E94CE733091BE2A80919E2AD7
:10F3600038133AC02091BF2A80919F2A281334C0B5
:10F370009091C02A8091A02A98132EC08091C12A12
:10F380004091A12A841328C03C872D879E878F87B0
:10F390008B8D81111AC02E89888D9A8D891B922F91
:10F3A000969596959695891B280F2E8B87FD8195AE
:10F3B0009F89392F36953695931B980F9F8B822FF7
:10F3C000869586958695890F888F81E08093A22FF8
:10F3D000888D8A8F198A188A498D842F8F7090E0C2
:10F3E000FC013197E830F10508F074C2E057FF4F97
:10F3F0000C9499868091A22F80FF14C083E0898F9E
:10F4000080E48093A22F198A188A80919A2A909179
:10F410009B2A009709F408C122E42093A22F0E949E
:10F42000CE7C02C18091C32A8F73823009F052C210
:10F4300027CF8091A22F80FF70C08091C32A8F7345
:10F44000823109F06AC08091C22A282F207F30E0E3
:10F45000213531050CF445C082958F7090E00597F9
:10F46000880F991F880F991F3091701A20E0E22FA2
:10F47000F0E0E817F9078CF5EE55F54D30A53111A0
:10F4800005C02093711A1092701A2BC0313011F4FC
:10F490002F5FEDCF3230E1F441A54430C9F4209321
:10F4A000711A3093701A82A590E0982F882723A5AF
:10F4B000822B90936F1A80936E1A893D24E09207F5
:10F4C00010F088ED94E09B8B8A8B9D8B8C8B09C010
:10F4D00041A5442311F0240FCACF2093711A309311
:10F4E000701A83E0898F8091BA2A88878091BB2A1D
:10F4F00089878091BC2A8A878091BD2A8B8781E089
:10F5000090E00E94CE7C82E48093A22F198A188A10
:10F5100010929B2A10929A2A87C080E28093A22F91
:10F520000E94E36FE091A72FF091A82F118E7ACD62
:10F530008091C32A80FF28C044FD26C0888999890C
:10F54000892B09F0C7C180919A2A90919B2A019634
:10F550000E94CE7C2091A22F822F80618093A22FC7
:10F5600080919A2A90919B2A892B19F022612093ED
:10F57000A22F0E94E36F81E090E0998B888B88E056
:10F58000898F1B8E81E10CC185FF1CC08091C82A28
:10F5900090E0982F88272091C92A822B2091A52FAF
:10F5A0003091A62F280F391F3093A62F2093A52F17
:10F5B00020919A2A30919B2A281B390B30939B2A41
:10F5C00020939A2A80919A2A90919B2A009749F039
:10F5D00044FD07C02091A22F22602093A22F0E94F9
:10F5E000CE7C8091C42A90E0982F88272091C52A4C
:10F5F000820F911D90936F1A80936E1A2C893D890A
:10F600002817390710F0892B21F430936F1A2093B3
:10F610006E1A80916E1A90916F1A9B8B8A8B8091D3
:10F62000A22F837009F456C110923E3010923D30E3
:10F630000E94E36F8091A22F85FF07C010923E3099
:10F6400010923D30198E84E1ABC084FF0AC0109245
:10F650003E3010923D3081E090E0998B888B84E0C1
:10F660008FCF20913D3030913E3021153105E1F0B2
:10F6700080FF02C0198A188A88899989009781F4C5
:10F680008A899B898217930720F490933E30809358
:10F690003D3080913D3090913E30998B888B04C0F5
:10F6A00090933E3080933D301B8E80919C2A9091A8
:10F6B0009D2A9093A62F8093A52F80913D30909105
:10F6C0003E30892B59F088899989009739F08896BE
:10F6D00090939B2A80939A2A88E10BC08091A22F55
:10F6E00081FFF8C088E290E090939B2A80939A2A49
:10F6F00080E18093C32A5CC08091A22F80FFEAC082
:10F70000198E80E18093A22F0E94E36FE3C0809165
:10F710009A2A90919B2A009711F00E94CE7C90919A
:10F72000C32A8091A22F90FF0BC080FF06C087E004
:10F73000898F1A8E198A188A19C086E0898F16C097
:10F7400080FF1EC085E0898F198A188AC3C0809106
:10F750009A2A90919B2A009711F00E94CE7C80916A
:10F76000C32A80FF0DC087E0898F1A8E81E090E068
:10F770000E94CE7C80E18093A22F0E94E36F0FC095
:10F7800080919A2A90919B2A892B49F4A3C0809159
:10F79000A22F80FF9FC087E0898F1A8E9BC080E1D7
:10F7A0008093C32A88E290E090939B2A80939A2AC0
:10F7B00080E58093C22A88858093BE2A89858093BC
:10F7C000BF2A8A858093C02A8B858093C12A8C8525
:10F7D0008093BA2A8D858093BB2A8E858093BC2A1C
:10F7E0008F858093BD2A86E08093AB2A8C819D8192
:10F7F0009093B72A8093B62A8E819F819093B92ADD
:10F800008093B82A8091393090913A30A0913B3062
:10F81000B0913C308093AE2A9093AF2AA093B02A47
:10F82000B093B12A88819981AA81BB818093B22A41
:10F830009093B32AA093B42AB093B52A898D84FFFC
:10F8400005C01092C52A1092C42A06C084E0809395
:10F85000C42A88ED8093C52A80E48093AA2A8091E7
:10F860009A2A90919B2A9093A42A8093A52A109279
:10F87000C92A1092C82A1092C72A1092C62A0E943A
:10F880002074809590959093C72A8093C62A85E42A
:10F890008093A22A1092A32A1092A92A1092A82A31
:10F8A0008091781A9091791A01969093791A8093A1
:10F8B000781A9093A62A8093A72A1092AD2A1092C4
:10F8C000AC2A0E940F74809590959093AD2A8093F6
:10F8D000AC2A04C010929B2A10929A2A1092A22F4E
:10F8E000DF91CF911F910F91FF90EF90DF90CF901C
:10F8F000BF90AF90089598278927982708950E9470
:10F900009F860895FC0180919C2A90919D2A22EA6D
:10F910003FE2281B390BAB01261737070CF4A9016E
:10F920001416150654F450933E3040933D30E817BA
:10F93000F90719F0BF010C94CE8A089580E88093EE
:10F940006100109261000E94635B0E94D24C0E9491
:10F950003F5F8091492890914A28009729F00197AC
:10F9600090934A2880934928C0904B28D0904C28E7
:10F97000E0904D28F0904E280E94FD5DC616D706F7
:10F98000E806F90611F30E94FD5D60934B28709321
:10F990004C2880934D2890934E28D7CF2091A72FA5
:10F9A0003091A82FBC01C90108960E94CE73E09146
:10F9B000A72FF091A82F80919E2A808780919F2A5F
:10F9C00081878091A02A82878091A12A83870895C8
:10F9D0002F923F924F925F926F927F928F929F925F
:10F9E000AF92BF92CF92DF92EF92FF920F931F934D
:10F9F000CF93DF93CDB7DEB763970FB6F894DEBF32
:10FA00000FBECDBF7C011B016A01FC01178216826B
:10FA1000838181FF66C3BE016F5F7F4F4B01F7019A
:10FA20009381F10193FD859193FF81911F018823BB
:10FA300009F453C3853239F493FD859193FF819185
:10FA40001F01853239F4B70190E00E94378B5601CF
:10FA50006501E5CF10E0512C20E02032A0F48B327C
:10FA600069F030F4803259F0833269F420612CC09F
:10FA70008D3239F0803339F4216026C02260246051
:10FA800023C0286021C027FD27C030ED380F3A3051
:10FA900078F426FF06C0FAE01F9F300D1124132FC3
:10FAA00013C06AE0569E300D1124532E20620CC004
:10FAB0008E3221F426FD11C3206406C08C3611F469
:10FAC000206802C0883641F4F10193FD859193FFCF
:10FAD00081911F018111C1CF9BEB980F933018F4D6
:10FAE0002061805E06C09BE9980F933008F0AAC1A0
:10FAF0002F7E26FF16E02F73722E853621F4F22F0B
:10FB0000F0647F2E08C0863621F4622F6068762E5E
:10FB100002C01111115077FE07C01C3348F4442471
:10FB20004394410E27E00BC0183030F4212F06C05B
:10FB300027E04CE3442E03C027E017E0412C560198
:10FB400074E0A70EB11CF6016081718182819381FE
:10FB5000042DA4010E94D6896C01098100FF02C016
:10FB600003FF06C071FC07C072FC08C0612C08C00E
:10FB70003DE2632E05C02BE2622E02C090E2692EA8
:10FB8000802F8C7099F1662011F084E001C083E031
:10FB9000851510F0512C0BC0581A73FC08C0B70122
:10FBA00080E290E00E94378B5A94C9F7F3CF662029
:10FBB00029F0B701862D90E00E94378B03FD03C02A
:10FBC0000FE410E102C00BE410E1F72DF0717F2E7D
:10FBD000F8018491882309F476C271108052B7012C
:10FBE00090E00E94378B0F5F1F4FF2CF77FE0FC060
:10FBF0004C0C04FF04C08A81813309F44A94141424
:10FC000074F5F8E0F41578F588E0482E2CC076FC01
:10FC10002AC0812F90E08C159D059CF06CEFC616D4
:10FC20006FEFD60674F0772D7068772E0AC0E2E089
:10FC3000F0E0EC0FFD1FE10FF11D8081803319F41E
:10FC400011501111F4CF77FE0EC044244394410E9D
:10FC5000812F90E0C816D9062CF41C1904C0442446
:10FC6000439401C010E077FE07C01C141D043CF44F
:10FC700096012F5F3F4F05C025E030E002C021E034
:10FC800030E0662011F02F5F3F4F112331F0412FFC
:10FC900050E04F5F5F4F240F351F452D50E0241774
:10FCA000350714F4521A01C0512C872D897049F47C
:10FCB000552039F0B70180E290E00E94378B5A94CA
:10FCC000F7CF662029F0B701862D90E00E94378B90
:10FCD00073FC09C0552039F0B70180E390E00E9421
:10FCE000378B5A94F7CF77FE5FC09C2D8D2DD7FEB2
:10FCF00002C090E080E0692E782E40E050E0C6011E
:10FD0000841991099D878C87960126193709280D3A
:10FD1000391D812F90E0EE27FF27E81BF90BFF87A5
:10FD2000EE87FFEF6F167F0669F4B7018EE290E071
:10FD30002B8B3A8B488B598B0E94378B598948897A
:10FD40003A892B89C614D70454F06C857D856615D5
:10FD500077052CF4F901E40FF51F818101C080E3E0
:10FD600071E0671A71084F5F5F4FEE85FF856E1671
:10FD70007F066CF0B70190E02B8B3A8B488B598B48
:10FD80000E94378B2B893A8948895989CACF6C14CC
:10FD90007D0439F49A81963318F4953311F404FFF5
:10FDA00081E3B70190E04BC08A81813309F00F7E77
:10FDB000B70190E00E94378B111105C074FE18C086
:10FDC00085E490E017C0B7018EE290E00E94378B87
:10FDD00082E066246394680EF401E80FF11D8081CF
:10FDE000B70190E00E94378B115041F3862DF1CF7F
:10FDF00085E690E0B7010E94378BD7FC05C0C1149F
:10FE0000D10439F404FF05C0D194C194D1088DE226
:10FE100001C08BE2B70190E00E94378B80E36AE07B
:10FE2000C616D1042CF08F5FFAE0CF1AD108F7CFB5
:10FE3000B70190E00E94378BB701C601C0960E94BF
:10FE4000378B41C1833631F0833779F0833509F040
:10FE500058C021C0560172E0A70EB11CF601808186
:10FE6000898301E010E0640114C05601F2E0AF0E96
:10FE7000B11CF601C080D18026FF03C0612F70E065
:10FE800002C06FEF7FEFC6012B8B0E94FD8A8C01B1
:10FE90002B892F7715C05601F2E0AF0EB11CF60189
:10FEA000C080D18026FF03C0612F70E002C06FEFD9
:10FEB0007FEFC6012B8B0E94BF8A8C012B892068A3
:10FEC000722E23FD1AC0852D90E008171907A8F49B
:10FED000B70180E290E00E94378B5A94F4CFF6018C
:10FEE00077FC859177FE81916F01B70190E00E94C8
:10FEF000378B51105A94015011090115110579F7EA
:10FF0000E2C0843611F0893651F5560127FF09C049
:10FF1000F4E0AF0EB11CF6016081718182819381A2
:10FF20000AC0F2E0AF0EB11CF60160817181882732
:10FF300077FD8095982F022F0F7697FF08C0909538
:10FF40008095709561957F4F8F4F9F4F00682AE095
:10FF500030E0A4010E94428CC82EC8183EC0022F77
:10FF6000853721F40F7E2AE030E01DC0097F8F36EF
:10FF700091F018F4883559F0B0C0803719F08837FF
:10FF800011F0ABC0006104FF09C0046007C024FF8A
:10FF900008C0066006C028E030E005C020E130E07F
:10FFA00002C020E132E0560107FF09C0F4E0AF0EC5
:10FFB000B11CF601608171818281938108C0F2E0F9
:10FFC000AF0EB11CF6016081718180E090E0A40168
:10FFD0000E94428CC82EC8180F7706FF0BC0202F36
:10FFE0002E7FC11650F404FF0AC002FD08C0202F66
:10FFF0002E7E05C0DC2C202F03C0DC2C01C0D12EAE
:020000021000EC
:1000000024FF0DC0FE01EC0DF11D8081803311F441
:10001000297E09C022FF06C0D394D39404C0822F46
:10002000867809F0D39423FD13C020FF06C01C2D51
:10003000D51418F4150D1D19D52CD51468F4B70175
:1000400080E290E02B8B0E94378BD3942B89F5CFE5
:10005000D51410F45D1801C0512C24FF12C0B70153
:1000600080E390E02B8B0E94378B2B8922FF17C0F7
:1000700021FF03C088E590E002C088E790E0B70167
:100080000CC0822F867859F021FD02C080E201C0A9
:100090008BE227FD8DE2B70190E00E94378BC116FD
:1000A00038F4B70180E390E00E94378B1150F7CF0E
:1000B000CA94F401EC0DF11D8081B70190E00E941B
:1000C000378BC110F5CF552009F4C2CCB70180E2BF
:1000D00090E00E94378B5A94F6CFF7018681978182
:1000E00002C08FEF9FEF63960FB6F894DEBF0FBE8E
:1000F000CDBFDF91CF911F910F91FF90EF90DF90D7
:10010000CF90BF90AF909F908F907F906F905F90B7
:100110004F903F902F9008955058BB27AA270ED09C
:100120004EC23FD230F044D220F031F49F3F11F460
:100130001EF4FFC10EF4E095E7FBF5C1E92F50D2A4
:1001400080F3BA17620773078407950718F071F4F4
:100150009EF568C20EF4E0950B2EBA2FA02D0B0170
:10016000B90190010C01CA01A0011124FF27591BFC
:1001700099F0593F50F4503E68F11A16F040A22F02
:10018000232F342F4427585FF3CF46953795279573
:10019000A795F0405395C9F77EF41F16BA0B620B72
:1001A000730B840BBAF09150A1F0FF0FBB1F661FB9
:1001B000771F881FC2F70EC0BA0F621F731F841FFC
:1001C00048F4879577956795B795F7959E3F08F022
:1001D000B3CF9395880F08F09927EE0F97958795E1
:1001E0000895DFD158F080E891E009F49EEFE0D166
:1001F00028F040E851E059F45EEF09C09AC112C2FC
:10020000E92FE078EDD168F3092E052AC1F326170E
:1002100037074807590738F00E2E07F8E02569F030
:10022000E025E0640AC0EF6307F8009407FADB01F9
:10023000B9019D01DC01CA01AD01EF9347D0BFD1E7
:100240000AD05F91552331F02BED3FE049E450FD9A
:1002500049EC63CF0895DF93DD27B92FBF7740E8DE
:100260005FE31616170648075B0710F4D92FE1D194
:100270009F938F937F936F9346D3E0E3F1E06CD12C
:100280009ED12F913F914F915F919AD2DD2349F0FA
:100290009058A2EA2AED3FE049EC5FE3D0785D2771
:1002A0004DDFDF918CC11BD108F481E008950CD0A3
:1002B00086C17ED140F075D130F021F45F3F19F056
:1002C00032C15111B0C135C18BD198F39923C9F313
:1002D0005523B1F3951B550BBB27AA27621773074C
:1002E000840738F09F5F5F4F220F331F441FAA1F00
:1002F000A9F333D00E2E3AF0E0E830D091505040C0
:10030000E695001CCAF729D0FE2F27D0660F771F6D
:10031000881FBB1F261737074807AB07B0E809F04F
:10032000BB0B802DBF01FF2793585F4F2AF09E3FE4
:10033000510568F0F8C077C15F3FECF3983EDCF3FD
:10034000869577956795B795F7959F5FC9F7880F5D
:10035000911D9695879597F90895E1E0660F771FAF
:10036000881FBB1F621773078407BA0720F0621B40
:10037000730B840BBA0BEE1F88F7E095089519F400
:100380000EF0D1C04FC1D5C033D1C8F39638C0F7F5
:1003900007F80F92E8942BE33AEA48EB5FE712D2B2
:1003A0000F920F920F924DB75EB70F92CAD1EDE543
:1003B000F1E0D2D04F915F91EF91FF91E595EE1F63
:1003C000FF1F49F0FE57E0684427EE0F441FFA95DF
:1003D000E1F74195550B36D10F9007FE2AC10895DC
:1003E00097FB0EF4A9D03EC0E89409C097FB3EF4F9
:1003F00090958095709561957F4F8F4F9F4F992372
:10040000A9F0F92F96E9BB279395F69587957795EF
:100410006795B795F111F8CFFAF4BB0F11F460FFAF
:100420001BC06F5F7F4F8F4F9F4F16C0882311F007
:1004300096E911C0772321F09EE8872F762F05C01B
:10044000662371F096E8862F70E060E02AF09A95B6
:10045000660F771F881FDAF7880F9695879597F9AB
:100460000895E894F92F96EBFF2381F012161306F6
:100470001406440B9395F695879577956795579550
:100480004040FF23B9F71BC099270895882351F4F2
:100490009850D2F7872B762F652F542F432F322F6A
:1004A00020E0B1F3121613061406440B88233AF029
:1004B0009A95440F551F661F771F881FCAF755234B
:1004C0004AF4440F551F11F460FF04C06F5F7F4F63
:1004D0008F4F9F4F880F9695879597F90895990F9D
:1004E0000008550FAA0BE0E8FEEF16161706E807FE
:1004F000F907C0F012161306E407F50798F0621B1F
:10050000730B840B950B39F40A2661F0232B242BF3
:10051000252B21F408950A2609F4A140A6958FEF12
:10052000811D811D089597F99F6780E870E060E064
:1005300008959FEF80EC0895909580957095609553
:1005400050954095309521953F4F4F4F5F4F6F4FDE
:100550007F4F8F4F9F4F0895DF93CF931F930F933C
:10056000FF92EF92DF927B018C01689405C0DA2E36
:10057000EF0126D1FE01E894A59125913591459191
:100580005591AEF3EF01DADDFE019701A801DA948F
:1005900079F7DF90EF90FF900F911F91CF91DF914E
:1005A000089500240A9416161706180609060895D9
:1005B00000240A9412161306140605060895092E3F
:1005C0000394000C11F4882352F0BB0F40F4BF2BAE
:1005D00011F460FF04C06F5F7F4F8F4F9F4F0895EE
:1005E00057FD9058440F551F59F05F3F71F04795E4
:1005F000880F97FB991F61F09F3F79F087950895C9
:10060000121613061406551FF2CF4695F1DF08C0E7
:10061000161617061806991FF1CF86957105610504
:1006200008940895E894BB2766277727CB0197F9AC
:1006300008959B01AC0160E070E080E89FE337CE55
:1006400072CF64C1D5DFE8F39923D9F3940F511D1C
:10065000BBF39150504094F059F0882332F0660F6C
:10066000771F881F91505040C1F79E3F510544F7B6
:10067000880F911D9695879597F908955F3FACF087
:10068000983E9CF0BB27869577956795B79508F4BB
:10069000B1609395C1F7BB0F58F711F460FFE8CF35
:1006A0006F5F7F4F8F4F9F4FE3CFBDCF0AD029EDB4
:1006B0003BE54EED5EE378C00EF028C13ACF68947A
:1006C00032CF96DFC8F39923D1F3C6F3DF93CF93EC
:1006D0001F930F93FF92C92FDD2788232AF02197BC
:1006E000660F771F881FDAF720E030E040E85FEB05
:1006F0009FE3883920F0803E30F021968F770DDD22
:10070000E5E8F1E003C009DDE2EBF1E025DF8B0174
:10071000BE01EC01FB2E6F5771097595771F880B91
:10072000990B64DE28E132E741E35FE349D0AF2D66
:100730009801AE01FF900F911F91CF91DF91FEDCE8
:100740003ECFFA01DC01AA0FBB1F9B01AC01BF57D2
:1007500028F422273327442750781FC0B75188F444
:10076000AB2F0024469537952795011CA395D2F30E
:10077000002069F0220F331F441FB395DAF30DD028
:10078000CBCC61307105A0E88A07B94630F49B01F3
:10079000AC016627772788279078309621F0208350
:1007A00031834283538308950BD009CFFADE28F0BA
:1007B000FFDE18F0952309F0B6CEBBCE112433CF5F
:1007C0000FDFA0F3959FD1F3950F50E0551F629F67
:1007D000F001729FBB27F00DB11D639FAA27F00D9A
:1007E000B11DAA1F649F6627B00DA11D661F829FC1
:1007F0002227B00DA11D621F739FB00DA11D621FA6
:10080000839FA00D611D221F749F3327A00D611DC2
:10081000231F849F600D211D822F762F6A2F1124A4
:100820009F5750408AF0E1F088234AF0EE0FFF1FF7
:10083000BB1F661F771F881F91505040A9F79E3F2E
:10084000510570F070CEEFCE5F3FECF3983EDCF3D5
:10085000869577956795B795F795E7959F5FC1F76B
:10086000FE2B880F911D9695879597F90895FA01AB
:10087000EE0FFF1F30962105310599F161157105C5
:1008800061F48038BFE39B0749F168949038810593
:1008900061F08038BFEF9B0741F0992342F5FF3F9D
:1008A000E1053105210511F1E8940894E795D90196
:1008B000AA2329F4AB2FBE2FF85FD0F310C0FF5F3F
:1008C00070F4A695E0F7F73950F019F0FF3A38F4D4
:1008D0009F779F930CD00F9007FC905808953EF09F
:1008E00028CE60E070E080E89FE308954FE79F77AF
:1008F0005F934F933F932F93E4DE2F913F914F915E
:100900005F9152DF41CD9B01AC014ECF9F3F31F053
:10091000915020F4879577956795B795880F911D2D
:100920009695879597F908950E949C84332312F435
:100930008A1B9B0B0C94AD84A29FB001B39FC00196
:10094000A39F700D811D1124911DB29F700D811DFB
:100950001124911D08950E949C84B7FF0895821B65
:10096000930B08950E949C84A59F900DB49F900DB9
:10097000A49F800D911D11240895B7FF0C94B2849B
:100980000E94B284821B930B0895DB018F939F9387
:100990000E94B284BF91AF91A29F800D911DA39F31
:1009A000900DB29F900D11240895AA1BBB1B51E11D
:1009B00007C0AA1FBB1FA617B70710F0A61BB70BCF
:1009C000881F991F5A95A9F780959095BC01CD0174
:1009D000089597FB072E16F4009407D077FD09D0F1
:1009E0000E94D58407FC05D03EF4909581959F4FD9
:1009F0000895709561957F4F0895A1E21A2EAA1B64
:100A0000BB1BFD010DC0AA1FBB1FEE1FFF1FA217BE
:100A1000B307E407F50720F0A21BB30BE40BF50BBB
:100A2000661F771F881F991F1A9469F76095709544
:100A3000809590959B01AC01BD01CF010895052ED5
:100A400097FB1EF400940E944A8657FD07D00E942F
:100A5000FD8407FC03D04EF40C944A8650954095D3
:100A6000309521953F4F4F4F5F4F0895689401C0D7
:100A7000E894F92FF12B12F00C946A85A0E0B0E015
:100A8000E4E4F5E80C946886092E059422F40E94AB
:100A90005286112392F4F0E80F26FFEFE094F094D1
:100AA00000951095B094C094D094A194BF0ACF0A39
:100AB000DF0AEF0AFF0A0F0B1F0B0E94F98507FCE4
:100AC0000E945286CDB7DEB7ECE00C948486689421
:100AD00001C0E8948F929F92CF93DF930E94F98593
:100AE000DF91CF919F908F900895DF93CF931F93C5
:100AF0000F939A9DF02D219FF00D8B9DF00D8A9DF7
:100B0000E02DF10D039FF00D029FE00DF11D4E9DB4
:100B1000E00DF11D5E9DF00D4F9DF00D7F936F93E5
:100B2000BF92AF925F934F93D5010E949C848B013B
:100B3000AC01D7010E949C84EB01E80FF91FD6019C
:100B40000E94C5852F913F91D6010E949C84C60FBB
:100B5000D71FE81FF91FAF91BF910E94C5852F9144
:100B60003F910E949C84C60FD71FE81FF91FD60132
:100B70000E949C84E60FF71F9801BE01CF0111244B
:100B80000F911F91CF91DF9108950E949C84460F91
:100B9000571FC81FD91F08F431960895E894DF93B2
:100BA000CF93FC01DB010E949C847F936F93E9014A
:100BB0009A01AC01BF93AF933F932F93DF010E9443
:100BC0009C8426F46C1B7D0B820B930B9E01EB0126
:100BD000FC010E94C585AF91BF912F913F910E946A
:100BE000C585BE01CF01F9012F913F91CF91DF91D2
:100BF000089588249924F401E401B0E49F93AA277E
:100C00009A158B049C04ED05FE05CF05D007A107BE
:100C100098F4AD2FDC2FCF2FFE2FE92D982C892EA5
:100C2000982F872F762F652F542F432F322F22276F
:100C3000B85031F7BF9127C01B2EBF91BB27220FA1
:100C4000331F441F551F661F771F881F991F881C5D
:100C5000991CEE1FFF1FCC1FDD1FAA1FBB1F8A148C
:100C60009B04EC05FD05CE05DF05A007B10748F0A4
:100C70008A189B08EC09FD09CE09DF09A00BB10B0E
:100C800021601A94E1F62EF49401AF01BE01CD016A
:100C9000000C089590958095709561957F4F8F4FCA
:100CA0009F4F0895609570958095909530954095EB
:100CB000509521953F4F4F4F5F4F6F4F7F4F8F4F55
:100CC0009F4F08952F923F924F925F926F927F9223
:100CD0008F929F92AF92BF92CF92DF92EF92FF924C
:100CE0000F931F93CF93DF93CDB7DEB7CA1BDB0BF8
:100CF0000FB6F894DEBF0FBECDBF09942A8839889D
:100D000048885F846E847D848C849B84AA84B984A3
:100D1000C884DF80EE80FD800C811B81AA81B981AF
:100D2000CE0FD11D0FB6F894DEBF0FBECDBFED01C3
:100D30000895EE0FFF1F0590F491E02D09946927A7
:100D40009627692778278727782708950F930830F3
:100D500090F0982F872F762F652F542F432F322F07
:100D600022270850F4CF220F331F441F551F661F40
:100D7000771F881F991F0A95B2F70F91089597FB67
:100D800010F8169400080F93083098F00850232F9D
:100D9000342F452F562F672F782F892F902DF4CF82
:100DA00005949795879577956795579547953795C6
:100DB00027950A95AAF70F9108952A0D3B1D4C1D02
:100DC0005D1D6E1D7F1D801F911F08950024A7FDCE
:100DD00000942A0F301D401D501D601D701D801D88
:100DE000901D08952A193B094C095D096E097F0978
:100DF000800B910B08952A153B054C055D056E058A
:100E00007F058007910708950024A7FD00942A1705
:100E10003005400550056005700580059005089572
:100E20008F929F92AF92BF92CF92DF92EF92FF92FA
:100E3000CF93DF93EC01688179818A819B81611571
:100E400071058105910521F464E279ED8BE597E068
:100E50002DE133EF41E050E00E941F8549015A0126
:100E60009B01AC01A7EAB1E40E94B2846B017C0152
:100E7000ACEEB4EFA50194010E94C084C60ED71E4B
:100E8000E81EF91EF7FE06C081E0C81AD108E10885
:100E900080E8F80AC882D982EA82FB82C6019F777D
:100EA000DF91CF91FF90EF90DF90CF90BF90AF9008
:100EB0009F908F9008950C9410878BED92E00C9486
:100EC0001087A0E0B0E08093DB029093DC02A09357
:100ED000DD02B093DE0208952F923F925F926F92EF
:100EE0007F928F929F92AF92BF92CF92DF92EF92BA
:100EF000FF920F931F93CF93DF938B01EA0161154C
:100F0000710521F0DB018C9311969C93209739F0A9
:100F10009E01225031092332310508F0FBC07C01CB
:100F20006701BFEFCB1ADB0A5601F7016080862DFF
:100F300090E00E94AE8A892B11F07601F1CFFDE29C
:100F40006F120AC0570182E0A80EB11CD70111969A
:100F50006C90772473940BC0BBE26B1207C05701EF
:100F6000E2E0AE0EB11CD70111966C90712CCE014F
:100F70008F7E892B89F4B0E36B1222C0F50180814A
:100F80008F7D883541F56180F2E0AF0EB11C872D71
:100F90008260782EC0E1D0E0C830D105F1F04CF489
:100FA000C230D10511F5C12CD12CE12CB0E4FB2EBF
:100FB0002FC0CA30D10531F0C031D10521F115C0A3
:100FC000209751F7CAE0D0E0ACECCA2EDC2CEC2C18
:100FD000ACE0FA2E1DC02097F9F6C8E0D0E0C12C95
:100FE000D12CE12CF0E1FF2E13C060E070E080E036
:100FF00090E89E01442737FD4095542F0E94FD84C0
:1010000069017A0105C0C12CD12CE12CE8E0FE2E4B
:10101000F50160E020E030E0A9014E01AA2497FC30
:10102000A094BA2C1F0170ED572E560CA9E0A515FF
:1010300070F48FEB860D8A3118F499EC592E06C0A6
:101040008FE9860D8A3130F589EA582E560C852DA8
:1010500090E08C179D07F4F467FD18C0C216D30604
:10106000E406F50680F0C501B4010E94C5849B0129
:10107000AC01250D311D411D511D213031054105AA
:10108000B0E85B0710F06FEF01C061E03196D1016D
:101090006C90C8CF872D81700115110571F0662302
:1010A00029F03197D801ED93FC9307C071FE19C068
:1010B0003297D801ED93FC9314C067FF12C08823C8
:1010C00029F020E030E040E050E804C02FEF3FEF8F
:1010D0004FEF5FE782E290E09093C8308093C73093
:1010E00016C0882341F050954095309521953F4F8B
:1010F0004F4F5F4F0CC057FF0AC082E290E09093C1
:10110000C8308093C7302FEF3FEF4FEF5FE7B90153
:10111000CA0104C060E070E080E090E0DF91CF9110
:101120001F910F91FF90EF90DF90CF90BF90AF9005
:101130009F908F907F906F905F903F902F90089539
:101140002F923F925F926F927F928F929F92AF9277
:10115000BF92CF92DF92EF92FF920F931F93CF93A4
:10116000DF938B01EA016115710521F0DB018C939E
:1011700011969C93209739F09E0122503109233219
:10118000310508F0D8C07C016701BFEFCB1ADB0A3C
:101190005601F7016080862D90E00E94AE8A892B6F
:1011A00011F07601F1CFFDE26F120AC0570182E023
:1011B000A80EB11CD70111966C90772473940BC0C4
:1011C000BBE26B1207C05701E2E0AE0EB11CD701C3
:1011D00011966C90712CCE018F7E892B89F4B0E32F
:1011E0006B1237C0F50180818F7D8835D1F4618025
:1011F000F2E0AF0EB11C872D8260782EC0E1D0E006
:10120000CA30D10551F1C031D10521F0C830D10526
:1012100099F409C0CC24CA94DC2CEC2CAFE0FA2E53
:1012200022C0209769F7C8E0D0E0CC24CA94DC2C17
:10123000EC2CFFE1FF2E17C06FEF7FEFCB019E017B
:10124000442737FD4095542F0E94FD8469017A019F
:101250000AC02097A9F6CAE0D0E0E9E9CE2EDC2C3E
:10126000EC2CE9E1FE2EF50160E020E030E0A90180
:101270004E01AA2497FCA094BA2C1F0170ED572EA2
:10128000560CA9E0A51570F48FEB860D8A3118F481
:1012900099EC592E06C08FE9860D8A3148F589EA06
:1012A000582E560C852D90E08C179D070CF56F3F3E
:1012B000D9F0C216D306E406F50698F0C501B401CC
:1012C0000E94C5849B01AC01852D90E0A0E0B0E0B8
:1012D000280F391F4A1F5B1F281739074A075B076A
:1012E00010F46FEF01C061E03196D1016C90C5CF71
:1012F0000115110551F0662311F0319703C071FEFD
:1013000004C03297D801ED93FC9370FE07C050954E
:101310004095309521953F4F4F4F5F4F67FF10C06D
:1013200082E290E09093C8308093C7306FEF7FEFF8
:101330008FEF9FEF07C060E070E080E090E002C0B8
:10134000B901CA01DF91CF911F910F91FF90EF90EA
:10135000DF90CF90BF90AF909F908F907F906F90D5
:101360005F903F902F900895662777270C94DB8C31
:10137000FC0188279927E89421912032E9F329304C
:1013800010F02E30C8F32B3241F02D3239F468942E
:1013900004C00E942F8B820F911D219120532A306F
:1013A000C0F31EF4909581959F4F0895283008F062
:1013B00027E03327DA01990F311D87FD91600096F0
:1013C0006105710539F432602E5F3D9330E32A9553
:1013D000E1F708959F3F30F080387105610509F00D
:1013E0003C5F3C5F3D93913008F08068911DDF9336
:1013F000CF931F930F93FF92EF92192F987F96959B
:10140000E92F96959695E90FFF27E355FF4E99270B
:101410003327EE24FF24A701E701059008940794E1
:1014200028F4360FE71EF81E491F511D660F771F5F
:10143000881F991F0694A1F70590079428F4E70EDA
:10144000F81E491F561FC11D770F881F991F661F61
:101450000694A1F70590079428F4F80E491F561F2B
:10146000C71FD11D880F991F661F771F0694A1F70C
:101470000590079420F4490F561FC71FD81F990FD6
:10148000661F771F881F0694A9F78491109517701F
:1014900041F0D695C79557954795F794E7941A95D7
:1014A000C1F7E3E5F0E168941590159135916591E8
:1014B000959105907FE27395E118F10A430B560B65
:1014C000C90BD009C0F7E10CF11E431F561FC91FFD
:1014D000D01D7EF4703311F48A95E6CFE894015064
:1014E00030F0080F0AF40027021708F4202F239584
:1014F000022F7A3328F079E37D932A95E9F710C01B
:101500007D932A9589F60694979567953795179553
:101510001794E118F10A430B560BC90BD00998F048
:1015200023957E9173957A3308F070E37C932013B2
:10153000B8F77E9170617D9330F0839571E37D9370
:1015400070E32A95E1F71124EF90FF900F911F911E
:10155000CF91DF91992787FD909508959111A8C3A8
:10156000803219F089508550D0F70895FB01DC01D5
:101570008D91059080190110D9F3990B0895FC0104
:101580000590615070400110D8F7809590958E0FAE
:101590009F1F08954AE75AE10C94088BFB01DC0178
:1015A00002C001900D9241505040D8F70895DC01DF
:1015B00001C06D9341505040E0F70895FB01DC01FC
:1015C0008D91019080190110D9F3990B0895FB01B9
:1015D000DC0101900D920020E1F70895FB01DC0190
:1015E0004150504048F001900D920020C9F701C0D1
:1015F0001D9241505040E0F70895FC016150704049
:1016000001900110D8F7809590958E0F9F1F089537
:10161000FA01A191B081009719F41097E1F0CD0182
:10162000DC01CD010D90002011F4C00113C0FB01BD
:101630002191222319F02015D9F7F3CFFB01219135
:10164000201519F41E92119606C02223C1F70D90A1
:101650000020A1F7D001FA01A193B08308957AE0A8
:10166000979F902D879F802D910D112408950F93A2
:101670001F93CF93DF93182F092FEB018B8181FDEF
:1016800003C08FEF9FEF20C082FF10C04E815F81AB
:101690002C813D81421753077CF4E881F9819F0139
:1016A0002F5F3F4F39832883108306C0E885F98573
:1016B000812F0995892B29F72E813F812F5F3F4F7D
:1016C0003F832E83812F902FDF91CF911F910F9118
:1016D0000895CF93DF93CDB7DEB7FE0135966191C4
:1016E0007191AF018091C3309091C4300E94E87C29
:1016F000DF91CF9108950F931F93CF93DF93CDB7D1
:10170000DEB7FE0137966191719103EC10E3D801C9
:101710008D919C91DC0113962C9113972860139660
:101720002C93AF010E94E87CD801ED91FC912381BC
:10173000277F2383DF91CF911F910F9108950F93FE
:101740001F93CF93DF93E091C330F091C430238196
:1017500021FF1BC0EC0100E010E089916091C330D3
:101760007091C430DB011896ED91FC911997882394
:1017700031F00995892B89F30FEF1FEFEECF8AE047
:101780000995892B11F4C80102C08FEF9FEFDF91FB
:10179000CF911F910F9108950F931F93CF93DF93D4
:1017A000CDB7DEB72E970FB6F894DEBF0FBECDBF14
:1017B0000D891E898F89988D26E02C831A830983D1
:1017C00097FF02C080E090E801979E838D83AE0171
:1017D000455E5F4F698D7A8DCE0101960E94E87C4F
:1017E0004D815E8157FD0AC02F813885421753070E
:1017F0000CF49A01F801E20FF31F10822E960FB637
:10180000F894DEBF0FBECDBFDF91CF911F910F9136
:1018100008950F931F93CF93DF93CDB7DEB72E9725
:101820000FB6F894DEBF0FBECDBF8C01CA0146E0F3
:101830004C831A83098377FF02C060E070E861502F
:1018400071097E836D83A901BC01CE0101960E94BE
:10185000E87C4D815E8157FD0AC02F813885421793
:1018600053070CF49A01F801E20FF31F10822E9631
:101870000FB6F894DEBF0FBECDBFDF91CF911F91A1
:101880000F910895FA01AA27283051F1203181F1F2
:10189000E8946F936E7F6E5F7F4F8F4F9F4FAF4F78
:1018A000B1E03ED0B4E03CD0670F781F891F9A1F8B
:1018B000A11D680F791F8A1F911DA11D6A0F711D3F
:1018C000811D911DA11D20D009F468943F912AE04B
:1018D000269F11243019305D3193DEF6CF01089533
:1018E000462F4770405D4193B3E00FD0C9F7F6CF64
:1018F000462F4F70405D4A3318F0495D31FD40522C
:10190000419302D0A9F7EACFB4E0A69597958795C1
:1019100077956795BA95C9F70097610571050895A0
:101920009B01AC010A2E069457954795379527954C
:10193000BA95C9F7620F731F841F951FA01D0895E4
:10194000DC01CB01FC01F999FECF06C0F2BDE1BD7F
:10195000F89A319600B40D9241505040B8F708956E
:10196000F999FECF92BD81BDF89A992780B5089567
:10197000A8E1B0E042E050E00C94A28CDC01CB0185
:1019800003C02D910E94C98C41505040D0F708955A
:10199000262FF999FECF1FBA92BD81BD20BD0FB68B
:1019A000F894FA9AF99A0FBE019608950E94C88C8D
:1019B000272F0C94C98C4F925F926F927F928F92D7
:1019C0009F92AF92BF92CF92DF92EF92FF920F93CE
:1019D0001F93CF93DF938B016115710521F0DB011C
:1019E0008C9311969C93EC015E01BFEFAB1ABB0A7E
:1019F0007501C8808C2D90E00E94AE8A892B11F071
:101A0000E501F2CFEDE2CE1208C07E01F2E0EF0E6A
:101A1000F11CC980DD24D39409C02BE2C21205C099
:101A20007E0142E0E40EF11CC980D12CE701219730
:101A300043E050E065E571E1CE010E945B8E892BA9
:101A4000D1F4E701229645E050E060E571E1CE0176
:101A50000E945B8E892B11F4E70127960115110571
:101A600019F0D801CD93DC93D11008C160E070E08B
:101A700080E89FE70CC143E050E06DE471E1CE01E6
:101A80000E945B8E892B59F40115110509F4FBC0E6
:101A9000B2E0EB0EF11CF801F182E082F4C0F70134
:101AA00060E070E0CB01C0E0D0E07F01A0EDAA2EA5
:101AB000AC0C29E02A1530F14D2D4260B42E2D2DAD
:101AC0002870D2FE04C0211125C0219623C0211107
:101AD0002197A5E0B0E09B01AC010E94B284660FA3
:101AE000771F881F991F6A0D711D811D911D68390F
:101AF000A9E97A078A07A9E19A0760F0BD2DB660C7
:101B0000BB2E08C02EEFA2120AC0D3FC50C04D2D30
:101B10004860B42E3196D701CC90DB2CC6CF2C2D4B
:101B20002F7D253409F043C0A081AD3241F4BD2D95
:101B3000B061DB2E7F0122E0E20EF11C0CC07F01C0
:101B4000AB3231F04FEFE41AF40A21E030E006C086
:101B5000A2E0EA0EF11CA18122E030E0A053AA30FD
:101B600018F0E21AF30A23C0F70120E030E0203831
:101B7000BCE03B075CF4A901440F551F440F551FFF
:101B8000240F351F220F331F2A0F311DAF014F5F66
:101B90005F4F7A01A081A053AA3010F4FA01E7CF79
:101BA000D4FE03C0319521953109C20FD31FD1FE58
:101BB00009C00115110531F0E1E0EE1AF108D80174
:101BC000ED92FC920E94F4812D2D2370233019F0A8
:101BD0006B017C0106C06B017C01F7FAF094F7F809
:101BE000F09420E030E0A901C701B6010E945381C2
:101BF000882309F440C0D7FF06C0D195C195D1090B
:101C00000CE611E102C004E811E14801B8E18B1AC9
